:100000000C94A40A0C94D50A0C94D50A0C94D50A25
:100010000C94D50A0C94D50A0C94D50A0C94D50AE4
:100020000C94D50A0C94D50A0C94D50A0C94D50AD4
:100030000C94D50A0C94BE7E0C94D50A0C94D50A67
:100040000C94D50A0C94D50A0C94D50A0C94D50AB4
:100050000C94D50A0C94D50A0C94D50A0C94939C54
:100060000C94D50A0C9483590C945A590C94D50AC3
:100070000C94D50A0C94D50A0C94D50A0C94D50A84
:100080000C94D50A0C94D50A0C94D50A0C94D50A74
:100090000C9430590C9407590C94D50A0C94D27FC7
:1000A0000C94D50A0C94D50A0C94D50A0C94D50A54
:1000B0000C94D50A0C94D50A0C94D50A0C94D50A44
:1000C0000C94D50A0C94D50A0C94D50A0C94DD58DE
:1000D0000C94B4580C94D50A0C948A580C9461581A
:1000E0000C94D50A021CE91C511C4A1C1A1C0A1C3F
:1000F000E91C061CE91CE91CE91CE91CE91C610B54
:10010000CA0B5B0C980DA00D7A0F34105211F4122B
:10011000F0134F1464146814E91CAA14AE141916D1
:10012000D417EE1715197419501AD01AD71AC31B01
:10013000D1426A437C4385438E439743A943B243EC
:10014000E143F343FC4305440E44A944B244BB4499
:100150002A872D871C8720872687648731873587E4
:100160003B873F87438749874D87518764875787F8
:100170005B875F87084AD73B3BCE016E84BCBFFDDF
:10018000C12F3D6C74319ABD56833DDA3D00C77F67
:1001900011BED9E4BB4C3E916BAAAABE0000008000
:1001A0003F07634236B79BD8A71A39685618AEBACC
:1001B000AB558C1D3CB7CC5763BD6DEDFD753EF660
:1001C000177231BF000000803F08000000BE92247B
:1001D00049123EABAAAA2ABECDCCCC4C3E000000B0
:1001E00080BEABAAAAAA3E00000000BF00000080AB
:1001F0003F0000000000084178D3BB4387D1133D86
:10020000190E3CC3BD4282AD2B3E68EC8276BED94E
:100210008FE1A93E4C80EFFFBE01C4FF7F3F00008D
:10022000000000004E414E494E495459494E46CDBA
:10023000CCCC3D0AD7233C17B7D13877CC2B32959D
:1002400095E6241FB14F0A000020410000C842007B
:10025000401C4620BCBE4CCA1B0E5AAEC59D740045
:10026000407A10F35A00A0724E18090010A5D4E885
:100270000000E87648170000E40B54020000CA9A18
:100280003B000000E1F5050000809698000000406A
:10029000420F000000A086010000001027000000AF
:1002A00000E803000000006400000000000A0000F5
:1002B0000000000100000000002C76D888DC674FA9
:1002C0000823DFC1DFAE59E1B1B796E5E3E453C6D9
:1002D0003AE651997696E8E6C28426EB898C9B62D1
:1002E000ED407C6FFCEFBC9C9F40F2BAA56FA5F47B
:1002F00090055A2AF75C936B6CF9676DC11BFCE0A3
:10030000E40D47FEF520E6B500D0ED902E030094F5
:100310003577050080841E080000204E0A0000008A
:10032000C80C333333330F986E12831141EF8D2194
:1003300014893BE65516CFFEE6DB18D1844B381BFB
:10034000F77C1D901DA4BBE424203284725E2281C0
:1003500000C9F124ECA1E53D274D6F74696F6E0073
:10036000555620496E742E00555620496E74656EA0
:1003700073697479004F3220436F6E6300434F32CC
:1003800020436F6E630053656E736F7220657272E7
:100390006F722100234E6F2073656E736F722100A0
:1003A000434F3220436F6E63004D65617375726910
:1003B0006E6700234E6F2073656E736F7220666FD9
:1003C0007220504D21004E6F2073656E736F722145
:1003D00000206E672F4C00504D313A322E353A31A5
:1003E00030004D6561737572696E672E2E00234E65
:1003F0006F2054422073656E736F723F00234E6FFF
:100400002073656E736F722100536F756E64204C9C
:100410006576656C004D6561737572696E672E2E29
:1004200000234E6F2073656E736F722100536F75DA
:100430006E64204C6576656C00234E6F2073656E8C
:10044000736F7220666F722074656D70202620684D
:10045000756D696469747921004E6F2053656E7300
:100460006F72210020666F722074656D70202620E7
:1004700068756D696469747921002353656E736FC3
:1004800072204572726F72200053656E736F722016
:100490004572726F7221002357726F6E6720736509
:1004A0006E736F7220666F722074656D70202620E7
:1004B00068756D6964697479210057726F6E672081
:1004C00053656E736F72210054656D702048756DB1
:1004D0006964697479004C6967687420496E746551
:1004E0006E7369747900466C616D652049520048ED
:1004F0002D6669656C6400536561726368204469A8
:1005000072656374696F6E00234E6F2070482073AC
:10051000656E736F72210070482076616C7565009E
:1005200023496E76616C6964206B65792100204DEA
:10053000756C746973656E736F7273004D756C744E
:100540006973656E736F72730044697361626C6581
:1005500000456E61626C65005265626F6F74696E12
:10056000672E2E2E002344413A2D3233002372652C
:10057000706C6965733D002353657474696E6773AD
:10058000206F6620616C6C2073656E736F72733AB6
:10059000002353697A65206F66206865616465721F
:1005A000202B20616C6C2073656E736F72733A2020
:1005B000002353697A65206F6620686561646572FF
:1005C0003A20002320616E64207265616479207492
:1005D0006F207573652100206D6F62696C65206CFA
:1005E0006F6767657220737461727465642000437D
:1005F000616C6962726174696F6E205072657373A9
:100600007572653D00536561206C6576656C2050A0
:100610002863616C63293D00234572726F723A70E2
:100620007265737375726520424D503038352C20D9
:10063000636865636B20776972696E672100495250
:100640002054656D702073656E736F7220666F75D0
:100650006E6400504D322E352073656E736F7220BC
:100660006C696B656C7920666F756E6400206D6FC8
:1006700062696C65206C6F67676572207374617264
:10068000746564202E2E2E2000576946692049503B
:100690003A002357694669204950206164647265B5
:1006A00073733A2000456455484B205345534C6FB3
:1006B000676765720053656E736F7220736C6F7439
:1006C00020616E6420747970653A0057656C636FC1
:1006D0006D6520746F20456455484B0023456E645A
:1006E000206F66204D756C746973656E736F722030
:1006F0004379636C6523002354696D6520647572CA
:100700006174696F6E3D002354696D6520696E7474
:10071000657276616C3D00576946692049503A0020
:10072000234D5320456E61626C656400234D532058
:1007300044697361626C6564002352657374207050
:100740006172616D657465727320746F2064656693
:1007500061756C742076616C756573004C6F6767AA
:100760006572204E616D653A2000696E7075742067
:1007700044535463616C6962726174653A00207617
:100780006F6C746167653D002354757262696469BA
:100790007479205570706572204C696D69743A20C7
:1007A0000020766F6C746167653D0023547572623A
:1007B0006964697479204C6F776572204C696D6942
:1007C000743A200023547572626964697479204C0C
:1007D0006F776572204C696D69742056696E663A50
:1007E00020004D61782072616E67653D0023566F71
:1007F0006C746167652073656E736F723A00342D97
:1008000032306D4100414353373132204D61783DE4
:1008100000414353373132204D61783D354100234B
:1008200043757272656E742073656E736F723A00F1
:1008300023445320546865726D6F6D657465722032
:1008400063616C6962726174656420666F722023F3
:1008500000234E6F206E65656420746F2063616CA9
:100860006962726174652063757272656E7420735B
:10087000656E736F72210023414353373132206319
:10088000757272656E742073656E736F72206F6619
:100890006673657420563D00235556207A65726F45
:1008A00020766F6C74616765203D00234F3220769F
:1008B0006F6C253D00234F322063616C6962726169
:1008C00074696F6E3A200023566F6C7461676528F7
:1008D00070483D3130293A0023566F6C746167656A
:1008E0002870483D34293A0067657453656C665436
:1008F00065737442697428293A20006973496E74DB
:10090000657272757074456E61626C656428312918
:100910003A2000676574496E746572727570744D23
:10092000617070696E672831293A200067657449E3
:100930006E74657272757074536F75726365283169
:10094000293A2000676574496E7465727275707417
:10095000536F7572636528293A2000676574526188
:10096000746528293A20332E31343135393F0061FE
:100970006363656C2E69734C6F77506F776572286F
:10098000293A2000616363656C2E697341736C655D
:10099000657028293A2000616363656C2E69735481
:1009A0006170536F757263654F6E5A28293A200043
:1009B000616363656C2E6973546170536F75726304
:1009C000654F6E5928293A2000616363656C2E6972
:1009D00073546170536F757263654F6E5828293A6E
:1009E0002000616363656C2E697341637469766985
:1009F0007479536F757263654F6E5A28293A2000D7
:100A0000616363656C2E6973416374697669747997
:100A1000536F757263654F6E5928293A20006973C8
:100A20004163746976697479536F757263654F6E4B
:100A30005828293A200069735461704465746563CD
:100A400074696F6E4F6E5A28293B2066616C73651E
:100A50003F20006973546170446574656374696F05
:100A60006E4F6E5A28293B20747275653F200069CD
:100A700073546170446574656374696F6E4F6E5929
:100A800028293B2066616C73653F200069735461BF
:100A900070446574656374696F6E4F6E5928293BA5
:100AA00020747275653F20006973546170446574E9
:100AB000656374696F6E4F6E5828293B2066616CC0
:100AC00073653F2000697354617044657465637495
:100AD000696F6E4F6E5828293B20747275653F20F0
:100AE000006765745375707072657373426974281A
:100AF000293B2066616C73653F2000676574537500
:100B000070707265737342697428293B2074727522
:100B1000653F200069734163746976697479416344
:100B200028293A20006973496E6163746976697493
:100B3000795A456E61626C656428293A20006973B0
:100B4000496E616374697669747959456E61626C46
:100B5000656428293A20006973496E616374697677
:100B600069747958456E61626C656428293A200081
:100B7000697341637469766974795A456E61626C10
:100B8000656428293A200069734163746976697441
:100B90007959456E61626C656428293A2000697351
:100BA000416374697669747958456E61626C6564F5
:100BB00028293A20006765744672656546616C6C49
:100BC0004475726174696F6E28293A2000676574F4
:100BD0004672656546616C6C5468726573686F6CCB
:100BE0006428293A200067657454696D65496E610F
:100BF0006374697669747928293A200067657449B5
:100C00006E61637469766974795468726573686F2C
:100C10006C6428292000676574416374697669747F
:100C2000795468726573686F6C6428292000676561
:100C300074446F75626C6554617057696E646F7748
:100C400028292000676574446F75626C6554617073
:100C50004C6174656E637928293A20006765745485
:100C600061704475726174696F6E28293A2000675B
:100C70006574417869734F66667365742826782CAD
:100C80002026792C20267A293A2000676574546141
:100C9000705468726573686F6C6428293A20005834
:100CA000595A2047733A200058595A20434F554EFD
:100CB00054533A2000736574206761696E735B5DFD
:100CC0003A006761696E735F6F7269675B5D3A00D6
:100CD000232D2D2D2D2D2D2D2D2D2D2D2D2D2D2D4E
:100CE0002D2D2D2D2D2D2D2D2D2D2D2D2D2D2D2D34
:100CF0002D2D2D2D2D00235265736F6C7574696F2A
:100D00006E3A20202000234D696E2056616C756577
:100D10003A2020202000234D61782056616C7565B3
:100D20003A202020200023556E69717565204944C2
:100D30003A2020202000234472697665722056658F
:100D4000723A202020002353656E736F723A202080
:100D5000202020202000232D2D2D2D204D61676E79
:100D6000657469632053656E736F72202D2D2D2D70
:100D70002D2D2D2D2D2D2D2D2D2D2D2D2D2D2D2DA3
:100D800000482D6669656C643A20280020202020E8
:100D90002020202020202020202020002020202073
:100DA000202020202020202020202000233A5368CB
:100DB0006F772F48696465204C4344002A3A546891
:100DC00069732048656C700044233A43616C696222
:100DD000726174696F6E00442A3A53657474696E67
:100DE00067730044423A5265736574204C6F6767BD
:100DF00065720044433A436C656172204C43440081
:100E000044443A4D756C746953656E736F72730028
:100E100044393A43757272656E7400566F6C746132
:100E200067652B43757272656E740044383A456C81
:100E30006563747269630044373A4D6F74696F6E0D
:100E40000044363A44532054656D700044353A5599
:100E50005620496E74656E736974790044343A4F54
:100E60003220636F6E632E0044333A434F32206367
:100E70006F6E632E0044323A504D28313A322E358F
:100E80003A3130290044323A504D28313A322E3529
:100E90003A3130292A0044313A54757262696469E2
:100EA00074790044303A566F6C7461676500393A62
:100EB0006F7220334420616363656C2E00393A49B8
:100EC0006E636C2E20616E672E00383A7048207673
:100ED000616C756500373A49522054656D70003772
:100EE0003A49522054656D702A00363A4D61676E5A
:100EF00065746963206669656C6400353A4761739F
:100F0000204C6576656C00343A495220466C616D20
:100F10006500333A4C6967687420496E742E00325C
:100F20003A616E642048656967687400323A5465B6
:100F30006D7020507265737375726500313A546537
:100F40006D702048756D696469747900303A536F2B
:100F5000756E64204C6576656C00303A536F756E23
:100F600064204C6576656C2A0054696D65206C615F
:100F70007073653A00576946692049503A004669DE
:100F80006E64696E6720576946692049500069742C
:100F900065726174696F6E3D0073656E736F722365
:100FA0003D0043757272656E74207374617475735D
:100FB0003A206379636C653D006E6379636C653DCF
:100FC000006E73656E736F72733D006D61786E7342
:100FD000656E736F72733D00656E61626C65643D32
:100FE00000234D756C746973656E736F7273206D39
:100FF0006561737572656D656E742073657474696F
:101000006E67733A007365703D006976616C3D00F0
:101010006E697465723D00230043616C2E20466149
:10102000696C65640043616C2E20446F6E65004EF0
:101030006F206E6565642100496E76616C6964207D
:101040005028506129005365614C6576656C2050CD
:10105000285061293A0043616C69627261746520AD
:1010600050004453542054656D702073656E736F47
:10107000720043757272656E742073656E736F7261
:10108000004F322073656E736F7200555620736582
:101090006E736F720043616C6962726174650046C1
:1010A00061696C65640054422063616C2E20646F3A
:1010B0006E65005570706572204C696D69743A3EBA
:1010C000004C6F776572204C696D69743A3E00542C
:1010D0007572626964697479004661696C6564005F
:1010E00070482063616C2E20646F6E65007048311B
:1010F0003020507265737320420070483420507263
:1011000065737320410043616C69627261746500AC
:10111000005EBCE2613FDD83C29C7E20A3FD1F41D7
:10112000009D23BE46DB65F88C11AF32CA57E974C7
:10113000416E676C65732F003E6128782C792C7A9C
:10114000292F673A004E6F2073656E736F7221000E
:1011500049522054656D7065726174757265004DF9
:101160006561737572696E672E2E004E6F20736510
:101170006E736F723F0049522054656D70657261E5
:1011800074757265004D6561737572696E672E2E98
:10119000004F6666206169722D636F6E642100499D
:1011A00074277320746F6F20636F6F6C2100546518
:1011B0006D702069732066696E6521004973206136
:1011C00069722D636F6E64206F6E3F0049742773E0
:1011D00020717569746520686F74210049742773E4
:1011E000207665727920686F742120004F66662032
:1011F0006169722D636F6E642100497427732074D6
:101200006F6F20636F6F6C210054656D7020697380
:101210002066696E6521004973206169722D636FD4
:101220006E64206F6E3F0049742773207175697476
:101230006520686F74210049742773207665727980
:1012400020686F74210054656D702048756D696465
:10125000697479004E6F2053656E736F7221004E72
:101260006F20445320546865726D6F6D65746572AC
:101270002100445320546865726D2E004D6F7469CF
:101280006F6E00556E6B6E6F776E00496E6475738E
:10129000747269616C20342D32306D4100414353CA
:1012A000373132204D61783D3541002343757272EC
:1012B000656E742073656E736F723A0000002100D2
:1012C000240027002A002D00300033000101000017
:1012D000040107010A0100002200250028002B005C
:1012E0002E003100340002010000050108010B014D
:1012F000000020002300260029002C002F003200CF
:1013000000010000030106010901050505050705A7
:1013100008080808020202020A0A08080404040471
:10132000010101010101010103030303030303039D
:10133000040707070C0C0C0C0C0C0C0C020202022C
:1013400006060606060606060B0B0B0B0B0B0B0B15
:1013500001021020200808102040102040800201C7
:1013600002010804020101020408102040808040AC
:1013700020100804020180040201804020100804AB
:101380000201080402010102040810204080010249
:1013900004081020408000000A0B02090C0D0E0802
:1013A000070304010000000000000000000000002E
:1013B000000000000000000000000000000000002D
:1013C00000001211100000000000000000000000EA
:1013D000000000000000000000000000496E76617F
:1013E0006C6964206B65792100202020202020205A
:1013F000202020202020202020002020202020200D
:1014000020202020202020202020002020202020FC
:1014100020202020202020202020200020202020EC
:10142000202020202020202020202020004E455455
:101430003D426C7565746F6F7468204C45004E4575
:10144000543D426C7565746F6F7468004E45543D31
:10145000576946690053657474696E67204661690F
:101460006C65640053657474696E6720446F6E65C3
:10147000004368616E6765204E6574776F726B3EDE
:1014800000547970653A0042542F57694669204EDE
:101490006574776F726B004368616E676520536592
:1014A0006E736F723E0043757272656E7420536581
:1014B0006E736F72004F7468657200496E642E20FF
:1014C000342D32306D4100414353373132203C33AB
:1014D000304100414353373132203C3230410041EA
:1014E0004353373132203C3541003E4D6178205620
:1014F0006F6C743A3E004368616E676520766F6C6E
:10150000746167653E00547970652000566F6C7495
:101510006167652053656E736F72004368616E6723
:1015200065207479706520746F0053656E736F72F7
:101530003D4448540054656D702048756D69646978
:1015400074790000C7A927AC11241FBECFEFD1E2E8
:10155000DEBFCDBF00E00CBF1CE0A0E0B2E0E8E8D9
:10156000F1E701E00BBF02C007900D92A837B10769
:10157000D9F724E1A8E7BCE001C01D92A732B20769
:10158000E1F71AE0C3EADAE000E006C021970109BA
:10159000802FFE010E9406B6C23AD10780E00807FC
:1015A000A9F70E94229D0C94B3B80C9400002F92CE
:1015B0003F924F925F926F927F928F929F92AF92E3
:1015C000BF92CF92DF92EF92FF920F931F93CF9330
:1015D000DF93CDB7DEB7C554D1090FB6F894DEBF9F
:1015E0000FBECDBF8C01E090970CF090980C8091CD
:1015F0001F14882349F06DE675E081E79FE00E94A3
:101600009557C8010E94595C680125E0C20ED11CA3
:1016100035E0C316D10420F18091970C9091980C7D
:101620000817190729F10E94A1410E94BE740C3EBF
:101630004FEF140724F01093980C0093970CB80107
:10164000CE0101960E945A5BBE016F5F7F4F8DE80D
:1016500092E10E94E255CE0101960E94C55608C053
:101660000E3F5FEF150721F40E94CE740C94DD1D30
:1016700064E67AE081E892E10E949B56F5E0CF169D
:10168000D10490F066E67CE0CE0101960E942957D5
:101690004AE050E06FEF7FEFCE0101960E94369353
:1016A000CE0101960E94C556F8017C96E632F105FE
:1016B00010F00C94E91C8827EE58FF4F8F4F0C94C4
:1016C00006B60E94A14189E390E00E94736A20E07F
:1016D00030E04AE754E40E948DB1AB01BC0121E047
:1016E000CE0101960E94CA5661EC75E0CE0180964B
:1016F0000E942957BE016F5F7F4FCE0180960E94E6
:10170000455664EC75E00E942E56BC0181E892E1DA
:101710000E94B056CE0180960E94C556CE01019619
:101720000E94C55668EC75E08BE792E10E949B56DB
:101730006BE772E1CE0101960E9421574AE050E02A
:1017400068E070E0CE0101960E949192CE01019670
:101750000E94C55661E872E1CE0101960E942157B0
:101760004AE050E06FEF7FEFCE0101960E94499072
:10177000CE0101960E94C5566BE772E181E892E1C5
:101780000E94DC558091D30C882311F40C941B1D0E
:101790000C946917E090B902F090BA020E94A1413E
:1017A00089E390E00E94736A20E030E04AE754E465
:1017B0000E948DB10E9417B4CE0101960E945A5B1F
:1017C00061EC75E0CE0180960E942957BE016F5FE3
:1017D0007F4FCE0180960E94455664EC75E00E94D2
:1017E0002E56BC0181E892E10E94B056CE0180964F
:1017F0000E94C556CE0101960E94C5568091851261
:1018000090918612099718F423E0D22E02C092E03C
:10181000D92E8091181183302CF5C7010E942477AE
:101820007C016091191170911A11072E000C880B20
:10183000990B0E942EB14B015C01B701FF0C880B84
:10184000990B0E942EB19B01AC01C501B4010E940D
:101850008DB120E030EC4FE754E40E947EB3AB0141
:10186000BC0103C040E050E0BA012D2DCE0101962D
:101870000E94CA566DEF75E0CE0180960E942957EE
:10188000BE016F5F7F4FCE0180960E94455660ED8E
:1018900075E00E942E56BC0181E892E10E94DC5561
:1018A000CE0180960E94C556CE0101960E94C55673
:1018B00063ED75E039CF8091D30C882309F42CC1F6
:1018C00087E39EE00E94E39061E0809102020E9423
:1018D0007B8860E0809100020E947B880E94709A61
:1018E0000E94D04A0E94ED4AAB01BC0123E0CE0128
:1018F00080960E94CA56BE01605E7F4FCE0101965F
:101900000E9421576AEF75E0CE0101960E942E5683
:10191000BC018BE792E10E94B056CE0101960E9475
:10192000C556CE0180960E94C55660E97AE0CE0188
:1019300001960E9429576BE772E1CE0101960E9441
:101940004556BC0181E892E10E94B056CE01019655
:101950000E94C5560E94ED4A6B017C010E94DC8802
:101960004B015C016EE170E080E090E00E94018933
:101970000E94ED4A2B013C010E94DC889B01AC01D6
:10198000281939094A095B0949015A0131ED8316C1
:1019900037E09306A104B1040CF441C0A7019601FD
:1019A000C301B2010E94B7B26B017C0120E030E0BC
:1019B000A9010E946DB418165CF426EA3BE944ECD8
:1019C0005BE3C701B6010E9428B187FF0BC027C0A7
:1019D00026EA3BE944EC5BEBC701B6010E946DB41B
:1019E0001816ECF0C501B40128EE33E040E050E0F9
:1019F0000E945AB2CA01B9010E942EB14B015C018A
:101A000020E030E04AE754E4C701B6010E948DB1FE
:101A1000A50194010E947EB3AB01BC0103C040E06C
:101A200050E0BA0122E0CE0180960E94CA56BE0163
:101A3000605E7F4FCE0101960E9421576CED75E0EC
:101A4000CE0101960E942E56BC0185E792E10E94CC
:101A5000B056CE0101960E94C556CE0180960E94D6
:101A6000C55660EE75E0CE0101960E94295765E7E4
:101A700072E1CE0101960E944556BC0181E892E1D7
:101A80000E94DC55CE0101960E94C55666E67CE0B8
:101A9000CE0101960E94295765E772E1CE010196B9
:101AA0000E944556BC018BE792E10E94DC55CE01B5
:101AB00001960E94C55669E573E0CE0101960E9429
:101AC00019574AE050E060E070E0CE0101960E94B4
:101AD0009192CE0101960E94C5566BE772E1CE014C
:101AE00001960E94215745E050E06FEF7FEFCE0155
:101AF00001960E944990CE0101960E94C55664EE5F
:101B000075E081E892E10E94CE5560E0809102028A
:101B10000E947B880C941B1D6091550270915602A7
:101B200080915702909158020E9442780C941B1D9C
:101B300080915B0290915C020E94457A0C941B1D7F
:101B400040915D0226964FAF269760E0842F0E9459
:101B50007B888091D30C811109C08091761181110D
:101B60000EC08FE090E0A0E0B0E00DC023E030E0D8
:101B700040E050E02CAF3DAF4EAF5FAF08C083E018
:101B800090E0A0E0B0E08CAF9DAFAEAFBFAF68E635
:101B900073E081E892E10E94565661E872E1CE015D
:101BA00001960E9421574AE050E06FEF7FEFCE018F
:101BB00001960E949192CE0101960E94C5562196EF
:101BC0001FAE219725961FAE2597212C312CC12CB5
:101BD000D12C760182E3682E712C812C912C54013A
:101BE00026968FAD26970E94B788092E000CAA0B67
:101BF000BB0B880E991EAA1EBB1E65E070E080E03C
:101C000090E00E94018991E0691A710849F74090BB
:101C10002102509022026090230270902402C5019C
:101C2000B4010E942EB120E030E040EA50E40E946E
:101C30008DB120E030E040E85AE30E948DB120E011
:101C400030E048E452E40E947EB3A30192010E9476
:101C5000B7B220E030E040E751E40E948DB14B0183
:101C60005C01A30192016AE979E989E390E40E94A9
:101C7000B7B29B01AC01C501B4010E947EB320E064
:101C800030E0A9010E94B8B220E030E040E251E427
:101C90000E948DB14B015C0121962FAD21972596B5
:101CA0003FAD2597A1010E946DB418163CF4219612
:101CB0008FAE219725969FAE2597150120E030E045
:101CC000A901B401C5010E9428B187FF04C0812C7D
:101CD000912CA12CB12C22E0A401B501CE0180965B
:101CE0000E94CA56BE01605E7F4FCE0101960E94DF
:101CF000215767EF75E0CE0101960E942E56BC0178
:101D00008BE792E10E94B056CE0101960E94C55623
:101D1000CE0180960E94C5566BE772E1CE01019616
:101D20000E9421574AE050E060E070E0CE01019649
:101D30000E944990CE0101960E94C5560E945D8A7C
:101D40008090171490901814A0901914B0901A1441
:101D5000A4E68A0E911CA11CB11C86169706A80643
:101D6000B90610F40C943C1D0E945D8A0E942CB1AF
:101D70004B015C0160911714709118148091191433
:101D800090911A140E942EB120E030E048EC51E40A
:101D90000E94B8B29B01AC01C501B4010E9428B1F8
:101DA00087FF02C00C943C1D6CE370E080E090E083
:101DB0000E940189BFEFCB1ADB0AEB0AFB0A2CADAC
:101DC0003DAD4EAD5FAD2C153D054E055F050CF0EC
:101DD00001CF64E670E080E090E00E9401890E94FB
:101DE000A14164E670E080E090E00E94018960E635
:101DF00073E08BE792E10E9456566BE772E1CE01E9
:101E000001960E94215744E150E060E070E0CE016D
:101E100001960E949192CE0101960E94C55622E041
:101E200021964FAD219725965FAD2597B101CE0143
:101E300080960E94CA56BE01605E7F4FCE01019619
:101E40000E94215767EF75E0CE0101960E942E5641
:101E5000BC018BE792E10E94B056CE0101960E9430
:101E6000C556CE0180960E94C5566BE772E1CE0141
:101E700001960E94215742E350E06FEF7FEFCE01C1
:101E800001960E944990CE0101960E94C55664E1D8
:101E900070E080E090E00E9401890E94C5416EE1FF
:101EA00070E080E090E00E9401896EE170E080E0E7
:101EB00090E00E9401896CEF75E0CE0101960E94CE
:101EC00029576BE772E1CE0101960E94455660E00A
:101ED00076E00E942E5661E872E10E944556BC01F0
:101EE00081E892E10E94B056CE0101960E94C5564B
:101EF0000C941B1D80915F029091600299270E94B3
:101F00002477BC01990F880B990B0E942EB12DE00C
:101F100038E643E55BE30E948DB16B017C012091C3
:101F200083023091840240918502509186020E9482
:101F300028B118164CF060916B0270916C02809180
:101F40006D0290916E021BC0209197023091980211
:101F50004091990250919A02C701B6010E946DB456
:101F600087FF05C0C701B6010E94D87208C0609102
:101F70007F0270918002809181029091820220E024
:101F800030E048EC52E40E948DB120E030E048EAB5
:101F900051E40E948DB1209125023091260240919A
:101FA0002702509128020E947EB36B017C0165E7F5
:101FB00073E08BE792E10E9456566BE772E1CE0127
:101FC00001960E94215742E350E060E070E0CE01AC
:101FD00001960E949192CE0101960E94C55622E080
:101FE000B701A601CE0101960E94CA566AE076E0CA
:101FF000CE0180960E942957BE016F5F7F4FCE01B0
:1020000080960E94455664E076E00E942E56BC0100
:1020100081E892E10E94B056CE0180960E94C5569A
:10202000CE0101960E94C55661E872E1CE0101968B
:102030000E94215742E350E06FEF7FEFCE010196FF
:102040000E944990CE0101960E94C5568091D30C02
:10205000882311F40C941B1D60E273E080E090E093
:102060000E9401890C941B1D0E94A14169EA73E042
:1020700081E892E10E94565661E872E1CE01019634
:102080000E9421574AE050E060E070E0CE010196E6
:102090000E949192CE0101960E94C55660EA73E0BB
:1020A0008BE792E10E9456566BE772E1CE010196F2
:1020B0000E94215744E150E06FEF7FEFCE0101967F
:1020C0000E944990CE0101960E94C55680917C0CD9
:1020D00090917D0C8230910549F40E9439898111DB
:1020E0001AC010927D0C10927C0C15C0892BC9F47B
:1020F0000E943989882339F082E090E090937D0C2A
:1021000080937C0C08C00E9439898111F5CF0E9410
:1021100039898111F1CF80917C0C90917D0C0297CF
:1021200041F164E973E081E892E10E94565661E86A
:1021300072E1CE0101960E9421574AE050E060E032
:1021400070E0CE0101960E949192CE0101960E940C
:10215000C55661E872E1CE0101960E94215766E6FC
:102160007CE0CE0101960E942E566BE772E10C9442
:10217000431A8AE090E00E94F8746B017C0120E031
:1021800030E0A9010E9428B1181634F08AE090E0EE
:102190000E94F8746B017C01BBE0AB2EB12C20E0F7
:1021A00030E042ED53E4C701B6010E9428B1181691
:1021B0008CF031E0A31AB10869F068EC70E080E0BF
:1021C00090E00E94018983E090E00E94F8746B0126
:1021D0007C01E5CF20E030E0A901C701B6010E94F3
:1021E00028B118163CF066E873E081E892E10E949D
:1021F000565631C020E030E048EC52E4C701B60149
:102200000E9428B187FF02C021E001C020E0B70191
:10221000A601CE0101960E94CA5669E076E0CE0181
:1022200080960E942957BE016F5F7F4FCE01809636
:102230000E9445566EE076E00E942E56BC0181E871
:1022400092E10E94B056CE0180960E94C556CE0102
:1022500001960E94C55661E872E1CE0101960E9486
:10226000215742E350E06FEF7FEFCE0101960E94CD
:102270004990CE0101960E94C5566DE773E08BE749
:1022800092E10E9456566BE772E1CE0101960E94E0
:10229000215742E350E060E070E0CE0101960E94D9
:1022A0009192D0CE0E945D8A2B013C0187E39EE093
:1022B0000E94E39064E670E080E090E00E94018973
:1022C00040E855E260E070E087E39EE00E94B7736B
:1022D00064E670E080E090E00E94018962EE73E0C5
:1022E0008BE792E10E9456566BE772E1CE010196B0
:1022F0000E94215742E350E06FEF7FEFCE0101963D
:102300000E949192CE0101960E94C55667ED73E03E
:102310008BE792E10E9456566BE772E1CE0101967F
:102320000E94215742E350E06FEF7FEFCE0101960C
:102330000E944990CE0101960E94C55680919D0C45
:1023400090919E0C8D7F1CAEA12CB12CC12CD12C58
:10235000E12CF12C019709F46FC0AE01405E5F4F94
:1023600059AF48AFCE014E969BAF8AAF0E945D8AAF
:10237000DC01CB0184199509A609B709883B9B406C
:10238000A105B10508F058C087E39EE00E947F5286
:10239000892B09F44AC02CED35E040E050E0209351
:1023A0003B0E30933C0E40933D0E50933E0E0E94E8
:1023B000837397FD06C082349105C9F780E090E0F1
:1023C00002C08FEF9FEF892B81F5AE014F5F5F4F0A
:1023D0001A014A010E94837397FF06C089818D34D8
:1023E00021F520E030E009C0D4018D934D01E8AD26
:1023F000F9ADEA17FB0771F7F1CFD1018D911D01FE
:10240000280F311DEAADFBADAE17BF07B1F72E5B4C
:102410003F4F8E8D90E0982F88274F8D840F911D10
:102420002817390711F40C94401D62E370E080E036
:1024300090E00E9401899ACF0E945D8ADC01CB0165
:1024400084199509A609B709883B9B40A105B105E8
:1024500018F42CAD2111BDC00E94A1416BE772E1BF
:10246000CE0180960E94215742E350E066E070E082
:10247000CE0180960E949192CE0180960E94C55610
:102480003CAD332311F40C94591D82E090E09093FD
:102490009E0C80939D0CB501CE0180960E945A5BE4
:1024A000B601CE0186960E945A5BB701CE01C29654
:1024B0000E945A5BBE016E5C7F4FCE018C960E94DB
:1024C000215769E177E0CE018C960E942E56BE011D
:1024D0006A5D7F4F0E94455669E177E00E942E5663
:1024E000BE01605E7F4F0E944556BC0181E892E1CB
:1024F0000E94B056CE018C960E94C556CE01C2965F
:102500000E94C556CE0186960E94C556CE01809681
:102510000E94C55661E872E1CE0180960E94215763
:102520004AE050E06FEF7FEFCE0180960E94499025
:10253000CE0180960E94C55661ED73E08CE793E171
:102540000E949557B501CE0180960E945A5BB60154
:10255000CE0186960E945A5BB701CE018C960E94EE
:102560005A5B62E176E0CE01C2960E942957BE0115
:10257000645D7F4FCE01C2960E94455666E67CE0C0
:102580000E942E56BE016A5D7F4F0E94455666E648
:102590007CE00E942E56BE01605E7F4F0E94455631
:1025A00062E276E00E942E56BC0181E892E10E9430
:1025B000B056CE01C2960E94C556CE018C960E949E
:1025C000C556CE0186960E94C556CE0180960E94C1
:1025D000C55662E370E080E090E00E94018987E3E5
:1025E0009EE00E94E3901BC6E0905902F0905A02D0
:1025F00068E276E08BE792E10E949B560E94A1413F
:102600006BE772E1CE0101960E9421574AE050E04B
:102610006FEF7FEFCE0101960E949192CE0101965D
:102620000E94C556C7010E941C7824966CAF7DAFEE
:102630008EAF9FAF249780902F0290903002A09091
:102640003102B0903202A501940160912B02709189
:102650002C0280912D0290912E020E94B7B22B0184
:102660003C0120E030E0A9010E9428B1882309F450
:1026700053C0C0903702D0903802E0903902F090F9
:102680003A0220E030E0A901C701B6010E9428B15A
:1026900018160CF041C08091330290913402A09141
:1026A0003502B09136028CAF9DAFAEAFBFAF9C018B
:1026B000AD01C701B6010E9428B1882369F1A701C5
:1026C00096016CAD7DAD8EAD9FAD0E947EB30E9434
:1026D000B3B46CAF7DAF8EAF9FAFA50194012496CC
:1026E0006CAD7DAD8EAD9FAD24970E94B7B2A301B6
:1026F00092010E947EB32CAD3DAD4EAD5FAD0E9408
:102700008DB10E94EBB39B01AC01C701B6010E94E1
:102710008DB16B017C0103C0C12CD12C76016BE71C
:1027200072E1CE0101960E9421574AE050E060E03C
:1027300070E0CE0101960E949192CE0101960E9416
:10274000C55620E030E64AEE56E4C701B6010E94C5
:102750006DB418163CF46EEE73E081E892E10E94CD
:10276000565625C021E0B701A601CE0180960E94F1
:10277000CA5662E376E0CE0101960E942957BE0157
:10278000605E7F4FCE0101960E94455666E376E07B
:102790000E942E56BC0181E892E10E94B056CE0103
:1027A00001960E94C556CE0180960E94C55661E8EA
:1027B00072E1CE0101960E9421574AE050E06FEF8E
:1027C0007FEFCE0101960E944990CE0101960E94B2
:1027D000C55664E670E080E090E00E94018936CC46
:1027E000E090B902F090BA020E94A14165E070E069
:1027F00080E090E00E9401898091181183302CF5CF
:10280000C7010E9424777C016091191170911A11FF
:10281000072E000C880B990B0E942EB14B015C0116
:10282000B701FF0C880B990B0E942EB19B01AC01E4
:10283000C501B4010E948DB120E030EC4FE754E4B3
:102840000E947EB3AB01BC0103C040E050E0BA017E
:1028500023E0CE0101960E94CA566DEF75E0CE01CD
:1028600080960E942957BE016F5F7F4FCE018096F0
:102870000E94455660ED75E00E942E56BC0181E82D
:1028800092E10E94B056CE0180960E94C556CE01BC
:1028900001960E94C5566AE376E00C94940B9091E1
:1028A000960C81E089278093960C8091D30C882325
:1028B00031F061E872E18AE99DE00E94AE6F68EC58
:1028C00070E080E090E0CCCB1092D30C0C941B1DF8
:1028D00081E08093D30C8093841180917B118823B5
:1028E00049F166E278E08DE892E10E949B5686EE1F
:1028F0009FEF9093980C8093970C20917E113091CC
:102900007F1180918011909181118217930724F09B
:102910001092811110928011109272111092731105
:1029200010927411109275116CE271E080E090E0E9
:102930000E9401896DE872E183E992E10E94B0563C
:102940008091970C9091980C9093CE0C8093CD0C25
:102950000C941B1D0E94F8410C941B1D84ED9EE0FD
:102960000E94E39040E052EC61E070E084ED9EE074
:102970000E94B7738CED95E0A0E0B0E08093D80E94
:102980009093D90EA093DA0EB093DB0E64E670E05C
:1029900080E090E00E94018980917C0C90917D0CF8
:1029A000019759F483E090E00E948077811140C044
:1029B00010927D0C10927C0C1AC081E090E00E9475
:1029C0008077882339F081E090E090937D0C8093AC
:1029D0007C0C0DC083E090E00E9480778111F3CFE2
:1029E00083E090E00E9480778111EDCF06C0809156
:1029F0007C0C90917D0C0197D9F06DE274E08BE72F
:102A000092E10E9456566BE772E1CE0101960E9458
:102A1000215744E150E06FEF7FEFCE0101960E9415
:102A20004990CE0101960E94C55661E274E0CDC086
:102A300065E174E081E892E10E94565661E872E136
:102A4000CE0101960E942157CE0101960E94659207
:102A5000CE0101960E94C55662E370E080E090E0EE
:102A60000E94018961E872E1CE0101960E9421571E
:102A700042E350E06FEF7FEFCE0101960E9491920A
:102A8000CE0101960E94C55669E074E08BE792E1A1
:102A90000E9456566BE772E1CE0101960E942157C3
:102AA00044E150E06FEF7FEFCE0101960E94499024
:102AB000CE0101960E94C5568BEB88A38AEA89A3B2
:102AC00081E08AA3C12CD12C412C512C3201212C24
:102AD000312CC6016AE070E00E94F3B5892B49F4FD
:102AE00043E050E0BE01605E7F4F84ED9EE00E94B7
:102AF000245265E070E080E090E00E940189BFEF21
:102B0000CB1ADB0AE12CF12C812C912C540184EDA1
:102B10009EE00E947F52892B81F4E4E08E1691049E
:102B2000A104B10454F094E02916310464F4A0E93E
:102B3000CA16A1E0DA0669F606C0F6E0EF16F1045F
:102B40000CF4E3C7F0CFC301B2010E942EB120E024
:102B500030E040E251E40E947EB320E030E040E803
:102B60005EE30E948DB16B017C0120E030E040EA21
:102B700051E40E946DB4181634F521E0B701A601A6
:102B8000CE0101960E94CA566FE877E0CE0180968A
:102B90000E942957BE016F5F7F4FCE0180960E9431
:102BA000455662E476E00E942E56BC0181E892E12F
:102BB0000E94B056CE0180960E94C556CE01019665
:102BC0000E94C55606C06DEF73E081E892E10E9455
:102BD000565661E872E1CE0101960E9421574AE003
:102BE00050E060E070E0CE0101960E949192CE012B
:102BF00001960E94C55661E872E1CE0101960E94DD
:102C0000215766E67CE0CE0101960E942E566BE7C6
:102C100072E10E944556BC0181E892E10E94B056E3
:102C2000CE0101960E94C55684ED9EE00E94E3907D
:102C30000DCA68EC74E0CE0101960E9419574AE073
:102C400050E06FEF7FEFCE0101960E944990CE01D8
:102C500001960E94C5566091B7027091B8028091AA
:102C6000290290912A020E942568E4E18E2E912C7F
:102C7000A12CB12CC12CD12CAFEFCA1ADA0AC50194
:102C8000B4010E9401896091B7027091B8028091ED
:102C9000290290912A020E9425687C01B3E0CB169C
:102CA000D10434F08EE1C816D10444F4EF2851F079
:102CB00094E1890E911CA11CB11CDECFE114F1043A
:102CC00009F00CC18091290290912A028B30910564
:102CD000C9F48091D9129091DA12A091DB12B091CF
:102CE000DC128093F90C9093FA0CA093FB0CB09338
:102CF000FC0C8091D5129091D612A091D712B09170
:102D0000D8121DC08631910521F30C9701F58091F1
:102D1000EC0C9091ED0CA091EE0CB091EF0C809327
:102D2000F90C9093FA0CA093FB0CB093FC0C8091DF
:102D3000E80C9091E90CA091EA0CB091EB0C809317
:102D4000F50C9093F60CA093F70CB093F80C40910F
:102D5000F90C5091FA0C6091FB0C7091FC0C21E085
:102D6000CE0101960E94CA5662EA7AE0CE018096B0
:102D70000E942957BE016F5F7F4FCE0180960E944F
:102D80004556BC0181E892E10E94B056CE01809682
:102D90000E94C556CE0101960E94C5564091F50C81
:102DA0005091F60C6091F70C7091F80C21E0CE0177
:102DB00001960E94CA5665E476E0CE0180960E9494
:102DC0002957BE016F5F7F4FCE0180960E94455606
:102DD000BC0181E892E10E94DC55CE0180960E9400
:102DE000C556CE0101960E94C55667E076E081E89F
:102DF00092E10E94CE5564E67AE0CE0101960E94EF
:102E0000295744E150E060E070E0CE0101960E9455
:102E10009192CE0101960E94C556C090F90CD090B7
:102E2000FA0CE090FB0CF090FC0C20E030E0A901E3
:102E3000C701B6010E946DB420E030E040E05FE3DE
:102E400087FD05C0C701B6010E94B8B204C0C70122
:102E5000B6010E94B7B20E9417B4AB01BC01CE010B
:102E600001960E946870BE016F5F7F4F8BE792E111
:102E70000E94E255CE0101960E94C55660E087E0AF
:102E80000E943D706BE772E18CE793E10E948757E7
:102E90006FED8CE793E10E9480576BE476E08CE75E
:102EA00093E10E9460586091F50C7091F60C80914E
:102EB000F70C9091F80C0E9417B44AE050E08CE7B0
:102EC00093E10E94165867E076E08CE793E10E9458
:102ED000605864E670E080E090E0C2C8EFEFEE1664
:102EE000FE06ACF06AEB74E0CE0101960E94195721
:102EF0004AE050E060E070E0CE0101960E949192BD
:102F0000CE0101960E94C55667E974E048C0FEEF05
:102F1000EF16FFEFFF0679F169E874E0CE01019644
:102F20000E9419574AE050E060E070E0CE0101963F
:102F30000E949192CE0101960E94C5566AE774E004
:102F400081E892E10E945656B701CE0101960E9497
:102F50005A5BBE016F5F7F4F81E892E10E94DC55B2
:102F6000CE0101960E94C55664E674E081E892E1C4
:102F70000E948C5560C569E574E0CE0101960E94FF
:102F800019574AE050E060E070E0CE0101960E94DF
:102F90009192CE0101960E94C55669E374E081E8E2
:102FA00092E10E94565647C580910402882309F495
:102FB00042C564E67AE0CE0101960E9429574AE0B4
:102FC00050E061E070E0CE0101960E949192CE0146
:102FD00001960E94C5560E94CF8E2DC58091D30CBC
:102FE00081110AC080917611811106C07EE1472EC1
:102FF000512C612C712C05C063E0462E512C612CA4
:10300000712C66ED74E081E892E10E94565661E809
:1030100072E1CE0101960E9421574AE050E06FEF25
:103020007FEFCE0101960E944990CE0101960E9449
:10303000C556812C912C54011CAE1DAE1EAE1FAE88
:1030400083E20E94227087E090E00E941D700E943F
:103050001B7066E970E080E090E00E94018983E2E5
:103060000E94227080E290E00E941D700E941B70FE
:1030700066E970E080E090E00E94018962E070E023
:1030800083E290E00E94FF91C12CD12C76018091C7
:10309000F51390E02091F613821B9109181619067A
:1030A0006CF48EE090E10E941D7DFE2CED2CDC2C5A
:1030B000CC24C80ED11CE11CF11CE9CFC701B6011C
:1030C0000E942EB12AE939E949E95FE30E947EB303
:1030D0000E9417B4AB01BC0184169506A606B7067C
:1030E00014F44A015B01CE0180960E946870BE0113
:1030F000605E7F4FCE0101960E9421576EE476E01C
:10310000CE0101960E942E56BC018BE792E10E94EF
:10311000B056CE0101960E94C556CE0180960E94FF
:10312000C5566BE772E1CE0101960E9421574EE130
:1031300050E060E070E0CE0101960E943693CE012F
:1031400001960E94C5562CAD3DAD4EAD5FAD2F5FD3
:103150003F4F4F4F5F4F2CAF3DAF4EAF5FAF42166B
:103160005306640675060CF06BCFB501A401CE01C1
:1031700080960E946870BE01605E7F4FCE0101960E
:103180000E9421576EE476E0CE0101960E942E56F1
:10319000BC018BE792E10E94B056CE0101960E94DD
:1031A000C556CE0180960E94C5566BE772E1CE01EE
:1031B00001960E9421574AE050E060E070E0CE01A5
:1031C00001960E949192CE0101960E94C556B501CA
:1031D000A401CE0101960E94687061EB79E0CE01F6
:1031E00080960E942957BE016F5F7F4FCE01809667
:1031F0000E94455662E576E00E942E5661E872E133
:103200000E944556BC0181E892E10E94B056CE0171
:1032100080960E94C556CE0101960E94C55662E373
:1032200070E080E090E00C943010E090B502F090F7
:10323000B60281E080932C0564E670E080E090E0C7
:103240000E9401890E94A141C7010E94247760E089
:1032500074E0681B790BCE0101960E945A5B67E50A
:1032600076E0CE0180960E942957BE016F5F7F4FA6
:10327000CE0180960E944556BC0181E892E10E94F1
:10328000B056CE0180960E94C556CE0101960E948E
:10329000C55660E087E00E943D7066EE74E0CE01A6
:1032A00001960E94195742E350E068E070E0CE01B9
:1032B00001960E949192CE0101960E94C55661E846
:1032C00072E1CE0101960E94215742E350E06FEF78
:1032D0007FEFCE0101960E944990CE0101960E9497
:1032E000C5566EE576E0C7C08091B3029091B402F6
:1032F0000E9424777C0190937F0C80937E0C62E384
:1033000070E080E090E00E940189B701CE01019653
:103310000E945A5BBE016F5F7F4F81E892E10E947D
:10332000E255CE0101960E94C5568091D31290912C
:10333000D412892B09F45EC06FEC72E1CE01809645
:103340000E942157BE01605E7F4FCE0101960E9410
:10335000215744E150E060E070E0CE0101960E9408
:103360009192CE0101960E94C55668E676E0CE01A4
:1033700001960E94295761E872E1CE0101960E94F0
:103380004556BC018BE792E10E94B056CE010196F2
:103390000E94C5566BE772E1CE0101960E9421574B
:1033A00044E150E06FEF7FEFCE0101960E9449901B
:1033B000CE0101960E94C556BE01605E7F4FCE01D0
:1033C00001960E94215766E67CE0CE0101960E949C
:1033D0002E566BE772E10E944556BC0181E892E1EE
:1033E0000E94B056CE0101960E94C556CE0180962D
:1033F0000C94241063E776E08BE792E10E949B56E1
:103400006BE772E1CE0101960E94215744E150E042
:1034100060E070E0CE0101960E949192CE0101968B
:103420000E94C55667E576E0CE0101960E942957B5
:1034300061E872E1CE0101960E944556BC018BE71E
:1034400092E10E94B056CE0101960E94C5566BE7EC
:1034500072E1CE0101960E94215744E150E06FEFE6
:103460007FEFCE0101960E944990CE0101960E9405
:10347000C55668E676E0CE0101960E94295761E8BC
:1034800072E1CE0101960E944556BC0181E892E1AD
:103490000E94B056CE0101960E94C5560C9426108B
:1034A00080910402882309F4C6C28091D30C811153
:1034B00004C080917611882329F082E090E00E9478
:1034C0007C45B9C2C0905502D0905602E090570298
:1034D000F090580220E030E040E450E4C701B6012B
:1034E0000E946DB418166CF420E030E04AEF54E40A
:1034F000C701B6010E948DB10E9417B46B017C0117
:1035000006C040E3C42E45E7D42EE12CF12C0E94E6
:10351000A14160E080E00E943D7067EF74E08CE7BD
:1035200093E10E94955761E080E00E943D706FEE4C
:1035300074E08CE793E10E94955764E670E080E0C8
:1035400090E00E9401890E945D8A6093780C7093DC
:10355000790C80937A0C90937B0C0E945D8A80900A
:10356000780C9090790CA0907A0CB0907B0CDC01D8
:10357000CB0188199909AA09BB098C159D05AE05CF
:10358000BF050CF058C283E090E00E947C450E9489
:103590005D8A64E170E080E090E00E940189DDCF07
:1035A0000E94AD608AE99DE00E941D5344C267E11C
:1035B00075E08BE792E10E9456566BE772E1CE010F
:1035C00001960E9421574AE050E060E070E0CE0191
:1035D00001960E949192CE0101960E94C5563091AB
:1035E00061023CAF80918E0C811105C00E945D8A02
:1035F00081E080938E0C8091860C811105C00E9421
:103600005D8A81E08093860C1092850C1092840C68
:103610002090840C3090850C48E2241631040CF084
:103620007CC08CAD0E94B788F101EE0FFF1FE05007
:10363000F34F918380830E94B37120E030E040EA31
:1036400050E40E948DB120E030E040E85AE30E944F
:103650008DB12B013C0180901D0290901E02A09024
:103660001F02B0902002A50194016091190270918F
:103670001A0280911B0290911C020E94B7B29B011A
:10368000AC0160E070E080EC90E40E94B7B26B01A6
:103690007C0120E030E0A9010E9428B120E030E068
:1036A00040E650E4811105C0C301B2010E948DB112
:1036B0001EC0C301B2010E948DB1A50194010E94F8
:1036C000B8B220E030E040E850E40E94B7B2A70171
:1036D00096010E947EB320E030E040EC50E40E946E
:1036E0008DB120E030E040E850E40E94B8B2609331
:1036F000800C7093810C8093820C9093830C64E116
:1037000070E080E090E00E9401895FEF251A350AA1
:103710003092850C2092840C7BCFC090800CD0908E
:10372000810CE090820CF090830C20E030E0A90145
:10373000C701B6010E946DB487FD1EC022E0B7012B
:10374000A601CE0101960E94CA5667E776E0CE0137
:1037500080960E942957BE016F5F7F4FCE018096F1
:103760000E944556BC0181E892E10E94B056CE010C
:1037700080960E94C55649C168E075E081E892E1F3
:103780000E94565646C180910402882309F453C111
:103790008091D30C81112BC080917611811127C0AB
:1037A000C0905502D0905602E0905702F090580217
:1037B00020E030E04AE754E4C701B6010E948DB131
:1037C0000E9417B44B015C0120E030E040EA50E475
:1037D000C701B6010E948DB120E030E040EA50E41C
:1037E0000E94B8B20E9417B4A501940108C021E05C
:1037F00030E040E050E06AE070E080E090E00E945D
:10380000FF6319C1C7010E94BF9415C1C7010E947F
:103810008E4D11C180911F14882309F40CC165E6F7
:1038200075E0CE0101960E941957CE0101960E94C3
:10383000586AFDC08091FE0C9091FF0C892BA1F479
:1038400081E090E09093FF0C8093FE0C8EED93E06E
:103850009093C80C8093C70C0E941A7468EC70E0B7
:1038600080E090E00E94018968E575E0CE01019654
:103870000E94195744E650E06FEF7FEFCE010196AA
:103880000E944990CE0101960E94C556E0E0F0E00A
:103890001995D1C00E94F5890E94A1410E94BE7471
:1038A000CAC090917B1181E0892780937B11882386
:1038B00069F161E575E081E892E10E9456560E9447
:1038C0005D8A609372117093731180937411909359
:1038D000751180917E1190917F11181619065CF474
:1038E00020918011309181112817390724F010920E
:1038F0008111109280119091821180917D11981701
:103900005CF0109282111092831106C069E475E098
:1039100081E892E10E94565680917B118093761146
:1039200061E872E1CE0101960E9421574AE050E021
:1039300068E070E0CE0101960E949192CE0101965E
:103940000E94C5566CE375E0CE0101960E9419579E
:103950004AE050E06FEF7FEFCE0101960E94499060
:10396000CE0101960E94C5566EE275E081E892E1B3
:103970000E948C556FE979E0CE0101960E9429578B
:1039800061E872E1CE0101960E944556BC0181E8D2
:1039900092E10E94B056CE0101960E94C5568091D8
:1039A000D30C809384118CE291E00E94407480914A
:1039B000D30C882309F43FC066E278E08DE892E1F9
:1039C0000E949B5686EE9FEF9093980C8093970CE5
:1039D00032C0F092980CE092970C8AE99DE00E9428
:1039E0001D5360E275E081E892E10E94565664E65C
:1039F0007AE0CE0101960E9429574AE050E060E04B
:103A000070E0CE0101960E949192CE0101960E9433
:103A1000C55661E872E1CE0101960E9421574AE045
:103A200050E06FEF7FEFCE0101960E944990CE01EA
:103A300001960E94C556809185129091861200973A
:103A4000A1F0419720F4023011050CF0A3C061E809
:103A500072E1CE0101960E942157CE0101960E948B
:103A6000586ACE0101960E94C55664E670E080E077
:103A700090E00E940189A1C00E94C5410C94D40E1F
:103A8000EC80F12CFE2CEE248D81E80EF11CCE8012
:103A9000D12CDC2CCC248F81C80ED11CA884B12C55
:103AA000BA2CAA248985A80EB11C21E02CAF0C9455
:103AB000151266EC73E081E892E10E94565661E8C7
:103AC00072E1CE0180960E9421574AE050E060E00A
:103AD00070E0CE0180960E944990CE0180960E94AF
:103AE000C55663EB73E081E892E10E9456568091DF
:103AF0009D0C90919E0C029711F00C94E91210927B
:103B00009E0C10929D0C0C94E91284ED9EE00E9494
:103B10007F52892B71F084ED9EE00E945D52E1E0BE
:103B2000F0E0EC0FFD1FEE0DFF1D80832FEFE21A7A
:103B3000F20A65E070E080E090E00E94018936E0E2
:103B4000E316F10401F5998188A198131CC09A81AC
:103B500089A1981318C09B818AA1981314C08D81E4
:103B600090E0A0E0B0E0BA2FA92F982F88272C81F1
:103B7000820F911DA11DB11D480E591E6A1E7B1E8C
:103B80004FEF241A340A5FEF851A950AA50AB50A81
:103B90000C94871561E872E1CE0101960E942157CD
:103BA0004AE050E06FEF7FEFCE0101960E9449900E
:103BB000CE0101960E94C5564ACFCB5BDF4F0FB6B0
:103BC000F894DEBF0FBECDBFDF91CF911F910F9153
:103BD000FF90EF90DF90CF90BF90AF909F908F902D
:103BE0007F906F905F904F903F902F9008952F920D
:103BF0003F924F925F926F927F928F929F92AF927D
:103C0000BF92CF92DF92EF92FF920F931F93CF93C9
:103C1000DF93CDB7DEB728970FB6F894DEBF0FBE9F
:103C2000CDBFFC0180E290E19387828780911D10D7
:103C300090E0958784878091EA1090E09787868747
:103C400080911A10853009F063C6809122109091FE
:103C50002310885891098D35910588F480911D10A5
:103C6000843041F4809124109091251080974797DB
:103C700008F47DC080911D10843408F05EC08091EE
:103C80001D108A3108F4D5C0809120109091211028
:103C9000843F914050F4118610868FEF9FEFDC0136
:103CA00084839583A683B7833CC080912210909132
:103CB000231085974B9708F0BCC006E2E02E00E188
:103CC000F02E82E090E040E050E0BA018C010F5FFE
:103CD0001F4F20911D1030E0021713076CF497015D
:103CE00022503109D9012D913C91275031092730BB
:103CF000310508F47FC0C801019795958795918794
:103D000080870C971CF41186108693C044835583DA
:103D10006683778384E090E00DC044835583668397
:103D200077838BE090E006C0448355836683778376
:103D30008CE090E0918380831EC580912410909147
:103D40002510825491098E9708F099CF20E030E039
:103D5000C12CD12C7601A9014A5D5F4EDA014D914B
:103D60005C91495051094930510598F088CF8091B4
:103D70002610909127100997099708F07BCF11869C
:103D800010868FEF9FEFDC0184839583A683B78332
:103D9000C2C5B901685D7F4EDB014D915C91475111
:103DA000510942315105C0F4D701C601880F991F4E
:103DB000AA1FBB1F6C017D016894C0F82C5F3F4FA8
:103DC0002038310541F620E230E031872087C48277
:103DD000D582E682F7829FC5DB014D915C9146500A
:103DE00051094730510508F04ACFCC0CDD1CEE1CC0
:103DF000FF1CE4CFD7012D913C91235131092F3085
:103E0000310550F4440F551F661F771F416002961D
:103E1000B4E0EB0EF11C5ACFD7012D913C912A5002
:103E200031092930310528F4440F551F661F771FCB
:103E3000EECF80911D108A3108F460C0809120106F
:103E4000909121108032934008F425CF8091221068
:103E500090912310C697869708F050C08091241047
:103E600090912510C697869708F048C0B8E2EB2ECF
:103E7000B0E1FB2E83E090E040E050E0BA018C011D
:103E80000F5F1F4F20911D1030E00217130764F4DD
:103E9000970122503109D9012D913C912C503109C3
:103EA0002B30310560F0C801019795958795918772
:103EB00080870C970CF031CF118610861FC0D70178
:103EC0002D913C91255231092B31310550F4440F8D
:103ED000551F661F771F41600296B4E0EB0EF11C80
:103EE000CECFD7012D913C912C5031092A3031058C
:103EF00028F4440F551F661F771FEECF80911D10C9
:103F0000823208F452C080912210909123100697BB
:103F1000079708F04AC046E2C42E40E1D42E82E062
:103F200090E040E050E0BA018C010F5F1F4F2091FC
:103F30001D1030E002171307F4F4D6011297ED902C
:103F4000FC9011979D01BEE1EB1AF108A7E1EA167A
:103F5000F104E0F4440F551F661F771F4160D6013E
:103F60002D913C91B4E0CB0ED11C2350310925306A
:103F70003105C8F0C801019795958795918780878D
:103F800040970CF0D1CE118610860FC0D9012D912B
:103F90003C912C5031092B30310538F4440F551F1A
:103FA000661F771FDCCF0296BFCF7F011C821B826A
:103FB00081E090E09A83898380911D108D3070F4A8
:103FC0001C821B8281E090E09A838983F7018485BB
:103FD0009585181619060CF474C0D1C029E733E092
:103FE000AE014D5F5F4FBE016F5F7F4FC7010E9403
:103FF0001B9C892B29F729E733E0AE014D5F5F4F0A
:10400000BE016F5F7F4FC7010E941B9C0197C1F6E5
:1040100029E733E0AE014D5F5F4FBE016F5F7F4F19
:10402000C7010E941B9C892B59F6812C912C5401AD
:1040300000E010E080911D1090E029813A8128175E
:10404000390794F529E733E0AE014D5F5F4FBE01BC
:104050006F5F7F4FC7010E941B9C6C0129E733E013
:10406000AE014D5F5F4FBE016F5F7F4FC7010E9482
:104070001B9CF1E0CF16D10451F4892B09F0A0CF9D
:10408000880C991CAA1CBB1C689480F80AC0CD2817
:1040900009F096CF019709F093CF880C991CAA1CC0
:1040A000BB1C0F5F1F4FC6CFD70119961C930E93F1
:1040B0001897F70184829582A682B78281E090E00A
:1040C00039CE0284F385E02D82E090E09A838983E3
:1040D0008281938189974E9708F051C083E090E0E8
:1040E0009A838983848195810B970A9708F047C04A
:1040F0002CEB31E0AE014D5F5F4FBE016F5F7F4F34
:10410000C7010E941B9C892BD1F52CEB31E0AE013D
:104110004D5F5F4FBE016F5F7F4FC7010E941B9CC9
:10412000019769F5412C512C320100E010E0F701B4
:104130002485358589819A81821793070CF02FC1D8
:104140002CEB31E0AE014D5F5F4FBE016F5F7F4FE3
:10415000C7010E941B9C5C010330110509F0E5C0FA
:104160002CEB31E0AE014D5F5F4FBE016F5F7F4FC3
:10417000C7010E941B9CA816B90609F4D6C0D70136
:104180001A96ED91FC911B9782819381C697869731
:10419000E0F4848195814B974597B8F4DF0116963A
:1041A0006F0126ECC20ED11C20E030E040E050E070
:1041B00060E070E080E090E00D911C911197095053
:1041C00011090830110508F4F4C080911D108933DD
:1041D00070F182819381895791098335910508F4A3
:1041E0001BC125C0D90112966D917C911397665120
:1041F00071096131710508F037C1D501C401880F1B
:10420000991FAA1FBB1F4C015D01689480F84E5F87
:104210005F4F2C5F3F4F4B33510509F40CC1D9015F
:104220006D917C916A50710969307105D8F2809165
:104230001D10823231F4828193810A97099708F424
:1042400023C1828193818957910983359105D0F4E7
:1042500080911D108132B0F084819581CA97899731
:1042600088F49F012A5F3F4F812C912C540143E039
:1042700050E0D9016D917C916A50710969307105E6
:1042800008F41EC1828193818C549109C59778F4FA
:1042900080911D10843031F48481958180974797F7
:1042A00008F46CC180911D10843408F04EC18091D7
:1042B0001D10863460F1828193810C970B9708F46E
:1042C000A9C125C0D90112966D917C9113976E51A9
:1042D00071096731710508F0D1C1D501C401880F9A
:1042E000991FAA1FBB1F4C015D01689480F84E5FA7
:1042F0005F4F2C5F3F4F4534510509F4A6C1D901EA
:104300006D917C916C5071096B307105D8F2809180
:104310001D10883508F4E4C1828193818558910984
:104320008B35910508F4BAC1DBC12CEB31E0AE014D
:104330004D5F5F4FBE016F5F7F4FC7010E941B9CA7
:104340006C010330110579F42CEB31E0AE014D5FC7
:104350005F4FBE016F5F7F4FC7010E941B9CC81655
:10436000D90609F00CCFA114B10459F4CA94CD2890
:1043700009F005CF440C551C661C771C689440F866
:104380000BC0AA94AB2809F0FACECD2809F0F7CEDD
:10439000440C551C661C771C0F5F1F4FC8CE11873D
:1043A0000087F701448255826682778282E090E03E
:1043B000C1CC12960D911C911397015111090D302A
:1043C0001105E0F401E00E940EB621601496AC15D0
:1043D000BD0509F0F1CEF701248335834683578369
:1043E00000E20E9429B62283338385E090E0918326
:1043F000808380E390E091878087BDC112960D9104
:104400001C911397045011090530110508F0DDCEF9
:1044100001E00E940EB6DACF84819581CA97899710
:1044200008F005CF9F012A5F3F4F812C912C54014A
:1044300043E050E0F4CE9F012A583F4FD9012D911F
:104440003C912A5031092930310508F0F0CE2CE199
:1044500030E0F70131872087D70184829582A682D8
:10446000B7828AE090E085C1D90112966D917C9166
:104470001397665071096730710508F0D8CE880C23
:10448000991CAA1CBB1CC3CE20911D10CF01820F0A
:10449000911D820F911DDC0112978D919C910A97BD
:1044A000099708F0CECEF701118610868FEF9FEFA7
:1044B000DC0184839583A683B78386E090E03ACCC1
:1044C000D90112966D917C911397665171096131F2
:1044D000710558F5D501C401880F991FAA1FBB1F8C
:1044E0004C015D01689480F84E5F5F4F2C5F3F4F39
:1044F0004332510509F0BDCE9F012A5B3F4FD901E0
:104500002D913C912A5031092930310508F0BACE5D
:1045100020E130E0F70131872087D701848295823E
:10452000A682B78286E090E024C1D90112966D91EF
:104530007C911397665071096730710508F0A2CE1F
:10454000880C991CAA1CBB1CCFCF848195818954EF
:104550009109C39708F0ABCE9F012A5F3F4FAF018F
:104560004A575F4F812C912C5401D9016D917C9158
:104570006950710969307105B8F099CE86819781CB
:104580000997099708F08ECED70119961C921E92B2
:1045900018978FEF9FEFDC01F70184839583A68343
:1045A000B78387E090E0C6CBD90112966D917C91DC
:1045B00013976651710961317105E0F4D501C401A9
:1045C000880F991FAA1FBB1F4C015D01689480F8DA
:1045D0002C5F3F4F2417350741F620E230E0F7010A
:1045E00031872087D70184829582A682B78287E0AF
:1045F00090E0BFC0D90112966D917C9113976650DF
:1046000071096730710508F052CE880C991CAA1CFC
:10461000BB1CDECF848195810997099708F077CE7E
:10462000868197818C974F9708F071CE8085918510
:1046300089974D9708F06BCE9F01265F3F4F812CE5
:10464000912C540145E050E05ACE9F0126573F4F30
:10465000D9012D913C912C5031092B30310508F0B6
:1046600056CE20E230E0F70131872087D7018482DF
:104670009582A682B78288E090E07BC0D90112962D
:104680006D917C911397695071096930710508F03B
:104690003ECE880C991CAA1CBB1C29CE8481958116
:1046A000825491098E97E0F48F01045C1F4F8DE1D5
:1046B00090E040E050E020911D1030E0245031099E
:1046C000821793070CF063C0980122503109D90179
:1046D0002D913C91295031092830310508F46EC0E4
:1046E00080911D10803209F07EC0828193810697EF
:1046F000069708F078C0848195810997099708F09A
:1047000072C09F012A5F3F4FAF01425C5F4F812C17
:10471000912C5401D9016D917C91665071096630DC
:10472000710508F060C0D90112966D917C911397C4
:10473000695171096331710508F0D5C0D501C40113
:10474000880F991FAA1FBB1F4C015D01689480F858
:104750002C5F3F4F24173507E9F62EE030E0F701D4
:1047600031872087D70184829582A682B7828FE025
:1047700090E08D939C9381E090E0D0C0D8012D9182
:104780003C91285131092231310550F1CB0101977B
:1047900095958795D70119969C938E9318978A972C
:1047A0000CF49ECF052E000C660B770BF7014483AB
:1047B00055836683778389E090E0BCCABC016F5F54
:1047C0007F4FD8012D913C91275031092730310579
:1047D000A8F6440F551F416002960C5F1F4F6BCF28
:1047E000440F551FF9CFD7011C962D903C901D9773
:1047F000B6E02B1631040CF486C08F010E5F1F4FFC
:1048000075EC872E7DE9972E7CE1A72E71E8B72EF7
:10481000E3E0CE2ED12CF801648175816080718037
:1048200080E090E00E942CB16D837E838F83988717
:10483000B30180E090E00E942CB12B013C012DECF3
:104840003CEC4CE45FE30E948DB19B01AC016D81B7
:104850007E818F8198850E9428B187FD19C02DEC3B
:104860003CEC4CE45FE36D817E818F8198850E94F2
:104870008DB19B01AC01C301B2010E9428B1E82FA8
:10488000880FFF0BEE27FF0FEE1FFF27319602C0A8
:10489000E0E0F0E0A501940163E971E080E091E0DF
:1048A0000E94D0B54F01FF0FAA08BB0886269726A5
:1048B000A826B926FFEFCF1ADF0A0E5F1F4F2C1470
:1048C0003D0409F0A8CFD70114968D929D92AD9228
:1048D000BC92179780E290E019969C938E9318975C
:1048E0008FEF9FEF46CFD90112966D917C91139770
:1048F000695071096930710508F075CF880C991CF1
:10490000AA1CBB1C25CF82E080931A1010921D10A8
:1049100080E090E003C083E090E00CCA28960FB6D8
:10492000F894DEBF0FBECDBFDF91CF911F910F91E5
:10493000FF90EF90DF90CF90BF90AF909F908F90BF
:104940007F906F905F904F903F902F9008955F926F
:104950006F927F928F929F92AF92BF92CF92DF928F
:10496000EF92FF920F931F93CF93DF93CDB7DEB7F4
:10497000E4970FB6F894DEBF0FBECDBF66E277E0D6
:10498000CE010B960E942957BE01655F7F4F89E9D2
:1049900092E10E94F187811116C06CE277E0CE01AE
:1049A00001960E942957BE016F5F7F4F89E992E10E
:1049B0000E94F18711E0811101C010E0CE01019643
:1049C0000E94C55601C011E0CE010B960E94C5564B
:1049D000112309F476C026E030E045E050E069E9B3
:1049E00072E1CE0101960E943D57BE016F5F7F4F7D
:1049F0008BE792E10E94E255CE0101960E94C556D6
:104A00008BE792E10E9410556B017C0169E67BE027
:104A1000CE0101960E942957BE016F5F7F4F89E941
:104A200092E10E94A187AC014F5F5F4F69E972E19B
:104A3000CE010B960E94EC41BE01655F7F4F8BE774
:104A400092E10E94E255CE010B960E94C556CE011E
:104A500001960E94C5568BE792E10E9410559B017A
:104A6000E7E0F2E041E050E0A0910702B0910802D7
:104A7000A417B5075CF0A281B3812A173B0711F494
:104A8000138212824F5F5F4F3296EECF9601220F54
:104A9000331FF901E95FFD4F7183608382E090E08D
:104AA0000E94157669E972E1CE0101960E942157B4
:104AB000CE0101960E946592CE0101960E94C556D4
:104AC00049C062E377E0CE010B960E942957BE01F0
:104AD000655F7F4F89E992E10E94F187811116C0DD
:104AE00068E377E0CE0101960E942957BE016F5F0F
:104AF0007F4F89E992E10E94F18711E0811101C0A5
:104B000010E0CE0101960E94C55601C011E0CE0111
:104B10000B960E94C556112349F1E7E0F2E081E0CF
:104B200090E020910702309108022817390774F0AD
:104B3000863091051CF49383828305C09C012E5F0F
:104B40003F4F3383228301963296EBCF82E090E091
:104B50000E9415761092C80C1092C70C80E090E06D
:104B60000E946A74109254020C94B7306EE377E09E
:104B7000CE010B960E942957BE01655F7F4F89E9E0
:104B800092E10E94F187811116C065E477E0CE01C1
:104B900001960E942957BE016F5F7F4F89E992E11C
:104BA0000E94F18711E0811101C010E0CE01019651
:104BB0000E94C55601C011E0CE010B960E94C55659
:104BC0001123F9F08091FE0C9091FF0C892BA1F438
:104BD00081E090E09093FF0C8093FE0C8EED93E0CB
:104BE0009093C80C8093C70C0E941A7468EC70E014
:104BF00080E090E00E940189E0E0F0E019950C94DB
:104C0000B7306CE477E0CE010B960E942957BE01C5
:104C1000655F7F4F89E992E10E94F187811116C09B
:104C200064E577E0CE0101960E942957BE016F5FCF
:104C30007F4F89E992E10E94F18711E0811101C063
:104C400010E0CE0101960E94C55601C011E0CE01D0
:104C50000B960E94C5561123B1F06CE577E0CE01AA
:104C600001960E9429576AE673E1CE0101960E94DF
:104C70004556BC0181E892E10E94B056CE010196F2
:104C80000E94C55638C066E677E0CE010B960E94BA
:104C90002957BE01655F7F4F89E992E10E94F18744
:104CA000811116C06DE677E0CE0101960E9429576A
:104CB000BE016F5F7F4F89E992E10E94F18711E0A9
:104CC000811101C010E0CE0101960E94C55601C0BD
:104CD00011E0CE010B960E94C556112351F16CE5EF
:104CE00077E081E892E10E94565660E773E181E83F
:104CF00092E10E94DC556FE979E0CE0101960E94B5
:104D0000295761E872E1CE0101960E944556BC0127
:104D1000CE010B960E942157CE010B960E94586A35
:104D2000CE010B960E94C556CE0101960E94C55633
:104D300019CF64E777E0CE010B960E942957BE0198
:104D4000655F7F4F89E992E10E94F187811116C06A
:104D50006AE777E0CE0101960E942957BE016F5F96
:104D60007F4F89E992E10E94F18711E0811101C032
:104D700010E0CE0101960E94C55601C011E0CE019F
:104D80000B960E94C556112311F169E377E081E883
:104D900092E10E94565661E872E1CE0101960E94AE
:104DA0002157CE0101960E94586ACE0101960E94B9
:104DB000C5560E9404811092540266E777E089E9A3
:104DC00092E10E949B560E9457810C94B73060E894
:104DD00077E0CE010B960E942957BE01655F7F4F99
:104DE00089E992E10E94F187811116C067E877E0B6
:104DF000CE0101960E942957BE016F5F7F4F89E95E
:104E000092E10E94F18711E0811101C010E0CE0112
:104E100001960E94C55601C011E0CE010B960E947A
:104E2000C556112309F48CC069E67BE0CE010196DA
:104E30000E942957BE016F5F7F4F89E992E10E946E
:104E4000A187AC014F5F5F4F69E972E1CE010B961C
:104E50000E94EC41BE01655F7F4F8BE792E10E94AB
:104E6000E255CE010B960E94C556CE0101960E94D6
:104E7000C5568BE792E10E9410558B016CE277E0FA
:104E800081E892E10E94565680917B11882331F08F
:104E900060E277E081E892E10E9456560115110523
:104EA00011F40C94A330CE0101960E944A4CCE011D
:104EB00001960E94586ACE0101960E94C5560230A2
:104EC00011050CF44FCE67E775E0CE010B960E94FA
:104ED0001957BE01655F7F4FCE0101960E94215791
:104EE000CE0101960E94586ACE0101960E94C556D5
:104EF000E12CF12C80917D11082E000C990BE81605
:104F0000F9068CF4B701CE0101960E942F4BCE0119
:104F100001960E94586ACE0101960E94C556FFEF85
:104F2000EF1AFF0AE7CFCE010B960E94C55602305A
:104F3000110509F417CE8CE291E00E94947412CE10
:104F40006EE877E0CE010B960E942957BE01655F9F
:104F50007F4F89E992E10E94F187811116C065E9CE
:104F600077E0CE0101960E942957BE016F5F7F4F07
:104F700089E992E10E94F18711E0811101C010E0FE
:104F8000CE0101960E94C55601C011E0CE010B96DC
:104F90000E94C556112309F488C369E972E1CE0164
:104FA0008F960E94215769E67BE0CE0101960E9410
:104FB0002957BE016F5F7F4FCE018F960E94A18758
:104FC000AC014F5F5F4FBE01615D7F4FCE0189969F
:104FD0000E94EC41CE0101960E94C556BE01615D62
:104FE0007F4FCE0101960E942157CE0101960E946B
:104FF0006592CE0101960E94C55662E977E0CE0126
:1050000001960E942957BE016F5F7F4FCE0189969E
:105010000E9465878C01CE0101960E94C55664E608
:105020007AE0CE0183960E94295764E67AE0CE01A9
:105030004D960E9429571016110684F5A8014F5F5E
:105040005F4F8DA59EA54817590790F4BE01675D77
:105050007F4FCE0101960E94EC41BE016F5F7F4FF2
:10506000CE0183960E94E255CE0101960E94C5565C
:10507000980140E050E0BE01675D7F4FCE01019690
:105080000E943D57BE016F5F7F4FCE014D960E943B
:10509000E255CE0101960E94C5560DC064E67AE045
:1050A000CE0183960E949B56BE01675D7F4FCE0165
:1050B0004D960E94B05689A19AA1892B09F4E6C2A7
:1050C000CE014D960E9410557B0121E0E21AF108B5
:1050D00048E1E416F1041CF027E1E22EF12CF7FE82
:1050E00003C0EE24EA94FE2CB701CE010B960E9479
:1050F0005A5B64E977E0CE0101960E942957BE0110
:10510000655F7F4FCE0101960E944556BC01CE01DE
:1051100041960E942157CE0141960E946592CE0190
:1051200041960E94C556CE0101960E94C556CE01F9
:105130000B960E94C556BE016D5D7F4FCE018996CC
:105140000E94B05662E977E0CE0101960E9429578D
:10515000BE016F5F7F4FCE0189960E9465878C01EB
:10516000CE0101960E94C55664E67AE0CE01839690
:105170000E949B5664E67AE0CE014D960E949B56B3
:10518000101611060CF04DC0A8014F5F5F4F8DA5A2
:105190009EA54817590790F4BE01675D7F4FCE0169
:1051A00001960E94EC41BE016F5F7F4FCE01839656
:1051B0000E94E255CE0101960E94C556980140E03A
:1051C00050E0BE01675D7F4FCE0101960E943D57C2
:1051D000BE016F5F7F4FCE014D960E94E255CE011A
:1051E00001960E94C5568E010F5F1F4FC12CD12C16
:1051F000A7014F5F5F4F8AE0849F9001859F300D2C
:105200001124F901E558FE4E5F018E9D90018F9D9E
:10521000300D1124A90147575E4E3A018AE2582EFB
:10522000C0C064E67AE0CE0183960E949B56BE0120
:10523000675D7F4FCE014D960E94B056D4CFCE0110
:105240004D96C114D10409F0B9C05FEFE516F5061B
:1052500009F4B4C00E941B55A114B10439F044E014
:1052600050E0B501CE014D960E947F87B501CE0179
:1052700041960E94295769E977E0CE010B960E947A
:105280002957BE016F5E7F4FCE010B960E94455697
:10529000BC01CE0147960E942157CE0147960E943D
:1052A0006592CE0147960E94C556CE010B960E948C
:1052B000C556CE0141960E94C55689A19AA1029772
:1052C00008F475C061E070E0CE014D960E947B55F8
:1052D000082E000C990B803391050CF44C96E52DAB
:1052E000E81B8E2FF3018083FFEFCF1ADF0ABE0188
:1052F0006D5D7F4FCE0189960E94B05662E977E0DE
:10530000CE010B960E942957BE01655F7F4FCE01EB
:1053100089960E9465874C01CE010B960E94C55666
:1053200064E67AE0CE0183960E949B5664E67AE0BA
:10533000CE014D960E949B56181419040CF044C0DF
:10534000A4014F5F5F4F8DA59EA54817590790F4A4
:10535000BE01675D7F4FCE010B960E94EC41BE01FE
:10536000655F7F4FCE0183960E94E255CE010B967A
:105370000E94C556940140E050E0BE01675D7F4F3A
:10538000CE010B960E943D57BE01655F7F4FCE0157
:105390004D960E94E255CE010B960E94C5560E5FB7
:1053A0001F4F89A19AA1892B09F049CF1BC0CE01BB
:1053B0004D960E941055F301608396CF0E941055C0
:1053C000F8017183608390CF64E67AE0CE01839622
:1053D0000E949B56BE01675D7F4FCE014D960E9495
:1053E000B056DDCF2FEFE216F20609F07DC062E97C
:1053F00077E0CE010B960E942957BE01655F7F4F73
:10540000CE0183960E9465878C01CE010B960E9487
:10541000C55617FF3BC109811A811016110634F4D5
:10542000093111052CF008E110E002C001E010E0A4
:1054300000937D11B801CE0141960E945A5B67EA44
:1054400077E0CE010B960E942957BE016F5E7F4F19
:10545000CE010B960E944556BC01CE0147960E9494
:105460002157CE0147960E946592CE0147960E9431
:10547000C556CE010B960E94C556CE0141960E949C
:10548000C556C114D10459F18B819C8197FF02C08C
:1054900080E090E090937F1180937E1141E0C416EC
:1054A000D104E9F08D819E81181619062CF480171D
:1054B000910724F48C0102C001E010E00150009338
:1054C000821152E0C516D10451F08F8198851816CB
:1054D000190614F081E090E08150809383118CE2F2
:1054E00091E00E944074D2C080917C11082E000C83
:1054F000990BE816F9060CF083C0B601CE0141966F
:105500000E945A5B61EB77E0CE010B960E9429570F
:10551000BE016F5E7F4FCE010B960E944556BC01C7
:10552000CE0147960E942157CE0147960E94659270
:10553000CE0147960E94C556CE010B960E94C556D5
:10554000CE0141960E94C5568AE08E9DF0018F9D46
:10555000F00D1124E558FE4E81E0878783E090E04E
:10556000918B808B938B828BC114D10409F48EC0F4
:105570008B819C818038910514F08FE790E0803812
:105580002FEF920714F480E89FEF878741E0C4165D
:10559000D10409F47BC08AE08E9DF0018F9DF00D4F
:1055A0001124E558FE4E8D819E8197FF02C080E058
:1055B00090E0918B808B52E0C516D10409F466C04F
:1055C0008AE08E9DF0018F9DF00D1124E558FE4E6E
:1055D0008F81988597FF02C080E090E0938B828B4B
:1055E00080917D11082E000C990BE816F9061CF02D
:1055F000E394E0927D118CE291E00E94947446C0A5
:10560000BE016D5D7F4FCE0147960E94215760918C
:105610007C11062E000C770BCE0141960E945A5B3E
:1056200069EB77E0CE010B960E942957BE01695EB7
:105630007F4FCE010B960E9445566AEC77E00E94A0
:105640002E56BE016F5E7F4F0E944556BC01CE01B3
:1056500047960E94B056CE010B960E94C556CE01C9
:1056600041960E94C556BE01695E7F4FCE010B96E2
:105670000E942157CE010B960E94586ACE010B96CC
:105680000E94C556CE0147960E94C556CE014D9642
:105690000E94C556CE0183960E94C556CE018996BA
:1056A0000E94C556CE018F968EC26EEC77E0CE0179
:1056B0000B960E942957BE01655F7F4F89E992E1F1
:1056C0000E94F187811116C063ED77E0CE0101964B
:1056D0000E942957BE016F5F7F4F89E992E10E94C6
:1056E000F18711E0811101C010E0CE0101960E9406
:1056F000C55601C011E0CE010B960E94C55611237C
:10570000C9F169E67BE0CE0101960E942957BE01EE
:105710006F5F7F4F89E992E10E94A187AC014F5FE3
:105720005F4F69E972E1CE010B960E94EC41BE0128
:10573000655F7F4F8BE792E10E94E255CE010B96A9
:105740000E94C556CE0101960E94C5568BE792E194
:105750000E9410556115710521F481E080932E059A
:1057600006C06130710509F0FDC910922E050E9436
:10577000CE74F8C968ED77E0CE010B960E942957E8
:10578000BE01655F7F4F89E992E10E94F187811137
:1057900016C06CED77E0CE0101960E942957BE013C
:1057A0006F5F7F4F89E992E10E94F18711E08111DB
:1057B00001C010E0CE0101960E94C55601C011E063
:1057C000CE010B960E94C556112309F466C143E031
:1057D00050E069E972E1CE0101960E94EC41BE0100
:1057E0006F5F7F4F8BE792E10E94E255CE010196F9
:1057F0000E94C5566BE772E1CE0101960E942157C7
:10580000CE0101960E946592CE0101960E94C55676
:105810001092C80C1092C70C6BE772E1CE01019692
:105820000E94215760E0CE0101960E94BB55811174
:1058300004C0CE0101960E941C56BE016F5F7F4FCF
:1058400086E793E10E94B056CE0101960E94C556AC
:105850006BE772E1CE0101960E94215760E0CE0114
:1058600001960E94BB55811104C0CE0101960E9491
:105870001C56BE016F5F7F4F80E793E10E94B056D8
:10588000CE0101960E94C55640917A1350917B1328
:105890004115510549F088E091E1009729F0BC01DC
:1058A00086E793E10E947F874091741350917513AE
:1058B0004115510549F086E691E1009729F0BC01B8
:1058C00080E793E10E947F878091C70C9091C80C7C
:1058D0000E946A746DEF76E0CE0101960E9429570E
:1058E0006BE772E1CE0101960E944556BC01CE01E4
:1058F00041960E942157CE0101960E94C556809183
:10590000621190916311892B39F4BE016F5E7F4F54
:105910008AE99DE00E94875768EB7BE080E090E099
:105920000E9401898091621190916311029709F0A0
:105930009BC06BE772E1CE0147960E94215760EE53
:1059400077E0CE0101960E942957CE0101960E9470
:1059500053ACCE0101960E94C55664EF71E080E021
:1059600090E00E94018963EE77E0CE0101960E94EB
:105970002957CE0101960E9453ACCE0101960E9498
:10598000C55664EF71E080E090E00E9401896CEE02
:1059900077E0CE0101960E942957CE0101960E9420
:1059A00053ACCE0101960E94C55664EF71E080E0D1
:1059B00090E00E94018965EF77E0CE0101960E9498
:1059C0002957CE0101960E9453ACCE0101960E9448
:1059D000C55664EF71E080E090E00E94018963E0C9
:1059E00078E0CE0101960E942957CE0101960E94CF
:1059F00053ACCE0101960E94C55664EF71E080E081
:105A000090E00E9401896DEF76E0CE0101960E9440
:105A10002957BE01695E7F4FCE0101960E9445560F
:105A2000BC01CE010B960E942157CE0101960E9427
:105A3000C556CE010B960E941B55BE01655F7F4F78
:105A4000CE0101960E942157CE0101960E9453ACCF
:105A5000CE0101960E94C556CE010B960E94C556F6
:105A6000CE0147960E94C55668EB7BE080E090E04F
:105A70000E94018968E071E1CE0101960E942957D8
:105A8000CE0101960E946592CE0101960E94C556F4
:105A900010925402CE01419696C061E178E0CE01A9
:105AA0000B960E942957BE01655F7F4F89E992E1FD
:105AB0000E94F187811116C066E178E0CE0101965F
:105AC0000E942957BE016F5F7F4F89E992E10E94D2
:105AD000F18711E0811101C010E0CE0101960E9412
:105AE000C55601C011E0CE010B960E94C556112388
:105AF00009F46CC044E050E069E972E1CE0101961E
:105B00000E94EC41BE016F5F7F4F8BE792E10E94E4
:105B1000E255CE0101960E94C55665E077E0CE01C0
:105B20000B960E9429576BE772E1CE010B960E94FB
:105B30004556BC01CE0101960E942157CE010B961D
:105B40000E94C5568091621190916311892B39F49E
:105B5000BE016F5F7F4F8AE99DE00E94875768EB27
:105B60007BE080E090E00E94018980916211909139
:105B70006311029779F4BE016F5F7F4FCE010B96E0
:105B80000E942157CE010B960E9453ACCE010B967A
:105B90000E94C55668EB7BE080E090E00E9401899E
:105BA000BE016F5F7F4FCE010B960E942157CE0141
:105BB0000B960E946592CE010B960E94C5561092DC
:105BC0005402CE0101960E94C556D1C26BE178E025
:105BD000CE010B960E942957BE01655F7F4F89E970
:105BE00092E10E94F187811116C06FE178E0CE0149
:105BF00001960E942957BE016F5F7F4F89E992E1AC
:105C00000E94F18711E0811101C010E0CE010196E0
:105C10000E94C55601C011E0CE010B960E94C556E8
:105C2000112309F463C069E972E18BE792E10E94F4
:105C3000B05681E08093540269E972E1CE01019689
:105C40000E942157CE0101960E946592CE010196D5
:105C50000E94C5568091621190916311029709F1DB
:105C60006BE772E18AE99DE00E94875768EB7BE071
:105C700080E090E00E940189CE0101960E941A6F97
:105C8000BE016F5F7F4F89E992E10E94E255CE012C
:105C900001960E94C55660ED77E080E090E00E949A
:105CA00001898091621190916311029771F46BE701
:105CB00072E1CE0101960E942157CE0101960E9409
:105CC00053ACCE0101960E94C55680919D129091D1
:105CD0009E12892B11F40C94B2256FE979E0CE0164
:105CE00001960E94295769E972E10DC863E278E0E4
:105CF000CE010B960E942957BE01655F7F4F89E94F
:105D000092E10E94F187811116C069E278E0CE012C
:105D100001960E942957BE016F5F7F4F89E992E18A
:105D20000E94F18711E0811101C010E0CE010196BF
:105D30000E94C55601C011E0CE010B960E94C556C7
:105D4000112309F45DC08091621190916311019754
:105D500011F00C94B225CE0101960E94C1508D81A4
:105D60009E81009709F4F9C1E981FA8120812223FB
:105D700009F4F3C1079708F4F0C167E177E0CE01B9
:105D80000B960E94195748EC50E06FEF7FEFCE0161
:105D90000B960E943693CE010B960E94C556BE010B
:105DA0006F5F7F4FCE010B960E94215740ED57E069
:105DB0006FEF7FEFCE010B960E944990CE010B96BC
:105DC0000E94C5566FE278E0CE010B960E942957DB
:105DD00069E972E1CE010B960E944556BC01CE01E5
:105DE00041960E942157CE0141960E94586ACE01E9
:105DF00041960E94C556CE010B960E94C556ADC174
:105E00006DE378E0CE010B960E942957BE01655FD5
:105E10007F4F89E992E10E94F187811116C062E407
:105E200078E0CE0101960E942957BE016F5F7F4F37
:105E300089E992E10E94F18711E0811101C010E02F
:105E4000CE0101960E94C55601C011E0CE010B960D
:105E50000E94C556112361F125E030E044E050E096
:105E600069E972E1CE0101960E943D57BE016F5F64
:105E70007F4F8BE792E10E94E255CE0101960E948E
:105E8000C55669E972E1CE0101960E942157CE0103
:105E900001960E946592CE0101960E94C5568BE73D
:105EA00092E10E941055CB010E94EF930C94B22511
:105EB00067E478E0CE010B960E942957BE01655F2A
:105EC0007F4F89E992E10E94F187811116C06EE44B
:105ED00078E0CE0101960E942957BE016F5F7F4F87
:105EE00089E992E10E94F18711E0811101C010E07F
:105EF000CE0101960E94C55601C011E0CE010B965D
:105F00000E94C556112361F127E030E046E050E0E1
:105F100069E972E1CE0101960E943D57BE016F5FB3
:105F20007F4F8BE792E10E94E255CE0101960E94DD
:105F3000C5568BE792E10E941055672B19F4109219
:105F40001F1403C081E080931F1469E972E1CE0140
:105F500001960E942157CE0101960E946592FDC0D4
:105F600065E578E0CE0101960E942957BE016F5F7A
:105F70007F4F89E992E10E94F187182FCE010196A7
:105F80000E94C556112309F476C080919D1290910C
:105F90009E12079708F4EBC046E050E069E972E111
:105FA000CE0101960E94EC41BE016F5F7F4F8BE7EF
:105FB00092E10E94E255CE0101960E94C5568BE700
:105FC00092E10E94055560935002709351028093B4
:105FD00052029093530267E077E081E892E10E94D9
:105FE0005656409150025091510260915202709168
:105FF000530221E0CE0101960E94CA56BE016F5F96
:106000007F4FCE010B960E9421576EED75E0CE01B9
:106010000B960E942E56BC0181E892E10E94DC554D
:10602000CE010B960E94C556CE0101960E94C55620
:1060300061E872E1CE0101960E942157CE010196DE
:106040000E94586ACE0101960E94C5560E945D8A40
:1060500028EE33E040E050E00E9486B2CA01B90168
:106060000E942CB16093CF0C7093D00C8093D10C14
:106070009093D20C7CC06CE578E0CE0101960E9432
:106080002957BE016F5F7F4F89E992E10E94F18736
:10609000182FCE0101960E94C556112309F463C042
:1060A00080919D1290919E12079708F460C046E07F
:1060B00050E069E972E1CE0101960E94EC41BE0117
:1060C0006F5F7F4F8BE792E10E94E255CE01019610
:1060D0000E94C5568BE792E10E94055560935502D8
:1060E00070935602809357029093580267EF76E0C0
:1060F00081E892E10E945656409155025091560215
:10610000609157027091580221E0CE0101960E94E1
:10611000CA56BE016F5F7F4FCE010B960E9421577A
:106120006EED75E0CE010B960E942E56BC0181E803
:1061300092E10E94DC55CE010B960E94C556CE011D
:1061400001960E94C55661E872E1CE0101960E9457
:106150002157CE0101960E94586ACE0101960E94F5
:10616000C5560C94B2252ED0182F8823A1F010917B
:106170005402112379F069E972E1CE0101960E947F
:106180002157CE0101960E946592CE0101960E9490
:10619000C55601C011E0812FE4960FB6F894DEBF1A
:1061A0000FBECDBFDF91CF911F910F91FF90EF9068
:1061B000DF90CF90BF90AF909F908F907F906F9027
:1061C0005F9008952F923F924F925F926F927F92CD
:1061D0008F929F92AF92BF92DF92EF92FF920F93B6
:1061E0001F93CF93DF93CDB7DEB7A8970FB6F89480
:1061F000DEBF0FBECDBF7E0145E1E40EF11C60E9BC
:1062000078E0C7010E942957B70189E992E10E940D
:10621000F187811117C066E07AE0CE0101960E94F5
:106220002957BE016F5F7F4F89E992E10E94F18794
:10623000DD24D394811101C0D12CCE0101960E949E
:10624000C55602C0DD24D394C7010E94C556DD2087
:1062500009F4DFC080919D1290919E12409718F032
:10626000D12C0C94CC3B42E050E069E972E1CE01C4
:1062700001960E94EC41BE016F5F7F4F8BE792E178
:106280000E94E255CE0101960E94C5566BE772E16D
:10629000CE0101960E942157CE0101960E9465927F
:1062A000CE0101960E94C5568BE792E10E940555EA
:1062B00020E030E048EC52E40E948DB10E9417B417
:1062C000AB01BC01409343025093440260934502EA
:1062D00070934602CE0101960E946870CE0101962D
:1062E0000E946592CE0101960E94C55660914302BC
:1062F0007091440280914502909146028B019C016D
:1063000000591F452140310901341C49210531053F
:10631000D0F063E678E0CE0101960E9429576BE742
:1063200072E1CE0101960E94455666E778E00E9430
:106330002E56BC0181E892E10E94B056CE01019632
:106340000E94C5564BC01A821982FE01339626E080
:10635000DF011D922A95E9F70E942EB120E030E07E
:1063600048EC52E40E947EB38E010F5F1F4F22E083
:1063700047E00E9498ACBC0181E892E10E949B56E4
:1063800066E878E0C7010E94295761E872E1C70119
:106390000E94455663E978E00E942E56BC0181E8D0
:1063A00092E10E94B056C7010E94C5561092C80CD7
:1063B0001092C70C8091430290914402A091450233
:1063C000B09146028093EC109093ED10A093EE10E4
:1063D000B093EF1080E090E00E946A746FE979E07A
:1063E000CE0101960E94295761E872E1CE01019623
:1063F0000E944556BC01C7010E942157C7010E9457
:10640000586AC7010E94C556CE0101960E94C55622
:10641000BCC768E978E0C7010E942957B70189E93C
:1064200092E10E94F187811117C06DE978E0CE01F9
:1064300001960E942957BE016F5F7F4F89E992E163
:106440000E94F187DD24D394811101C0D12CCE01AB
:1064500001960E94C55602C0DD24D394C7010E9454
:10646000C556DD20C1F126E030E044E050E069E9A6
:1064700072E1CE0101960E943D57BE016F5F7F4FD2
:106480008BE792E10E94E255CE0101960E94C5562B
:106490008BE792E10E94105570936511609364112F
:1064A00070932A026093290269E972E1CE01019694
:1064B0000E942157CE0101960E946592CE0101965D
:1064C0000E94C5561092C80C1092C70C80E090E054
:1064D0000E946A745AC762EA78E0CE0183960E94ED
:1064E0002957BE016D5D7F4F89E992E10E94F187D6
:1064F000811129C065EA78E0C7010E942957B701D8
:1065000089E992E10E94F187811117C068EA78E079
:10651000CE0101960E942957BE016F5F7F4F89E926
:1065200092E10E94F187DD24D394811101C0D12C26
:10653000CE0101960E94C55602C0DD24D394C70146
:106540000E94C55602C0DD24D394CE0183960E94DA
:10655000C556DD2009F45EC10AE010E0412C512C43
:106560003201AA24AA9443E0B42E6EE170E080E0E8
:1065700090E00E940189809161020E94B788B50174
:106580000E94F3B5072E000C880B990B0E942EB1C8
:1065900020E030E040EA50E40E948DB19B01AC0164
:1065A000C301B2010E94B8B22B013C010150110994
:1065B000E1F620E030E040E251E40E947EB32B019E
:1065C0003C016BEA78E0CE0183960E942957BE0118
:1065D0006D5D7F4F89E992E10E94F18781110C94F2
:1065E000C03B6FEA78E0C7010E942957B70189E9EB
:1065F00092E10E94F187811116C063EB78E0CE0131
:1066000001960E942957BE016F5F7F4F89E992E191
:106610000E94F18711E0811101C010E0CE010196C6
:106620000E94C55601C01D2DC7010E94C556CE014E
:1066300083960E94C556112309F446C020E030E03D
:1066400040E650E4C301B2010E948DB19B01AC0150
:1066500060E070E080E890E40E94B7B260931D02B1
:1066600070931E0280931F029093200268ED78E0E1
:1066700081E892E10E94565640911D0250911E02FF
:1066800060911F027091200222E0CE0101960E94CB
:10669000CA56BE016F5F7F4F81E892E10E94DC55D0
:1066A000CE0101960E94C55680911D0290911E0256
:1066B000A0911F02B09120028093101190931111AC
:1066C000A0931211B093131167EB78E0CE0183967B
:1066D0000E942957BE016D5D7F4F89E992E10E94BA
:1066E000F18781110C94C63B6CEB78E0C7010E94E6
:1066F0002957B70189E992E10E94F187811116C0FB
:1067000061EC78E0CE0101960E942957BE016F5FCF
:106710007F4F89E992E10E94F18711E0811101C068
:1067200010E0CE0101960E94C55601C01D2DC70183
:106730000E94C556CE0183960E94C556112309F4C6
:106740004EC020E030E040E650E4C301B2010E94B8
:106750008DB19B01AC0160E070E080E291E40E94A9
:10676000B7B26093190270931A0280931B02909340
:106770001C0267EC78E081E892E10E945656409155
:10678000190250911A0260911B0270911C0222E0C2
:10679000CE0101960E94CA56BE016F5F7F4F81E80D
:1067A00092E10E94DC55CE0101960E94C55680916F
:1067B000190290911A02A0911B02B0911C028093C1
:1067C000141190931511A0931611B09317111092F4
:1067D000C80C1092C70C80E090E00E946A746FE9C8
:1067E00079E0CE0101960E94295761E872E1CE015D
:1067F00001960E944556BC01C7010E942157C7015E
:106800000E94586AC7010E94C556CE0101960E9497
:10681000C556C2C766EC78E0C7010E942957B70188
:1068200089E992E10E94F187811117C06CEC78E050
:10683000CE0101960E942957BE016F5F7F4F89E903
:1068400092E10E94F187DD24D394811101C0D12C03
:10685000CE0101960E94C55602C0DD24D394C70123
:106860000E94C556DD2009F4BFC080919D12909111
:106870009E120797F8F046E050E069E972E1CE0118
:1068800001960E94EC41BE016F5F7F4F8BE792E162
:106890000E94E255CE0101960E94C5568BE792E117
:1068A0000E9405556093250270932602809327026B
:1068B0009093280280915F029091600299270E9434
:1068C0002477BC01990F880B990B0E942EB12DE003
:1068D00038E643E55BE30E948DB12B013C0120913A
:1068E00083023091840240918502509186020E9479
:1068F00028B118164CF060916B0270916C02809177
:106900006D0290916E021BC0209197023091980207
:106910004091990250919A02C301B2010E946DB454
:1069200087FF05C0C301B2010E94D87208C0609100
:106930007F0270918002809181029091820220E01A
:1069400030E048EC52E40E948DB12B013C0120E084
:1069500030E0A9010E9428B1181634F0412C512CC6
:1069600038EA632E31E4732E4092250250922602BB
:1069700060922702709228024092201150922111B9
:10698000609222117092231180911F14882381F04C
:1069900065EB78E081E79FE00E94955760912502C2
:1069A0007091260280912702909128020E94E55C56
:1069B0001092C80C1092C70C80E090E00E946A749C
:1069C0006BEA78E081E892E10E94565640912502F8
:1069D00050912602609127027091280222E0CE0198
:1069E00001960E94CA5686C262ED78E0C7010E94F5
:1069F0002957B70189E992E10E94F187811117C0F7
:106A000066ED78E0CE0101960E942957BE016F5FC6
:106A10007F4F89E992E10E94F187DD24D3948111AF
:106A200001C0D12CCE0101960E94C55602C0DD24C2
:106A3000D394C7010E94C556DD2009F46DC0B09003
:106A40005D0260E08B2D0E947B8809E110E0412C03
:106A5000512C32018B2D0E94B788BC01990F880BF5
:106A6000990B0E942EB19B01AC01C301B2010E949F
:106A7000B8B22B013C016AE070E080E090E00E9437
:106A800001890150110931F720E030E040EA50E47B
:106A9000C301B2010E948DB120E030EC4FE754E415
:106AA0000E947EB320E030E048EC51E40E947EB3C7
:106AB0006093210270932202809323029093240218
:106AC0006093361170933711809338119093391178
:106AD0001092C80C1092C70C80E090E00E946A747B
:106AE00068E978E081E892E10E94565640912102DF
:106AF00050912202609123027091240222E0CE0183
:106B000001960E94CA56BE016F5F7F4FC7010E9467
:106B1000215760ED75E06FC06AED78E0C7010E9413
:106B20002957B70189E992E10E94F187811117C0C5
:106B300060EE78E0CE0101960E942957BE016F5F9A
:106B40007F4F89E992E10E94F187DD24D39481117E
:106B500001C0D12CCE0101960E94C55602C0DD2491
:106B6000D394C7010E94C556DD2009F457C0809117
:106B70001B11082E000C990B0197039708F047C0D2
:106B800089E390E00E942477BC01990F880B990B50
:106B90000E942EB12AE137E64CE950E40E948DB103
:106BA00060931C1170931D1180931E1190931F11FF
:106BB0001092C80C1092C70C80E090E00E946A749A
:106BC00067E778E081E892E10E94565640911C11F7
:106BD00050911D1160911E1170911F1122E0CE0184
:106BE00001960E94CA56BE016F5F7F4FC7010E9487
:106BF000215766EE78E0C7010E942E56BC0181E85D
:106C000092E10E94DC55C7010E94C5567AC161E538
:106C100078E081E892E10E945656A9C369EE78E0D7
:106C2000C7010E942957B70189E992E10E94F187C3
:106C3000811117C06DEE78E0CE0101960E942957B0
:106C4000BE016F5F7F4F89E992E10E94F187DD24E9
:106C5000D394811101C0D12CCE0101960E94C5565A
:106C600002C0DD24D394C7010E94C556DD2009F47B
:106C70004BC126E030E044E050E069E972E1CE012A
:106C800001960E943D57BE016F5F7F4F8BE792E1F7
:106C90000E94E255CE0101960E94C5568BE792E113
:106CA0000E9410552B013C011B0169E67BE0CE01DF
:106CB00001960E942957BE016F5F7F4F89E992E1DB
:106CC0000E94A187AC014F5F5F4F69E972E1C70184
:106CD0000E94EC41B7018BE792E10E94E255C701A7
:106CE0000E94C556CE0101960E94C55610915B02C6
:106CF0008BE792E10E9405554B015C0180911F14C6
:106D00008823B9F06AE677E081E79FE00E94955713
:106D10004AE050E0B20181E79FE00E94165866E623
:106D20007CE081E79FE00E946058C501B4010E94A9
:106D3000E55C612FC7010E94557EF886EF821D82B7
:106D40001E82198289E08A8381E08B838C831C8A6E
:106D50001B8ACE0101960E94325FCE0101960E94ED
:106D6000C25ECE0101960E94EB5D0E8110E00B30F9
:106D7000110514F00AE010E0BBE54B16510408F4CD
:106D80004CC02FE9A22E2CE0B22E3501212C312C43
:106D90002101E12CF12CE016F106BCF46E2DCE01A0
:106DA00001960E947C5D9B01AC01F301619371939C
:106DB000819391933F01C201B1010E94B8B21B01BE
:106DC0002C01FFEFEF1AFF0AE6CFB801012E000CED
:106DD000880B990B0E942EB19B01AC01C201B1013D
:106DE0000E947EB32B013C01E12CF12CE016F10650
:106DF0000CF05AC0D5012D913D914D915C91C3018C
:106E0000B2010E94B7B2F50161937193819391939E
:106E10005F01FFEFEF1AFF0AE9CF1214130424F504
:106E20000215130524F041E0441A510804C028015A
:106E300081E0481A5108642DCE0101960E947C5DC4
:106E40009B01AC018201000F111F000F111F0156A1
:106E5000134FC501B4010E94B7B2D8016D937D9361
:106E60008D939C93139720C02328F1F48FE9682E0B
:106E70008CE0782EE12CF12CE016F106ACF46E2DAE
:106E8000CE0101960E947C5D9B01AC01C501B4015D
:106E90000E94B7B2F30161937193819391933F0183
:106EA000FFEFEF1AFF0AE8CFEFE9FCE0AAE3B1E158
:106EB00041915191619171914D935D936D937D934A
:106EC0004CE0E73CF407A1F71092C80C1092C70CF5
:106ED00080E090E00E946A7460E378E081E892E1EB
:106EE0000E94565644E050E069E972E1CE010196F5
:106EF0000E94EC41BE016F5F7F4F81E892E10E94EA
:106F0000DC55CE01019631C261EF78E0C7010E94E5
:106F10002957B70189E992E10E94F187811117C0D1
:106F200068EF78E0CE0101960E942957BE016F5F9D
:106F30007F4F89E992E10E94F187DD24D39481118A
:106F400001C0D12CCE0101960E94C55602C0DD249D
:106F5000D394C7010E94C556DD2009F418C127E06B
:106F600030E046E050E069E972E1CE0101960E940E
:106F70003D57BE016F5F7F4F8BE792E10E94E25564
:106F8000CE0101960E94C5568BE792E10E941055F2
:106F90008B0160931B1189E992E10E941B5566E603
:106FA0007CE0CE0101960E942957BE016F5F7F4FA2
:106FB00089E992E10E94A187AC014F5F5F4F69E9C7
:106FC00072E1C7010E94EC41C7010E940555609320
:106FD0001C1170931D1180931E1190931F11C701F6
:106FE0000E94C556CE0101960E94C5566FE178E019
:106FF00081E892E10E9456560430110594F4023063
:1070000011050CF058C001151105B1F00130110542
:1070100009F095C061E178E081E892E10E948C5529
:1070200071C00430110509F08AC06EEF77E081E885
:1070300092E10E948C55A2C020E030E0A90160914D
:107040001C1170911D1180911E1190911F110E94B1
:1070500028B1181664F080E090E0A0E8BFE38093C8
:107060001C1190931D11A0931E11B0931F1120911C
:107070001C1130911D1140911E1150911F1160E0A3
:1070800070E080EA90E40E947EB3AB01BC0122E094
:10709000C7010E94CA566FEF78E0CE0101960E94A8
:1070A0002957B701CE0101960E94455668E679E05E
:1070B0000E942E5657C065E078E081E892E10E9478
:1070C0008C558AE0809FB001819F700D1124CE0104
:1070D00001960E945A5BBE016F5F7F4FC7010E94FD
:1070E000215761E679E0C7010E942E56BC0181E874
:1070F00092E10E94DC55C7010E94C556CE0101965F
:107100000E94C55620E030E048E453E460911C1131
:1071100070911D1180911E1190911F110E9428B134
:10712000181664F180E090E4ACE1B5E480931C11A2
:1071300090931D11A0931E11B0931F111FC0609159
:107140001B11062E000C770BC7010E945A5B6AE0E8
:1071500079E0CE0101960E942957B701CE01019630
:107160000E944556BC0181E892E10E94DC55CE01A7
:1071700001960E94C556C7010E94C5561092C80CC0
:107180001092C70C80E090E00E946A74F0C061E148
:1071900079E0C7010E942957B70189E992E10E946D
:1071A000F187811117C068E179E0CE0101960E9454
:1071B0002957BE016F5F7F4F89E992E10E94F187F5
:1071C000DD24D394811101C0D12CCE0101960E94FF
:1071D000C55602C0DD24D394C7010E94C556DD20E8
:1071E00009F4D6C027E030E046E050E069E972E1FA
:1071F000CE0101960E943D57BE016F5F7F4F8BE726
:1072000092E10E94E255CE0101960E94C5568BE79D
:1072100092E10E9410556093181189E992E10E9451
:107220001B558BE792E10E94105561157105810590
:10723000910519F485E090E007C061307105810582
:10724000910539F489E190E090931A118093191116
:1072500023C066E67CE0CE0101960E942957BE015C
:107260006F5F7F4F89E992E10E94A187AC014F5F78
:107270005F4F69E972E1C7010E94EC41C7010E94BA
:10728000105570931A1160931911C7010E94C556C9
:10729000CE0101960E94C5561092C80C1092C70CE0
:1072A00080E090E00E946A746DEE77E081E892E100
:1072B0000E9456568091181183302CF562EE77E0CB
:1072C00081E892E10E948C556091191170911A1118
:1072D000CE0101960E945A5BBE016F5F7F4FC701CE
:1072E0000E94215767E47CE0C7010E942E56BC0132
:1072F00081E892E10E94DC55C7010E94C556CE018B
:1073000001960E94C55680911811833084F16091D6
:10731000191170911A11CE0183960E945A5B6091E7
:107320001811062E000C770BC7010E945A5B6AE009
:1073300079E0CE0101960E942957B701CE0101964E
:107340000E944556BE016D5D7F4F0E944556BC01AF
:1073500081E892E10E94DC55CE0101960E94C5565B
:10736000C7010E94C556CE0183960E94C55661E8AA
:1073700072E1CE0101960E942157CE0101960E9432
:10738000586ACE0101960E94C5561092540204C25A
:107390006FE179E0C7010E942957B70189E992E1BD
:1073A0000E94F187811117C063E279E0CE01019656
:1073B0000E942957BE016F5F7F4F89E992E10E94C9
:1073C000F187DD24D394811101C0D12CCE01019627
:1073D0000E94C55602C0DD24D394C7010E94C55641
:1073E000DD2009F455C08091590290915A020E9403
:1073F0001C7860932B0270932C0280932D02909343
:107400002E026093041170930511809306119093DE
:10741000071180E090E5A3ECB7E4809333029093EA
:107420003402A0933502B09336028093FC109093FF
:10743000FD10A093FE10B093FF1080911F148823BD
:1074400081F064EC77E081E79FE00E9495576091BE
:107450002B0270912C0280912D0290912E020E949D
:10746000E55C1092C80C1092C70C80E090E00E947E
:107470006A7440912B0250912C0260912D02709100
:107480002E0222E0C7010E94CA5667E279E064C179
:1074900062E379E0C7010E942957B70189E992E1C7
:1074A0000E94F187811117C066E379E0CE01019651
:1074B0000E942957BE016F5F7F4F89E992E10E94C8
:1074C000F187DD24D394811101C0D12CCE01019626
:1074D0000E94C55602C0DD24D394C7010E94C55640
:1074E000DD2009F484C080919D1290919E12049732
:1074F000F0F044E050E069E972E1CE0101966CD70A
:10750000BE016F5F7F4F8BE792E10E94E255CE0193
:1075100001960E94C5568BE792E10E940555609343
:107520003702709338028093390290933A02809127
:10753000370290913802A0913902B0913A028093BB
:10754000F8109093F910A093FA10B093FB1080916B
:107550001F14882389F06BEA77E081E79FE00E949F
:10756000955760913702709138028091390290915D
:107570003A0242E00E94D9708091590290915A02D9
:107580000E941C7860932F02709330028093310226
:107590009093320260930011709301118093021155
:1075A0009093031180911F14882381F061EA77E0A2
:1075B00081E79FE00E94955760912F027091300201
:1075C00080913102909132020E94E55C1092C80CC9
:1075D0001092C70C80E090E00E946A7440912F02E4
:1075E000509130026091310270913202AFC062E47A
:1075F00079E0C7010E942957B70189E992E10E9409
:10760000F187811117C066E479E0CE0101960E94EE
:107610002957BE016F5F7F4F89E992E10E94F18790
:10762000DD24D394811101C0D12CCE0101960E949A
:10763000C55602C0DD24D394C7010E94C556DD2083
:1076400011F40C94303180919D1290919E12049708
:10765000F0F044E050E069E972E1CE010196BCD659
:10766000BE016F5F7F4F8BE792E10E94E255CE0132
:1076700001960E94C5568BE792E10E9405556093E2
:1076800033027093340280933502909336028091D6
:10769000330290913402A0913502B091360280936A
:1076A000FC109093FD10A093FE10B093FF108091FA
:1076B0001F14882389F068E877E081E79FE00E9443
:1076C0009557609133027091340280913502909108
:1076D000360242E00E94D9708091590290915A027C
:1076E0000E941C7860932B0270932C0280932D02D1
:1076F00090932E02609304117093051180930611EC
:107700009093071180911F14882381F06EE777E032
:1077100081E79FE00E94955760912B0270912C02A7
:1077200080912D0290912E020E94E55C1092C80C6F
:107730001092C70C80E090E00E946A7440912B0286
:1077400050912C0260912D0270912E0222E0C7010F
:107750000E94CA566AE379E0CE0101960E94295739
:10776000B701CE0101960E944556BC0181E892E125
:107770000E94B056CE0101960E94C556C701F5CDB4
:10778000CE0183960E94C5560C941E33CE0183967B
:107790000E94C5560C94A1338D2DA8960FB6F8946F
:1077A000DEBF0FBECDBFDF91CF911F910F91FF9034
:1077B000EF90DF90BF90AF909F908F907F906F90F1
:1077C0005F904F903F902F9008954F925F926F92ED
:1077D0007F929F92AF92BF92CF92DF92EF92FF92F1
:1077E0000F931F93CF93DF93CDB7DEB7A9970FB653
:1077F000F894DEBF0FBECDBF982E882351F0809144
:107800001F14882331F064E67AE081E79FE00E944C
:1078100095700E94285B60E08DE20E94855C60E1CB
:107820008DE20E94855C68E08DE20E94855C40905C
:10783000E5125090E6126090E7127090E812498EBF
:107840005A8E6B8E7C8EC090E912D090EA12E09036
:10785000EB12F090EC12CD8EDE8EEF8EF8A28091BE
:10786000ED129091EE12A091EF12B091F0128EA352
:107870009FA3A8A7B9A789A39AA3ABA3BCA3992048
:10788000C9F180911F148823A9F162EC7CE0CE013C
:1078900001960E941957CE0101960E946592CE0171
:1078A00001960E94C5568E01075E1F4F5E0195E24C
:1078B000A90EB11CD8016D917D918D919D918D0185
:1078C00046E00E94D97066E67CE081E79FE00E9476
:1078D0006058A016B10671F764E67AE0CE01019611
:1078E0000E942957CE0101960E946592CE01019611
:1078F0000E94C55623E938E144E85FE3C301B201C1
:107900000E948DB12B013C016D877E878F87988BFC
:1079100022E430E645E85FE3C701B6010E948DB17D
:107920006B017C01698B7A8B8B8B9C8B25E83BEE02
:1079300041E95FE36EA17FA188A599A50E948DB161
:107940006D8B7E8B8F8B988F4092E5125092E61252
:107950006092E7127092E812C092E912D092EA1295
:10796000E092EB12F092EC126093ED127093EE1233
:107970008093EF129093F012992009F4A0C08091A7
:107980001F14882309F49BC065EB7CE0CE010196AF
:107990000E941957CE0101960E946592CE01019670
:1079A0000E94C5568E01035F1F4F6E01B9E1CB0ED9
:1079B000D11C7801F80161917191819191918F01B0
:1079C00042E00E94D97066E67CE081E79FE00E9479
:1079D0006058C016D10671F764E67AE0CE010196D0
:1079E0000E942957CE0101960E946592CE01019610
:1079F0000E94C55641EF52E166E070E082E30E94CA
:107A00001E5CA090F112B090F212C090F312D090D0
:107A1000F4120091F5121091F61268EA7CE081E709
:107A20009FE00E9495574AE050E0B50181E79FE052
:107A30000E94165866E67CE081E79FE00E9460584D
:107A40004AE050E0B60181E79FE00E94165866E6E2
:107A50007CE081E79FE00E9460584AE050E0B80176
:107A600081E79FE00E94165864E67AE081E79FE094
:107A70000E949570CE0101960E94F45C6FE97CE053
:107A800081E79FE00E9495578E010F5F1F4FD8013D
:107A90006D917D918D919D918D014AE00E94D970EB
:107AA00066E67CE081E79FE00E9460580E151F05A6
:107AB00071F764E67AE081E79FE00E94957061E0EB
:107AC0008DE10E94855C9920B1F080911F1488237C
:107AD00091F06BE87CE081E79FE00E949557AE0152
:107AE0004B5D5F4F61E070E08DE10E941E5C8DA1F7
:107AF00090E00E94595C62E08EE10E94855C63E048
:107B00008FE10E94855C64E080E20E94855C9920A0
:107B100009F450C080911F14882309F44BC06FE60C
:107B20007CE081E79FE00E949557AE014B5D5F4F7F
:107B300061E070E08EE10E941E5CCDA0D12CAE0110
:107B40004B5D5F4F61E070E08FE10E941E5CEDA035
:107B5000F12CAE014B5D5F4F61E070E080E20E946E
:107B60001E5C0DA110E04AE050E0B60181E79FE005
:107B70000E94165866E67CE081E79FE00E9460580C
:107B80004AE050E0B70181E79FE00E94165866E6A0
:107B90007CE081E79FE00E9460584AE050E0B80135
:107BA00081E79FE00E94165864E67AE081E79FE053
:107BB0000E94957065E081E20E94855C9920B1F099
:107BC00080911F14882391F06CE57CE081E79FE0B1
:107BD0000E949557AE014B5D5F4F61E070E081E21E
:107BE0000E941E5C8DA190E00E94595C66E082E2DA
:107BF0000E94855C9920B1F080911F14882391F038
:107C000064E47CE081E79FE00E949557AE014B5D04
:107C10005F4F61E070E082E20E941E5C8DA190E007
:107C20000E94595C67E083E20E94855C9920B1F074
:107C300080911F14882391F06EE27CE081E79FE041
:107C40000E949557AE014B5D5F4F61E070E083E2AB
:107C50000E941E5C8DA190E00E94595C68E084E265
:107C60000E94855C9920B1F080911F14882391F0C7
:107C700066E17CE081E79FE00E949557AE014B5D95
:107C80005F4F61E070E084E20E941E5C8DA190E095
:107C90000E94595C69E085E20E94855C9920B1F000
:107CA00080911F14882391F06CEF7BE081E79FE0C7
:107CB0000E949557AE014B5D5F4F61E070E085E239
:107CC0000E941E5C8DA190E00E94595C6AE086E2F1
:107CD0000E94855C9920B1F080911F14882391F057
:107CE00066EE7BE081E79FE00E949557AE014B5D19
:107CF0005F4F61E070E086E20E941E5C8DA190E023
:107D00000E94595C6BE088E20E94855C9920B1F08A
:107D100080911F14882391F06DEC7BE081E79FE058
:107D20000E949557AE014B5D5F4F61E070E088E2C5
:107D30000E941E5C8DA190E00E94595C6CE089E27B
:107D40000E94855C992009F479C080911F148823D2
:107D500009F474C065EB7BE081E79FE00E949557D2
:107D6000AE014B5D5F4F61E070E089E20E941E5CF6
:107D70008DA190E00E94595C6EE97BE081E79FE075
:107D80000E94955766E070E087E20E946B5C90E08D
:107D90000E94595C67E87BE081E79FE00E9495576D
:107DA00065E070E087E20E946B5C90E00E94595CA5
:107DB00060E77BE081E79FE00E94955764E070E018
:107DC00087E20E946B5C90E00E94595C67E57BE073
:107DD00081E79FE00E94955762E070E087E20E9491
:107DE0006B5C90E00E94595C6EE37BE081E79FE072
:107DF0000E94955761E070E087E20E946B5C90E022
:107E00000E94595C65E27BE081E79FE00E94955704
:107E100060E070E087E20E946B5C90E00E94595C39
:107E200064E17BE081E79FE00E94955763E070E0AA
:107E300087E20E946B5C90E00E94595C41E067E041
:107E400070E087E20E949A5C41E063E070E087E2C4
:107E50000E949A5C41E063E070E08AE20E949A5CD2
:107E6000992091F080911F14882371F06BEF7AE0D4
:107E700081E79FE00E94955763E070E08AE20E94EC
:107E80006B5C90E00E94595C40E063E070E08AE245
:107E90000E949A5C992091F080911F14882371F0C0
:107EA00061EE7AE081E79FE00E94955763E070E021
:107EB0008AE20E946B5C90E00E94595C41E062E0C3
:107EC00070E08AE20E949A5C992091F080911F14E0
:107ED000882371F065EC7AE081E79FE00E94955776
:107EE00062E070E08AE20E946B5C90E00E94595C64
:107EF00040E062E070E08AE20E949A5C992091F092
:107F000080911F14882371F068EA7AE081E79FE08E
:107F10000E94955762E070E08AE20E946B5C90E0FC
:107F20000E94595C41E061E070E08AE20E949A5C44
:107F3000992091F080911F14882371F06CE87AE009
:107F400081E79FE00E94955761E070E08AE20E941D
:107F50006B5C90E00E94595C40E061E070E08AE276
:107F60000E949A5C992091F080911F14882371F0EF
:107F70006FE67AE081E79FE00E94955761E070E04C
:107F80008AE20E946B5C90E00E94595C41E060E0F4
:107F900070E08AE20E949A5C992091F080911F140F
:107FA000882371F063E57AE081E79FE00E949557AE
:107FB00060E070E08AE20E946B5C90E00E94595C95
:107FC00040E060E070E08AE20E949A5C992091F0C3
:107FD00080911F14882371F066E37AE081E79FE0C7
:107FE0000E94955760E070E08AE20E946B5C90E02E
:107FF0000E94595C41E066E070E087E20E949A5C72
:1080000041E065E070E087E20E949A5C41E064E054
:1080100070E087E20E949A5C40E062E070E087E2F4
:108020000E949A5C40E061E070E087E20E949A5C06
:1080300040E060E070E087E20E949A5C992009F4D9
:1080400075C080911F14882309F470C06EE17AE036
:1080500081E79FE00E94955766E070E08BE20E9406
:108060006B5C90E00E94595C60E07AE081E79FE001
:108070000E94955765E070E08BE20E946B5C90E097
:108080000E94595C62EE79E081E79FE00E9495577B
:1080900064E070E08BE20E946B5C90E00E94595CAF
:1080A00069EC79E081E79FE00E94955762E070E01B
:1080B0008BE20E946B5C90E00E94595C60EB79E07F
:1080C00081E79FE00E94955761E070E08BE20E949B
:1080D0006B5C90E00E94595C67E979E081E79FE082
:1080E0000E94955760E070E08BE20E946B5C90E02C
:1080F0000E94595C64E879E081E79FE00E9495570F
:1081000063E070E08BE20E946B5C90E00E94595C3F
:108110006FE679E081E79FE00E94955764E070E0A8
:108120008CE20E946B5C90E00E94595C40E064E04D
:1081300070E08CE20E949A5CAE014B5D5F4F61E0A3
:1081400070E08CE20E941E5C6DA1607F66608CE234
:108150000E94855C992009F45FC080911F148823D8
:1081600009F45AC06BE579E081E79FE00E949557DA
:10817000AE014B5D5F4F61E070E08CE20E941E5CDF
:108180006DA16F7070E066507109072E000C880BAE
:10819000990B0E942EB19B01AC0160E070E080E081
:1081A00090E40E9426B520E030E048EC50E40E94C4
:1081B0008DB10E94E55C64E479E081E79FE00E9474
:1081C0009557AE014B5D5F4F61E070E080E30E9428
:1081D0001E5C6DA14AE050E081E79FE00E94CA5C0E
:1081E0006CE279E081E79FE00E94955761E070E0E2
:1081F00080E30E946B5C90E00E94595C63E179E04F
:1082000081E79FE00E94955761E070E08FE20E9455
:108210006B5C90E00E94595C41E061E070E08FE2AD
:108220000E949A5C992091F080911F14882371F02C
:108230006BEF78E081E79FE00E94955761E070E086
:108240008EE20E946B5C90E00E94595C41E061E02C
:1082500070E08EE20E949A5C40E067E070E081E3AB
:108260000E949A5C992009F455C080911F148823BC
:1082700009F450C068EE78E081E79FE00E949557CE
:1082800067E070E081E30E946B5C90E00E94595CC3
:108290006AE479E081E79FE00E946058AE014B5D9F
:1082A0005F4F61E070E080E00E941E5C8DA10E9443
:1082B000AE7F64E67AE081E79FE00E9495700DE171
:1082C00010E060EA76E081E79FE00E94605840E1BC
:1082D00050E0B80181E79FE00E9416586EE479E013
:1082E00081E79FE00E946058AE014B5D5F4F61E007
:1082F00070E0802F0E941E5C8DA10E94AE7F64E61C
:108300007AE081E79FE00E9495700F5F1F4F0A336C
:108310001105B9F6A9960FB6F894DEBF0FBECDBF12
:10832000DF91CF911F910F91FF90EF90DF90CF9051
:10833000BF90AF909F907F906F905F904F90089507
:10834000089580912E058823F9F080912D058823CA
:10835000D9F081E00E942C708BE39FE10197F1F747
:1083600060E080E00E943D706CE97DE08CE793E185
:108370000E94955761E080E00E943D706CE87DE0CE
:108380008CE793E10C949557089580912E058823EE
:1083900049F080912D05882329F060E08CE793E176
:1083A0000C94A97E0895FF920F931F93CF93DF93B0
:1083B000EC01F62E08811981C8010E9444B2F8161A
:1083C00021F06F2DC8010E944CB2CE01DF91CF91F8
:1083D0001F910F91FF900895CF93DF93EC01FB0164
:1083E000248135810E943D57CE01DF91CF910895C0
:1083F0003F924F925F926F927F928F929F92AF9235
:10840000BF92CF92DF92EF92FF920F931F93CF9381
:10841000DF93CDB7DEB7E4970FB6F894DEBF0FBE9B
:10842000CDBF8091CC13882319F01092CC134CC38C
:1084300081E08093CC1364E67AE0CE0185960E94B9
:10844000295764E67AE0CE018B960E94295700E016
:1084500010E082E0382E98EEC92E93E0D92EE12C60
:10846000F12CF8013197E031F10530F48827E85616
:10847000FF4F8F4F0C9406B664E67AE0CE018596E6
:108480000E949B568091621190916311892B31F467
:108490006CE077E0CE0185960E949B568091621138
:1084A00090916311019731F460E177E0CE018596F8
:1084B0000E949B568091621190916311029731F452
:1084C00066E177E0CE0185960E949B5689A59AA524
:1084D000892B31F060E773E1CE0185960E94DC556F
:1084E00061E579E0CE0101960E9429576AE673E1C1
:1084F000CE0101960E944556BC01CE018B960E948A
:10850000B056CE0101960E94C5568091621190919D
:108510006311019709F03BC2BE016B5D7F4FCE0135
:1085200001960E94215748EC50E06FEF7FEFCE019B
:1085300001960E949192CE0101960E94C556BE01FD
:10854000655D7F4FCE0101960E94215740ED57E0B7
:108550006FEF7FEFCE0101960E944990CE01019608
:108560000E94C556CE0101960E94C1508D819E8108
:108570000097A1F0E981FA812081222379F0079701
:1085800068F065E77FE0CE0185960E945656BE01F1
:108590006F5F7F4FCE018B960E94B056CE01019641
:1085A00096C069E67FE0CE0185960E9456560E94ED
:1085B0005D8A4B015C010E945D8AA70196010E94C1
:1085C00086B2CA01B90120E831E541E050E00E94DD
:1085D00086B220E13EE040E050E00E945AB229AB72
:1085E0003AAB4BAB5CAB2CE330E040E050E00E9498
:1085F0005AB229013A01AB01BC01CE0101960E9499
:108600006870B301A201CE0107960E94687049A963
:108610005AA96BA97CA9CE010D960E946870C5016C
:10862000B40120E03CE546E255E00E9486B2BA0182
:10863000A901CE0149960E946870BE01675E7F4F16
:10864000CE0143960E94215766E579E0CE0143961C
:108650000E942E56BE01635F7F4F0E94455669E51A
:1086600079E00E942E56BE01695F7F4F0E944556F9
:108670006CE579E00E942E56BE016F5F7F4F0E942D
:1086800045566EED75E00E942E56BC01CE014F9608
:108690000E942157CE0143960E94C556CE014996AD
:1086A0000E94C556CE010D960E94C556CE01079672
:1086B0000E94C556CE0101960E94C556BE01615E5C
:1086C0007F4FCE018B960E94E255CE014F960E94BD
:1086D000C5565DC180919D0C90919E0C019719F437
:1086E0006AE57FE002C06CE47FE0CE0185960E94DF
:1086F00056566CE37FE047C16CE27FE0CE01859681
:108700000E9456566FE17FE03EC162E17FE0CE01FC
:1087100085960E94565667E07FE035C16BEF7EE09C
:10872000CE0185960E9456566AEE7EE02CC180915D
:108730009D0C90919E0C039719F46FED7EE002C0A2
:1087400065ED7EE0CE0185960E9456566AEC7EE08D
:108750001AC16DEB7EE0CE0185960E9456566EEAF8
:108760007EE011C163EA7EE0CE0185960E945656F6
:108770006091191170911A11CE0107960E945A5BEF
:108780006FE67CE0CE0101960E942957BE01695F29
:108790007F4FCE0101960E94455667E47CE00E941F
:1087A0002E56BC01CE0185960E94DC55CE01019665
:1087B0000E94C556CE0107960E94C55666E97EE026
:1087C000E2C080919D0C90919E0C029719F465E88F
:1087D0007EE002C065E77EE0CE0185960E94565697
:1087E00068E67EE0D0C06CE57EE0CE0185960E9412
:1087F00056566CE47EE0C7C061E47EE0CE0185960B
:108800000E94565667E37EE0BEC06BE27EE0CE017A
:1088100085960E9456566BE17EE0B5C0B0901B1164
:1088200060E17EE0CE0185960E94565683E08B156E
:1088300074F092E0B9160CF045C0BB2081F081E0E5
:10884000B81261C06FE579E0CE01859659C094E019
:10885000B91259C063E679E081E892E151C0809095
:108860001C1190901D11A0901E11B0901F1120E0BE
:1088700030E048E452E4C501B4010E9428B187FF0A
:1088800002C033243394A501940160E070E080EAD3
:1088900090E40E947EB3AB01BC01232DCE0107966C
:1088A0000E94CA566DE879E0CE0101960E942957D0
:1088B000BE01695F7F4FCE0101960E94455668E672
:1088C00079E018C08B2D9AE08902B0011124CE0105
:1088D00007960E945A5B6FE67CE0CE0101960E94EB
:1088E0002957BE01695F7F4FCE0101960E94455610
:1088F00061E679E00E942E56BC01CE0185961CC02F
:108900000E94CE5523C060911B11062E000C770BE0
:10891000CE0107960E945A5B6CE27BE0CE01019685
:108920000E942957BE01695F7F4FCE0101960E94C8
:108930004556BC0181E892E10E94DC55CE010196CA
:108940000E94C556CE0107960E94C55660E07EE0A3
:108950001AC063EF7DE0CE0185960E94565663EE05
:108960007DE011C067ED7DE0CE0185960E945656F0
:1089700068EC7DE008C06CEB7DE0CE0185960E943E
:1089800056566CEA7DE0CE018B960E945656BE018B
:108990006B5D7F4FCE0101960E94215748EC50E05D
:1089A0006FEF7FEFCE0101960E943693CE010196C4
:1089B0000E94C556BE01655D7F4FCE0101960E94A3
:1089C000215748EC50E06FEF7FEFCE0101960E94F7
:1089D0004990CE0101960E94C5560E94D09A982EC9
:1089E000A12CB12C91106DC08FEFA81AB80A95E692
:1089F000A916B10451F00E94D09A982E64E170E05B
:108A000080E090E00E940189EDCF64E67AE089E998
:108A100092E10E949B56CE0101960E94D26DBE014A
:108A20006F5F7F4F89E992E10E94E255CE01019686
:108A30000E94C55680919D1290919E12892B89F4B7
:108A400061E070E0CE0101960E94058EBE016F5F6D
:108A50007F4F89E992E10E94E255CE0101960E9482
:108A6000C55680919D1290919E12892B89F461E0E8
:108A700070E0CE0101960E94A38CBE016F5F7F4F14
:108A800089E992E10E94E255CE0101960E94C55605
:108A900080919D1290919E12892B51F48091CC135C
:108AA000882331F00F5F1F4F0131110509F0D9CC38
:108AB000CE018B960E94C556CE0185960E94C55662
:108AC00003C01092CC13F4CFE4960FB6F894DEBF37
:108AD0000FBECDBFDF91CF911F910F91FF90EF900F
:108AE000DF90CF90BF90AF909F908F907F906F90CE
:108AF0005F904F903F9008954F925F926F927F9258
:108B00008F929F92AF92BF92CF92DF92EF92FF929D
:108B10000F931F93CF93DF93CDB7DEB7C654D10920
:108B20000FB6F894DEBF0FBECDBF8C0164E67AE0CD
:108B3000CE01C7960E94295764E67AE0CE01CD9611
:108B40000E942957BE016F5F7F4F86EB92E10E9422
:108B50000A548D889E88AF88B88C498C5A8C6B8C4F
:108B60007C8C8D8D9E8DAF8DB8A127968CAF9DAFDF
:108B7000AEAFBFAF2797C8010197039708F0BCC1FC
:108B8000A3019201C501B40190580E942BB32BEDB3
:108B90003FE049EC5FE30E94B8B220913F02309180
:108BA000400240914102509142020E94B8B26B01D2
:108BB0007C0120E030E0A9010E9428B187FD09C0B6
:108BC000C092DC0CD092DD0CE092DE0CF092DF0C57
:108BD00010C02BED3FE049EC50E4C701B6010E9404
:108BE000B8B26093DC0C7093DD0C8093DE0C909334
:108BF000DF0CC090DC0CD090DD0CE090DE0CF0902F
:108C0000DF0C2BED3FE049EC50E4C701B6010E94B8
:108C10006DB4181684F42BED3FE049EC50E4C70125
:108C2000B6010E94B7B26093DC0C7093DD0C8093A8
:108C3000DE0C9093DF0C20E030E044E353E46091DD
:108C4000DC0C7091DD0C8091DE0C9091DF0C0E94A9
:108C50008DB12BED3FE049E450E40E947EB3609378
:108C6000D80C7093D90C8093DA0C9093DB0C0E9493
:108C700017B4CE018B960E945A5B6BE679E0CE0169
:108C800085960E942957BE01655D7F4FCE0185966E
:108C90000E94455665E779E00E942E56BC0187E8A0
:108CA00092E10E94B056CE0185960E94C556CE0133
:108CB0008B960E94C556C090D80CD090D90CE090ED
:108CC000DA0CF090DB0C20E030E044EB52E4C7011A
:108CD000B6010E9428B118168CF020E030E040E088
:108CE0005FE3C701B6010E94B8B20E9417B4CE017B
:108CF0008B960E945A5B6CE779E022C020E030E05E
:108D000044E353E4C701B6010E9428B118169CF150
:108D1000A701960160E070E884E393E40E94B7B293
:108D20006093D80C7093D90C8093DA0C9093DB0C81
:108D30000E9417B4CE018B960E945A5B6FE779E0D0
:108D4000CE0185960E942957BE01655D7F4FCE01F9
:108D500085960E944556BC01CE01C7960E94B0562A
:108D6000CE0185960E94C556CE018B960E94C556AF
:108D70006FEB7BE061C020E030E047E853E4C701DF
:108D8000B6010E9428B11816FCF020E030E044E360
:108D900053E4C701B6010E94B7B220E030E040E0E2
:108DA0005FE30E94B8B26093D80C7093D90C8093A3
:108DB000DA0C9093DB0C0E9417B4CE018B960E94C4
:108DC0005A5B6FE779E01EC0A701960160E070E092
:108DD00084EB93E40E94B7B220E030E040E05FE330
:108DE0000E94B8B26093D80C7093D90C8093DA0CBF
:108DF0009093DB0C0E9417B4CE018B960E945A5BB5
:108E00006CE779E0CE0185960E942957BE01655D29
:108E10007F4FCE0185960E944556BC01CE01C79674
:108E20000E94B056CE0185960E94C556CE018B9603
:108E30000E94C55662E879E0CE01CD960E949B560D
:108E4000BE01695C7F4FCE0185960E9421574AE0A2
:108E500050E060E070E0CE0185960E949192CE01D4
:108E600085960E94C5560E945D8AC0901B14D090C2
:108E70001C14E0901D14F0901E14A4E6CA0ED11C20
:108E8000E11CF11CC616D706E806F90608F424C250
:108E90000E945D8A0E942CB16B017C0160911B14C1
:108EA00070911C1480911D1490911E140E942EB17B
:108EB00020E030E048EC51E40E94B8B29B01AC01E4
:108EC000C701B6010E9428B187FD06C266E67CE0B4
:108ED000CE0185960E942957BE01635C7F4FCE016B
:108EE00085960E944556BC01CE01C7960E94DC556E
:108EF000CE0185960E94C556C8010297029708F0D8
:108F0000C5C120E030E040E251E4C501B4010E9457
:108F10008DB16B017C0120E030E040E251E4C301FF
:108F2000B2010E948DB14B015C0120E030E040E2D3
:108F300051E427966CAD7DAD8EAD9FAD27970E9415
:108F40008DB12B013C010E945D8A2091780C3091FB
:108F5000790C40917A0C50917B0C621B730B840B43
:108F6000950B0E942CB120E030E04AE754E40E94C7
:108F70007EB3AB01BC0123E0CE018B960E94CA56A2
:108F80006DE879E0CE0185960E942957BE01655DA6
:108F90007F4FCE0185960E94455663E97BE00E9493
:108FA0002E56BC0185E792E10E94B056CE0185960F
:108FB0000E94C556CE018B960E94C55665E772E1A8
:108FC000CE0185960E94215767E872E1CE01859611
:108FD0000E944556BE01695C7F4F0E944556BC0108
:108FE000CE01C7960E94B056CE0185960E94C55606
:108FF00061E87DE081E892E10E94565621E0B701E8
:10900000A601CE0185960E94CA56BE016B5D7F4FB8
:1090100081E892E10E94DC55CE0185960E94C556FA
:1090200021E0B301A201CE01C1960E94CA5621E0FF
:10903000B501A401CE018B960E94CA5666E67CE07B
:10904000CE0185960E942957BE01655D7F4FCE01F6
:1090500085960E94455666E67CE00E942E56BE012B
:109060006F5C7F4F0E94455664E879E00E942E565F
:10907000BC0181E892E10E94DC55CE0185960E94F8
:10908000C556CE018B960E94C556CE01C1960E9450
:10909000C556A7019601C701B6010E948DB16B01AB
:1090A0007C01A5019401C501B4010E948DB19B0111
:1090B000AC01C701B6010E94B8B26B017C01A301EB
:1090C0009201C301B2010E948DB19B01AC01C701A5
:1090D000B6010E94B8B20E9476B56B017C01609324
:1090E000D40C7093D50C8093D60C9093D70C68E871
:1090F00079E081E892E10E94CE5521E0B701A60116
:10910000CE0185960E94CA56BE016B5D7F4FCE018F
:109110008B960E94215769E979E0CE018B960E94D7
:109120002E56BC0187E892E10E94B056CE018B9684
:109130000E94C556CE0185960E94C55667E872E129
:1091400081E892E10E94DC55C090D40CD090D50CFF
:10915000E090D60CF090D70C20E030E04AE754E4E1
:10916000C701B6010E946DB487FD29C020E030E040
:109170004AE754E4C701B6010E947EB3AB01BC01CB
:1091800023E0CE0185960E94CA56BE016B5D7F4FDB
:10919000CE018B960E9421576AE979E0CE018B9629
:1091A0000E942E56BC0187E892E10E94B056CE0183
:1091B0008B960E94C556CE0185960E94C55620E02A
:1091C00030E64AE656E46091D40C7091D50C80915B
:1091D000D60C9091D70C0E9428B1BE01695C7F4FDC
:1091E00087FF50C0CE0185960E9421576CE879E038
:1091F000CE0185960E942E5661E872E10E94455686
:10920000BC0181E892E10E94B056CE0185960E9491
:10921000C55603301105A1F461E872E1CE018596CF
:109220000E942157CE0185960E94586ACE018596EC
:109230000E94C55664E67AE081E892E10E949B565E
:109240006FE879E0CE0185960E94295767E872E1C0
:10925000CE0185960E944556BC01CE018B960E9498
:1092600021574AE050E06FEF7FEFCE018B960E94CE
:109270004990CE018B960E94C556CE0185960E94DC
:10928000C55604C081E892E10E94B0566AE070E0E1
:1092900080E090E00E940189CE01CD960E94C556E3
:1092A000CE01C7960E94C556CA5BDF4F0FB6F89431
:1092B000DEBF0FBECDBFDF91CF911F910F91FF9009
:1092C000EF90DF90CF90BF90AF909F908F907F9066
:1092D0006F905F904F90089564E67AE0CE01859696
:1092E0000E942957CE0185960E94C590CE01859691
:1092F0000E94C556BE01635C7F4F8CE793E10E94DC
:109300008757E4CD1F93CF93DF93CDB7DEB7A897F0
:109310000FB6F894DEBF0FBECDBF182F0E94285B9A
:109320008EE10E94227062E08EE090E10E94657DF5
:1093300060E08EE090E10E94657D0E941B708EE1EE
:109340000E94227061E08EE090E10E94657D60E203
:109350008EE090E10E94657D0E941B7080E290E0AB
:109360009093BA128093B91280E090E8A9E8B4E42F
:109370008093670290936802A0936902B0936A0297
:1093800080E090E0A5E7B4E48093630290936402E8
:10939000A0936502B0936602BE016F5F7F4F86EBBC
:1093A00092E10E94BD53112309F484C066E57DE07B
:1093B00081E79FE00E94955781E79FE00E94AA6F96
:1093C00066E47DE081E79FE00E949557BE016F5FF4
:1093D0007F4F81E79FE00E94957066E37DE081E723
:1093E0009FE00E9495576D857E858F8598890E94A4
:1093F000A67066E27DE081E79FE00E94955769894B
:109400007A898B899C890E94A67066E17DE081E75C
:109410009FE00E94955720E030E040E251E4698DE2
:109420007A8D8B8D9C8D0E948DB142E00E94D97007
:1094300068E979E081E79FE00E94957066E07DE051
:1094400081E79FE00E94955720E030E040E251E440
:109450006D8D7E8D8F8D98A10E948DB142E00E940E
:10946000D97068E979E081E79FE00E94957066EF26
:109470007CE081E79FE00E94955720E030E040E2E9
:1094800051E469A17AA18BA19CA10E948DB142E017
:109490000E94D97068E979E081E79FE00E949570A9
:1094A00060ED7CE081E79FE00E94955781E79FE0B7
:1094B0000E94AA6F64EF71E080E090E00E94018951
:1094C000A8960FB6F894DEBF0FBECDBFDF91CF9147
:1094D0001F9108950F931F9360E0809102020E94F4
:1094E0004D8883E090E00197F1F761E080910202FE
:1094F0000E944D8883E290E00197F1F760E080914F
:1095000002020E944D8880910002909101029927E9
:10951000FC01E05BFC4E6491FC01E65FFC4EE491D3
:10952000F0E0EE0FFF1FE051FD4E8591949100E4B5
:1095300012E42FE030E0462F0E94DD9C611571059A
:109540008105910549F0DC01CB010196A11DB11DFA
:10955000BC01CD019F7003C060E070E0CB010E94B0
:109560002CB120E030E048EC52E40E947EB3209120
:10957000E00C3091E10C4091E20C5091E30C0E9420
:109580008DB120E030E44CE156E40E947EB320E04F
:1095900030E040E05FE30E948DB11F910F9108958C
:1095A00023E333E948E853E40E947EB320E030E04F
:1095B00040E85FE30E94B8B20E9476B526E636EA3C
:1095C00045EA53E40E948DB16093E00C7093E10C86
:1095D0008093E20C9093E30C0895CF92DF92EF9288
:1095E000FF9278DF6B017C0120E030E040E050E446
:1095F0000E946DB418161CF46DDF6B017C0120E035
:1096000030E040E050E4C701B6010E946DB4181686
:109610001CF460DF6B017C0120E030E040E050E4AE
:10962000C701B6010E946DB418161CF453DF6B011C
:109630007C0120E030E040E050E4C701B6010E9428
:109640006DB418162CF4FF90EF90DF90CF9042CFBE
:10965000C701B601FF90EF90DF90CF900895BF92C1
:10966000CF92DF92EF92FF920F931F93CF93DF93EE
:10967000CDB7DEB762970FB6F894DEBF0FBECDBF91
:109680008C016B0166E67CE0CE010D960E942957A5
:1096900067E170E1C8010E94195776012FEFE21AC5
:1096A000F20AB701CE0101960E945A5BBE016F5FBC
:1096B0007F4FCE0107960E94215769E177E0CE01E6
:1096C00007960E942E56BC01C8010E94DC55CE01AF
:1096D00007960E94C556CE0101960E94C5568AE0A3
:1096E000B82EBE9CC001BF9C900D1124FC01E55812
:1096F000FE4E7F018081082E000C990B0E945DB800
:10970000892B09F4B2C0B701CE0101960E942957F6
:10971000BE016F5F7F4FCE0107960E9421576EE812
:109720007BE0CE0107960E942E56BC01C8010E9424
:10973000DC55CE0107960E94C556CE0101960E94C7
:10974000C556BC9CC001BD9C900D11249C012558A0
:109750003E4E7901F9016685062E000C770BCE018D
:1097600001960E945A5BBE016F5F7F4FCE01079644
:109770000E9421576CE979E0CE0107960E942E568F
:10978000BE01635F7F4F0E944556BC01C8010E9425
:10979000DC55CE0107960E94C556CE0101960E9467
:1097A000C55660E170E1C8010E948C55F7016785DC
:1097B000062E000C770BCE0101960E945A5BBE016B
:1097C0006F5F7F4FCE0107960E942157BE01635FF6
:1097D0007F4FCE0107960E944556BC01C8010E94EA
:1097E000DC55CE0107960E94C556CE0101960E9417
:1097F000C5566AE070E1C8010E948C55F701608986
:109800007189CE0101960E945A5BBE016F5F7F4F46
:10981000CE0107960E942157BE01635F7F4FCE01A4
:1098200007960E944556BC01C8010E94DC55CE0136
:1098300007960E94C556CE0101960E94C55665E066
:1098400070E1C8010E948C55F70162897389CE01CD
:1098500001960E945A5BBE016F5F7F4FC8010E9454
:10986000DC55CE0101960E94C556CE010D960E9490
:10987000C556C80162960FB6F894DEBF0FBECDBFC5
:10988000DF91CF911F910F91FF90EF90DF90CF90DC
:10989000BF900895EF92FF920F931F93CF93DF93A2
:1098A000CDB7DEB768970FB6F894DEBF0FBECDBF59
:1098B0008C0166E67CE0CE010D960E9429576EE988
:1098C00079E0CE0143960E94295761EE7FE0C801FE
:1098D0000E941957BE016D5E7F4FC8010E94DC5582
:1098E00068ED7FE0C8010E948C558BE7E82E81E18E
:1098F000F82EF701608170E0CE0101960E945A5B5C
:10990000BE016F5F7F4FCE0107960E942157BE01B7
:10991000635F7F4FCE0107960E944556BC01C80188
:109920000E94DC55CE0107960E94C556CE010196D5
:109930000E94C5566BEC7FE0C8010E948C55F70170
:109940006181062E000C770BCE0101960E945A5BB6
:10995000BE016F5F7F4FCE0107960E942157BE0167
:10996000635F7F4FCE0107960E944556BC01C80138
:109970000E94DC55CE0107960E94C556CE01019685
:109980000E94C55661EC7FE0C8010E948C55F7012A
:109990006281062E000C770BCE0101960E945A5B65
:1099A000BE016F5F7F4FCE0107960E942157BE0117
:1099B000635F7F4FCE0107960E944556BC01C801E8
:1099C0000E94DC55CE0107960E94C556CE01019635
:1099D0000E94C55669EB7FE0C8010E948C55F701D3
:1099E00063817481CE0101960E945A5BBE016F5F54
:1099F0007F4FCE0107960E942157BE016D5E7F4FBB
:109A0000CE0107960E944556BC01C8010E94DC5554
:109A1000CE0107960E94C556CE0101960E94C556FA
:109A200062EA7FE0C8010E948C55F701658176816A
:109A3000CE0101960E945A5BBE016F5F7F4FCE013F
:109A400007960E942157BE01635F7F4FCE010796A4
:109A50000E944556BC01C8010E94DC55CE01079604
:109A60000E94C556CE0101960E94C55669E97FE065
:109A7000C8010E948C55F7016781062E000C770BF8
:109A80006F5F7F4FCE0101960E945A5BBE016F5FF0
:109A90007F4FCE0107960E942157BE01635F7F4F23
:109AA000CE0107960E944556BC01C8010E94DC55B4
:109AB000CE0107960E94C556CE0101960E94C5565A
:109AC0006EE87FE0C8010E948C55F7016085062E84
:109AD000000C770BCE0101960E945A5BBE016F5FAE
:109AE0007F4FC8010E94DC55CE0101960E94C556E9
:109AF000CE0143960E94C556CE010D960E94C556D2
:109B0000C80168960FB6F894DEBF0FBECDBFDF91D7
:109B1000CF911F910F91FF90EF9008950F931F9396
:109B2000CF93DF93CDB7DEB72C970FB6F894DEBF97
:109B30000FBECDBF8C0164E67AE089E992E10E9414
:109B40009B560830110509F0DAC066E071E1CE01DC
:109B500001960E94195744E650E06FEF7FEFCE0167
:109B600001960E949192CE0101960E94C5566AEF1D
:109B700070E1CE0101960E94195744E650E060E082
:109B800070E0CE0101960E944990CE0101960E949C
:109B9000C5568AE99DE051D54CE251E061E070E0A4
:109BA000CE0101960E94DF5F80911F148823D1F0BF
:109BB00061EA79E0CE0107960E942957BE016F5FE6
:109BC0007F4FCE0107960E94455664E277E00E94DF
:109BD0002E56BC0181E79FE00E94AE6FCE01079632
:109BE0000E94C55661E679E0CE0107960E9429578A
:109BF000BE01695F7F4FCE0101960E94F187182F49
:109C0000CE0107960E94C556112309F470C264EA7A
:109C100079E089E992E10E949B5688E090E0909378
:109C2000980C8093970C0E94E230182F6DEE70E133
:109C3000CE0107960E94195744E650E060E070E0BC
:109C4000CE0107960E944990CE0107960E94C55604
:109C50008AE99DE0F2D448E552E061E070E0CE018F
:109C600007960E94DF5FBE01695F7F4FCE010196BC
:109C7000A9D7CE0107960E94C55680911F1488234C
:109C8000C1F061EA79E0CE0107960E942957BE0132
:109C90006F5F7F4FCE010796F8D764E277E0DED79B
:109CA000BC0181E79FE00E94AE6FCE0107960E9443
:109CB000C55663E476E0CE0107960E942957BE019F
:109CC000695F7F4FCE0101960E94F187082FCE0178
:109CD00007960E94C556002309F409C269EA79E093
:109CE00089E992E10E949B560E94E230882309F4A0
:109CF000FEC1112309F4FBC160EE70E1E5C0093F2C
:109D00002FEF120709F0F4C06FEC70E1CE0101965D
:109D10000E94195744E650E06FEF7FEFCE010196A5
:109D20000E949192CE0101960E94C55661EC70E1AD
:109D3000CE0101960E94195744E650E060E070E0C1
:109D4000CE0101960E944990CE0101960E94C5560F
:109D50008AE99DE072D44CE251E064E070E0CE010B
:109D600001960E94DF5F80911F148823B9F061EA99
:109D700079E0CE0107960E942957BE016F5F7F4FA1
:109D8000CE01079682D764E277E068D7BC0181E70D
:109D90009FE00E94AE6FCE010796F7D760E070E0BB
:109DA000CE010196A8D6082E000C990BC0970A97F1
:109DB00008F0A0C16FEA79E0CE0107960E9429570A
:109DC000BE016F5F7F4FCE0107965FD7BC0189E967
:109DD00092E1C6D7CE010796D8D789EF9FEF90932F
:109DE000980C8093970C0E94E230182F63EB70E17F
:109DF000CE0107960E94195744E650E060E070E0FB
:109E0000CE0107960E944990CE010796BED78AE9F7
:109E10009DE013D448E552E065E070E0CE0107967E
:109E20000E94DF5FBE01695F7F4FCE010196CAD6F7
:109E3000CE010796AAD780911F148823B9F061EA52
:109E400079E0CE0107960E942957BE016F5F7F4FD0
:109E5000CE0107961AD764E277E000D7BC0181E70C
:109E60009FE00E94AE6FCE0107968FD760E070E052
:109E7000CE01019640D6082E000C990BC0970A9788
:109E800008F038C164EB79E0CE010796E2D7BE0155
:109E90006F5F7F4FCE010796F8D6BC0189E992E14A
:109EA0005FD7CE01079671D789EF9FEF9093980CFB
:109EB0008093970C0E94E230882309F41BC1112380
:109EC00009F418C166EA70E1CE010796B2D744E6FC
:109ED00050E060E070E0CE0107960E944990CE010C
:109EE000079653D764E67AE089E992E124D7FBC06C
:109EF00065E970E1CE0101969CD744E650E06FEF32
:109F00007FEFCE0101960E949192CE0101963DD73E
:109F100064E67AE089E992E10ED7053F8FEF1807F2
:109F200041F462ED78E089E992E105D76BE870E1F0
:109F300023C0063F2FEF120741F466EC78E089E971
:109F400092E1F9D661E870E117C0013F8FEF180781
:109F500041F460EE78E089E992E1EDD662E770E1E4
:109F60000BC0023F2FEF1207A9F469EB79E089E9F2
:109F700092E1E1D662E670E1CE0101965AD744E65D
:109F800050E06FEF7FEFCE0101960E944990CE0125
:109F90000196B3C00230110509F071C066E570E1A9
:109FA000CE01019646D744E650E06FEF7FEFCE0139
:109FB00001960E949192CE010196E7D666E470E187
:109FC000CE01019636D744E650E06FEF7FEFCE0129
:109FD00001960E944990CE010196D7D644EF51E0F8
:109FE00066E070E0CE0101960E94DF5FBE016F5F08
:109FF0007F4F89E992E1E6D5CE010196C6D68091E0
:10A000009D1290919E12059708F479C060E070E06F
:10A0100089E992E170D5082E000C990BC0970A9738
:10A0200008F06DC089E992E1FBD4613523EC720739
:10A03000810591050CF463C00E942EB120E030E050
:10A0400048EC52E40E947EB3AB01BC0122E0CE0199
:10A050000796A0D660E978E0CE010196FAD6BE0157
:10A06000695F7F4FCE01019610D6BC0189E992E16C
:10A0700077D6CE01019689D6CE0107963EC06FE213
:10A0800070E1CE010196D5D644E650E06FEF7FEF48
:10A09000CE0101960E944990CE01019676D664E6E3
:10A0A0007AE089E992E147D60B3E8FEF180709F471
:10A0B0005DC080919D1290919E12892BB1F556C082
:10A0C00068EC70E080E090E00E94018969E170E155
:10A0D000CE010196AED644EF51E06FEF7FEFCE0197
:10A0E00001960E944990CE0101964FD63FC069ED7E
:10A0F00070E1EACE6FE970E1E7CE47D6DACF68E3E8
:10A1000070E1CE01019695D648EE53E06FEF7FEFF8
:10A11000CE0101960E944990CE01019636D664E6A2
:10A120007AE089E992E107D6C4CF0E94E230882321
:10A1300039F268EC70E080E090E00E94018965E20D
:10A1400070E1CE01019675D644EF51E06FEF7FEFDD
:10A15000CE0101960E944990CE01019616D6109329
:10A16000980C0093970CC8010E94D70A2C960FB642
:10A17000F894DEBF0FBECDBFDF91CF911F910F913D
:10A1800008956F927F928F929F92AF92BF92CF92DB
:10A19000DF92EF92FF920F931F93CF93DF93CDB790
:10A1A000DEB768970FB6F894DEBF0FBECDBF6C0167
:10A1B0008091621190916311019729F064E67AE031
:10A1C000C60147D62AC165EC79E0CE010D9641D68D
:10A1D000BE01635F7F4F8AE99DE099D66CE271E032
:10A1E00080E090E00E940189CE0143960E941A6FA0
:10A1F00064E670E080E090E00E940189E12CF12C9F
:10A2000085E0A82EB12C9AE0892E912C60ED79E0A2
:10A21000CE0101961ED68F89988D892B69F06B88A7
:10A220007C8869817A81C3010E9499B8009721F0E6
:10A230008C010619170902C00FEF1FEFCE0101961E
:10A24000A4D5A8014F5F5F4FBE016D5E7F4FCE0169
:10A2500001960E94EC41BE016F5F7F4FCE010D96CB
:10A26000B1D4CE01019691D589899A89892B61F063
:10A2700060E070E0CE010D963ED4082E000C990BE4
:10A28000C0970A9708F4B4C010E06EE77FE0CE01F3
:10A290000196CFD544E150E06FEF7FEFCE010196FC
:10A2A0000E943693CE01019670D58FEFE81AF80A16
:10A2B00062E370E080E090E00E940189C701B5018F
:10A2C0000E94F3B5019759F5CE0101960E94D26D17
:10A2D0008D819E81892B51F0BE016F5F7F4F89E98F
:10A2E00092E13ED50E94578111E016C084E1E81644
:10A2F000F10494F0C701B4010E94F3B5892B61F415
:10A30000BE01635F7F4F8AE99DE001D668EC70E093
:10A3100080E090E00E940189CE01019636D5CE0101
:10A3200001960E941A6FBE016F5F7F4FCE01439668
:10A3300049D4CE01019629D562E370E080E090E037
:10A340000E94018984E6E816F10419F0112309F44A
:10A350005DCF80911F148823C9F06FE979E0CE01A9
:10A36000019677D5BE01635F7F4FCE0101968DD4F4
:10A37000BC01CE01079665D5CE0107960E94586AAA
:10A38000CE01079602D5CE010196FFD489899A891C
:10A39000892B59F060E070E0CE010D96ACD3082E09
:10A3A000000C990BC0970A9728F062ED79E0C6017E
:10A3B00050D517C06EED79E0CE0101964AD5BE01A9
:10A3C0006F5F7F4FCE010D960E94F187182FCE014F
:10A3D0000196DBD41111E9CFBE01635F7F4FC60147
:10A3E00020D5CE014396D1D4CE010D96CED415C042
:10A3F0006EED79E0CE0101962CD5BE016F5F7F4FE7
:10A40000CE010D960E94F187082FCE010196BDD492
:10A4100011E0002309F439CF37CFC60168960FB693
:10A42000F894DEBF0FBECDBFDF91CF911F910F918A
:10A43000FF90EF90DF90CF90BF90AF909F908F9064
:10A440007F906F9008950895CF92DF92EF92FF92E0
:10A450000F931F93CF93DF936C017A018B01C0E0C0
:10A46000D0E0CE15DF0581F0D8016D918D01D601C8
:10A47000ED91FC910190F081E02DC6011995892B99
:10A4800011F02196EECF7E01C701DF91CF911F9190
:10A490000F91FF90EF90DF90CF900895FC01538DC6
:10A4A000448D252F30E0842F90E0821B930B5417AE
:10A4B00010F0CF96089501970895FC01918D828D3B
:10A4C000981761F0828DDF01A80FB11D5D968C9108
:10A4D000928D9F5F9F73928F90E008958FEF9FEF13
:10A4E0000895FC01918D828D981731F0828DE80FCF
:10A4F000F11D858D90E008958FEF9FEF0895FC0189
:10A50000918D228D892F90E0805C9F4F821B910955
:10A510008F73992708958AE99DE0F1DF21E0892B67
:10A5200009F420E0822F089587E39EE0E8DF21E030
:10A53000892B09F420E0822F089584ED9EE0DFDF6F
:10A5400021E0892B09F420E0822F089581E79FE024
:10A55000D6DF21E0892B09F420E0822F0895FC0149
:10A56000848DDF01A80FB11DA35ABF4F2C91848D9C
:10A5700090E001968F739927848FA689B7892C93D1
:10A58000A089B1898C91837080648C93938D848D24
:10A59000981306C00288F389E02D80818F7D808327
:10A5A0000895EF92FF920F931F93CF93DF93EC01E7
:10A5B00081E0888F9B8D8C8D981305C0E889F9897F
:10A5C000808185FD25C0F62E0B8D10E00F5F1F4F9B
:10A5D0000F731127E02E8C8DE8120BC00FB607FC0D
:10A5E000FACFE889F989808185FFF5CFCE01B7DF01
:10A5F000F2CF8B8DFE01E80FF11DE35AFF4FF08281
:10A600009FB7F8940B8FEA89FB89808180620AC02A
:10A610009FB7F894EE89FF896083E889F989808182
:10A620008370806480839FBF81E090E0DF91CF9151
:10A630001F910F91FF90EF900895CF93DF93EC015E
:10A64000888D8823C1F0EA89FB89808185FD05C05A
:10A65000A889B9898C9186FD0EC00FB607FCF5CF8D
:10A66000808185FFF2CFA889B9898C9185FFEDCFD4
:10A67000CE0175DFE8CFDF91CF91089580E090E0C3
:10A68000892B19F063DF811116C080E090E0892BDF
:10A6900019F053DF811112C080E090E0892B19F08E
:10A6A00043DF81110EC080E090E0892B79F033DF29
:10A6B00081110AC008950E940000E7CF0E940000A7
:10A6C000EBCF0E940000EFCF0C94000008950E9491
:10A6D00046B80F931F93CF93DF93EC018881998144
:10A6E000009729F02A813B812617370788F48B01D0
:10A6F0006F5F7F4F0E9466B7009761F099838883F0
:10A700001B830A832C813D81232B11F4FC011082D1
:10A7100081E001C080E0DF91CF911F910F910895FA
:10A72000EF92FF920F931F93CF93DF936115710503
:10A7300011F480E01BC041155105B9F07B01EC011B
:10A740008C819D818A01080F191FB801CE01C1DFDC
:10A75000882379F3288139818C819D81B701820F0B
:10A76000931F0E9475B81D830C8381E0DF91CF9108
:10A770001F910F91FF90EF9008950F931F93CF9328
:10A78000DF938C01EB0188E2FB0111928A95E9F7D6
:10A790004BE050E066EE79E0CE010E948AB81B865D
:10A7A00081E090E0A0E0B0E08C879D87AE87BF8716
:10A7B000F80185899689A789B08D888B998BAA8B9A
:10A7C000BB8B82E090E0A0E0B0E08C8B9D8BAE8BE9
:10A7D000BF8B1CA21DA21EA21FA280E090E0A8E4D5
:10A7E000B4E4888F998FAA8FBB8F80E090E0A8E4B3
:10A7F000B4EC8C8F9D8FAE8FBF8F8DEC9CECACE456
:10A80000BEE388A399A3AAA3BBA3DF91CF911F9115
:10A810000F9108954F925F926F927F928F929F92C5
:10A82000AF92BF92CF92DF92EF92FF920F931F935E
:10A83000CF93DF938C01EB0184E2FB0111928A95A7
:10A84000E9F78EE10E94227083E090E00E941D7083
:10A850000E941B7066E08EE158D78091F51390E05E
:10A860002091F613821B910986309105ECF38EE05E
:10A8700090E10E941D7D882E8EE090E10E941D7D5A
:10A88000982E8EE090E10E941D7D682E8EE090E172
:10A890000E941D7D782E8EE090E10E941D7D482E45
:10A8A0008EE090E10E941D7D582EB82CA12CB501A0
:10A8B0006929072E000C880B990B0E942EB14B01C1
:10A8C0005C01F8016583768387839087D42CC12C43
:10A8D000B6016529072E000C880B990B0E942EB13A
:10A8E000F8016187728783879487F62CE12CB70182
:10A8F0006729072E000C880B990B0E942EB1F801D6
:10A90000658776878787908B118A128A138A148AC3
:10A9100084E290E0A0E0B0E088839983AA83BB83BF
:10A9200085899689A789B08D8C839D83AE83BF83EB
:10A9300082E090E0A0E0B0E088879987AA87BB8793
:10A94000188A198A1A8A1B8AC0906702D0906802F6
:10A95000E0906902F0906A02A7019601C501B40176
:10A960000E947EB320E030E048EC52E40E948DB1BA
:10A970006C8B7D8B8E8B9F8BA7019601F801618577
:10A980007285838594850E947EB320E030E048EC98
:10A9900052E40E948DB1688F798F8A8F9B8F2091AE
:10A9A0006302309164024091650250916602F801A1
:10A9B00065857685878590890E947EB320E030E0AA
:10A9C00048EC52E40E948DB16C8F7D8F8E8F9F8FEB
:10A9D00081E0DF91CF911F910F91FF90EF90DF9079
:10A9E000CF90BF90AF909F908F907F906F905F902F
:10A9F0004F900895862F0C942588862F642F0C94F1
:10AA00004D88862F642F0C947B88FC018081918176
:10AA1000009711F00C94B7AC60E070E0CB010895A2
:10AA2000FC0180819181009711F00C94BAAC60E038
:10AA300070E0CB010895AF92BF92CF92DF92EF9278
:10AA4000FF920F931F93CF93DF93DC01CD90DC90A7
:10AA50001197C114D10409F443C01496CD91DC912F
:10AA600015972097E9F18C0176015701BFEFAB1ADA
:10AA7000BB0AF7018081082E000C990B0E94F8B0E8
:10AA8000892B11F07501F1CF2197CC0DDD1D888147
:10AA9000082E000C990B0E94F8B0892B29F0CE15D6
:10AAA000DF0510F02197F3CFAE014F5F5F4F4E19D6
:10AAB0005F09D80115965C934E931497CE14DF046A
:10AAC00020F4B701C6010E9463B8D801ED91FC9152
:10AAD000119714968D919C911597E80FF91F10828C
:10AAE000DF91CF911F910F91FF90EF90DF90CF906A
:10AAF000BF90AF900895FC012481358162177307E0
:10AB000048F480819181009729F0FC01E60FF71F3E
:10AB10008081089580E00895EF92FF920F931F9334
:10AB2000CF93DF936115710511F480E01DC08B0197
:10AB3000EC01CB010E94E7AC0097A9F02C813D818C
:10AB40007C01E20EF31EB701CE01C3DD882369F359
:10AB5000288139818C819D81B801820F931F0E94C9
:10AB6000E0ACFD82EC8281E0DF91CF911F910F91EB
:10AB7000FF90EF900895CF93DF931F921F92CDB770
:10AB8000DEB769831A8241E050E0BE016F5F7F4FFC
:10AB9000C7DD0F900F90DF91CF910895611571057A
:10ABA00049F0FB0101900020E9F73197AF01461B06
:10ABB000570BB6CD80E00895FB014481558160813B
:10ABC0007181AECD0F931F93CF93DF938C01EB0177
:10ABD000FC0180819181009739F06881798161154C
:10ABE0007105A1F40E94DDB688819981F8019183F5
:10ABF00080838A819B81938382838C819D819583CD
:10AC00008483198218821B821A820FC0F801428144
:10AC100053812C813D814217530720F30E9475B860
:10AC20008C819D81F801958384831D821C82DF9134
:10AC3000CF911F910F910895CF93DF93EC018881FD
:10AC40009981009711F00E94DDB6198218821D8249
:10AC50001C821B821A82DF91CF910895CF93DF93DC
:10AC6000EC016115710559F0FB0101900020E9F735
:10AC70003197AF01461B570B53DD811102C0CE0146
:10AC8000DBDFCE01DF91CF910895CF93DF93EC010D
:10AC9000FB01448155816081718142DD811102C0D7
:10ACA000CE01CADFCE01DF91CF910895EF92FF92DE
:10ACB0000F931F93CF93DF93EC018B016115710507
:10ACC00049F0CB010E94E7AC7C01BC01CE0101DD63
:10ACD000811103C0CE01B0DF07C0FD82EC82B80154
:10ACE000888199810E94E0ACCE01DF91CF911F91C4
:10ACF0000F91FF90EF900895EF92FF920F931F93A3
:10AD0000CF93DF93EC017B018A01BA01E2DC811170
:10AD100003C0CE0191DF07C01D830C83B70188817A
:10AD200099810E9475B8CE01DF91CF911F910F914B
:10AD3000FF90EF900895CF93DF93EC0161157105BB
:10AD400051F0FB0101900020E9F73197AF01461B5C
:10AD5000570BD2DF01C070DFCE01DF91CF91089594
:10AD6000CF93DF93EC01FB018617970751F06081C9
:10AD700071816115710521F044815581BDDF01C0EC
:10AD80005BDFCE01DF91CF910895FC01808191813D
:10AD90000C94DDB6EF92FF920F931F93CF93DF9346
:10ADA000CDB7DEB7A1970FB6F894DEBF0FBECDBF0B
:10ADB0007C01CB01BA01F701118210821382128249
:10ADC0001582148242E0420F8E010F5F1F4F0E94D6
:10ADD00098ACBC01C701AFDFA1960FB6F894DEBFF7
:10ADE0000FBECDBFDF91CF911F910F91FF90EF90DC
:10ADF0000895CF93DF931F921F92CDB7DEB7FC016A
:10AE000011821082138212821582148269831A823F
:10AE1000BE016F5F7F4F8FDF0F900F90DF91CF915B
:10AE20000895FC011182108213821282158214820D
:10AE3000C9CEFC0111821082138212821582148203
:10AE400035CFFC0111821082138212821582148286
:10AE500087CFFC0111821082138212821582148224
:10AE60006115710549F0FB0101900020E9F7319768
:10AE7000AF01461B570B40CF0895BF92CF92DF9290
:10AE8000EF92FF920F931F93CF93DF937C016B019F
:10AE90008A01E9012417350720F4812F8901C42F85
:10AEA000D82F64E67AE0C701D4DFD60114968D91DD
:10AEB0009C91159708171907C0F48C179D0708F483
:10AEC000EC01D601ED91FC911197EC0FFD1FB080C4
:10AED00010826D917C91600F711FC7012CDFD6012C
:10AEE000ED91FC91EC0FFD1FB082C701DF91CF9176
:10AEF0001F910F91FF90EF90DF90CF90BF9008953A
:10AF0000DC01ED91FC910190F081E02D1994DB01C1
:10AF100014964D915C9115976D917C91DC01ED91AA
:10AF2000FC910280F381E02D1994EF92FF920F9330
:10AF30001F93CF93DF938C017B01C0E0D0E0F7013A
:10AF4000EC0FFD1F6491662361F0D801ED91FC9137
:10AF50000190F081E02DC8011995892B11F02196FF
:10AF6000EECFCE01DF91CF911F910F91FF90EF9027
:10AF700008956115710579F0FB0101900020E9F752
:10AF80003197AF01461B570BDC01ED91FC9102801C
:10AF9000F381E02D199480E090E008958F929F92C4
:10AFA000AF92BF92EF92FF920F931F93CF93DF93D5
:10AFB000CDB7DEB7A1970FB6F894DEBF0FBECDBFF9
:10AFC0007C01FA01CB0119A2223008F42AE08E019B
:10AFD0000F5D1F4F822E912CA12CB12CBF01A5011A
:10AFE00094010E9486B2F901CA01015011096A3028
:10AFF00014F4605D01C0695CD8016C93232B242B91
:10B00000252B61F7B801C701B4DFA1960FB6F894FC
:10B01000DEBF0FBECDBFDF91CF911F910F91FF908B
:10B02000EF90BF90AF909F908F900895CF92DF9256
:10B03000EF92FF920F931F93CF93DF93411551052A
:10B0400079F4DC01ED91FC910190F081E02DDF912C
:10B05000CF911F910F91FF90EF90DF90CF901994B7
:10B060006B01770FEE08FF084A305105E9F4F7FE4F
:10B0700019C0EC016DE244DF8C0144275527BA0169
:10B080004C195D096E097F092AE0CE0187DF800F28
:10B09000911FDF91CF911F910F91FF90EF90DF9063
:10B0A000CF9008952AE001C0242FB701A601DF91B7
:10B0B000CF911F910F91FF90EF90DF90CF906ECFC7
:10B0C00058CF1F920F920FB60F9211240BB60F920A
:10B0D0002F933F934F935F936F937F938F939F93A0
:10B0E000AF93BF93EF93FF938AE99DE038DAFF9126
:10B0F000EF91BF91AF919F918F917F916F915F91F0
:10B100004F913F912F910F900BBE0F900FBE0F905C
:10B110001F9018951F920F920FB60F9211240BB625
:10B120000F922F933F934F935F936F937F938F93E0
:10B130009F93AF93BF93EF93FF938AE99DE00E94A3
:10B140000C88FF91EF91BF91AF919F918F917F916B
:10B150006F915F914F913F912F910F900BBE0F9088
:10B160000FBE0F901F9018951F920F920FB60F925F
:10B1700011240BB60F922F933F934F935F936F93CE
:10B180007F938F939F93AF93BF93EF93FF9387E347
:10B190009EE0E5D9FF91EF91BF91AF919F918F9183
:10B1A0007F916F915F914F913F912F910F900BBEC7
:10B1B0000F900FBE0F901F9018951F920F920FB611
:10B1C0000F9211240BB60F922F933F934F935F93DF
:10B1D0006F937F938F939F93AF93BF93EF93FF935F
:10B1E00087E39EE00E940C88FF91EF91BF91AF91A1
:10B1F0009F918F917F916F915F914F913F912F918F
:10B200000F900BBE0F900FBE0F901F9018951F92BE
:10B210000F920FB60F9211240BB60F922F933F93FC
:10B220004F935F936F937F938F939F93AF93BF934E
:10B23000EF93FF9384ED9EE092D9FF91EF91BF9140
:10B24000AF919F918F917F916F915F914F913F91BE
:10B250002F910F900BBE0F900FBE0F901F9018955F
:10B260001F920F920FB60F9211240BB60F922F93CD
:10B270003F934F935F936F937F938F939F93AF937E
:10B28000BF93EF93FF9384ED9EE00E940C88FF91A3
:10B29000EF91BF91AF919F918F917F916F915F914E
:10B2A0004F913F912F910F900BBE0F900FBE0F90BB
:10B2B0001F9018951F920F920FB60F9211240BB684
:10B2C0000F922F933F934F935F936F937F938F933F
:10B2D0009F93AF93BF93EF93FF9381E79FE03FD995
:10B2E000FF91EF91BF91AF919F918F917F916F915E
:10B2F0005F914F913F912F910F900BBE0F900FBE1A
:10B300000F901F9018951F920F920FB60F92112455
:10B310000BB60F922F933F934F935F936F937F934F
:10B320008F939F93AF93BF93EF93FF9381E79FE03A
:10B330000E940C88FF91EF91BF91AF919F918F91E7
:10B340007F916F915F914F913F912F910F900BBE25
:10B350000F900FBE0F901F901895DC0180E0615098
:10B3600098F02D91982F9227E92FEF70F0E0E05F91
:10B37000FE4E249192959F70E92FF0E0E05EFE4E24
:10B38000E491822F8E27EBCF0895EF92FF920F93D7
:10B390001F93CF93DF938C017B0140E065E50E9412
:10B3A000EB7DE70188E0E80EF11C699140E0C801FF
:10B3B0000E94EB7DCE15DF05C1F7DF91CF911F9184
:10B3C0000F91FF90EF9008956F927F928F929F92CE
:10B3D000AF92BF92CF92DF92EF92FF920F931F93A3
:10B3E000CF93DF93EC017B018A018E819F810E94C4
:10B3F0001E7E8823A1F1B7018E819F81C6DF40E0C8
:10B400006EEB8E819F810E94EB7D7801680189E05F
:10B41000C80ED11CAE80BF8088E0882E912C712C84
:10B4200066246394C5010E94987D81117628660C7C
:10B43000E1E08E1A9108B1F7F70171927F01EC15E6
:10B44000FD0541F78E819F810E941E7E813039F477
:10B4500068E0C80182DF91E0F8012085281390E0C0
:10B46000892FDF91CF911F910F91FF90EF90DF9087
:10B47000CF90BF90AF909F908F907F906F900895E6
:10B48000CF93DF93CDB7DEB729970FB6F894DEBF21
:10B490000FBECDBFAE014F5F5F4F96DF882389F0AF
:10B4A0008D818F3361F020F48F3159F489E00CC025
:10B4B0008F3519F08F3739F004C08BE005C08AE072
:10B4C00003C080E001C08CE029960FB6F894DEBF7F
:10B4D0000FBECDBFDF91CF910895BF92CF92DF9283
:10B4E000EF92FF920F931F93CF93DF93EC016B01C9
:10B4F0008D85811105C0CE010E941E7E811105C07F
:10B500001B861D861C8680E060C040E060EFCE0197
:10B510000E94EB7D01E0E12CB12C11E0CE010E94F4
:10B52000987DF82ECE010E94987D91E0F91203C01B
:10B530008130B1F434C02E2D30E0F8121BC08B8561
:10B54000181738F4FE01E20FF31F8381802341F4C2
:10B5500002C0811729F0F12C193058F41C8709C05A
:10B56000FE01EE0DF11D8381802B8383FF24F39474
:10B5700009C0B12EFE01E20FF31F9381802F809549
:10B58000892383836F2DCE010E94BC7D1F5F000F36
:10B5900011F4E39401E087E08E1508F0BFCF113479
:10B5A00008F4AECFBB86B11002C081E08D878B81DD
:10B5B000882309F4A5CFDE011396F6012B968D9111
:10B5C0008193CA17DB07D9F781E0DF91CF911F91F3
:10B5D0000F91FF90EF90DF90CF90BF900895DF9292
:10B5E000EF92FF920F931F93CF93DF937C018B0118
:10B5F000D42EDC011696ED91FC91179713861586D3
:10B600001486DF011B9633961E92EA17FB07E1F7BB
:10B61000C0E0B801F701868197815FDFD82F8823CA
:10B6200069F0DC1208C067E0C80197DED801179600
:10B630009C91891721F0CF5FDC1658F7D0E08D2F51
:10B64000DF91CF911F910F91FF90EF90DF900895C0
:10B650001092F6131092F5131092780D1092990D26
:10B660001092760D81E08093750D1092500D61E07F
:10B6700084E10E944D8861E085E10E944D88E9EBFC
:10B68000F0E080818E7F808380818D7F808388E45D
:10B690008093B80085E48093BC008BE09DE7909395
:10B6A000E70C8093E60C8CE09DE79093E50C80938B
:10B6B000E40C08950F931F93CF93DF93CDB7DEB7BC
:10B6C00062970FB6F894DEBF0FBECDBF8C01CB01E1
:10B6D000F8011182108213821282158214824AE0CC
:10B6E000BE016F5F7F4F0E94F0ACBE016F5F7F4F66
:10B6F000C80121DB62960FB6F894DEBF0FBECDBF46
:10B70000DF91CF911F910F910895613208F060E2AF
:10B710000E94BD911092F6138093F5130895AF9295
:10B72000BF92CF92DF92EF92FF920F931F93CF932E
:10B73000DF93C82FD62F1092DD121092DE121092D6
:10B74000DF121092E0121092E11261E00E947B88F9
:10B7500060E08C2F0E944D886D2F70E080E090E0BB
:10B760000E94018960E08C2F0E947B888BE990E029
:10B770000197F1F700E911E08C2F0E942588892BB1
:10B7800031F401501109C1F78EEF9FEF4CC000E971
:10B7900011E08C2F0E942588019709F43FC018E220
:10B7A000D0E800E090E9E92EFF24F3948C2F0E946A
:10B7B0002588892B29F481E0E81AF108B9F7E4CF4C
:10B7C0000E94DC886B017C0180E9A82EBB24B39425
:10B7D0008C2F0E942588019729F481E0A81AB108CE
:10B7E000B9F7D2CF0E94DC88DC01CB018C199D090E
:10B7F000AE09BF098997A105B10538F0E02FF0E047
:10B80000EB52FD4E80858D2B8087D69511F40F5F0E
:10B81000D0E8115039F680E090E005C001501109E0
:10B8200009F0B7CFB1CFDF91CF911F910F91FF906A
:10B83000EF90DF90CF90BF90AF900895EF92FF927E
:10B840000F931F93CF93DF93C82F8B017A0183E56A
:10B850000E9422706C2F8EE090E10E94657D0E9414
:10B860001B7083E50E942270B80183E590E00E947E
:10B87000FF91E701CE018E199F093091F5132091B8
:10B88000F613321731F08EE090E10E941D7D89930E
:10B89000F1CF0817190729F01092E31281E0809385
:10B8A000E412DF91CF911F910F91FF90EF900C94D4
:10B8B0001B70CF93DF934AE050E0BC0181E79FE02B
:10B8C000B5DBEC0181E79FE00E94AA6F8C0F9D1F02
:10B8D000DF91CF9108951F93CF93DF931F92CDB740
:10B8E000DEB7162FAE014F5F5F4F61E070E0A6DF5D
:10B8F000898190E002C0959587951A95E2F781704D
:10B900000F90DF91CF911F910895CF93DF93D82FA0
:10B91000C62F83E50E9422706D2F8EE090E10E9479
:10B92000657D6C2F8EE090E10E94657DDF91CF9167
:10B930000C941B70FF920F931F93CF93DF931F9272
:10B94000CDB7DEB7182F062FF42EAE014F5F5F4F35
:10B9500061E070E073DF4981FF2049F021E030E0D1
:10B9600001C0220F0A95EAF7242B298309C081E040
:10B9700090E001C0880F0A95EAF7809584238983B7
:10B980006981812FC2DF0F90DF91CF911F910F91BD
:10B99000FF9008950F931F93CF93DF93EC019A01CB
:10B9A000452B19F40E94D15205C0462F50E060E0AB
:10B9B00070E0F4DA8C01CE010E94AA6F800F911F13
:10B9C000DF91CF911F910F910895CF93DF9342E0C4
:10B9D0000E94D970EC0181E79FE00E94AA6F8C0F52
:10B9E0009D1FDF91CF9108958F929F92AF92BF924A
:10B9F000CF92DF92EF92FF920F931F93CF93DF933B
:10BA000000D000D0CDB7DEB75C0141EF52E166E077
:10BA100070E082E313DF8091F1129091F2129A8329
:10BA200089838091F3129091F4129C838B8380918F
:10BA3000F5129091F6129E838D83CE0101966C01D2
:10BA400085EEE82E82E1F82E8501F6016191719173
:10BA50006F01F70181909190A190B1907F01072E25
:10BA6000000C880B990B0E942EB1A50194010E9435
:10BA70008DB1F80161937193819391938F01F1EFEF
:10BA8000EF16F2E1FF0609F726960FB6F894DEBF2F
:10BA90000FBECDBFDF91CF911F910F91FF90EF901F
:10BAA000DF90CF90BF90AF909F908F900895CF93ED
:10BAB000DF93C82F809169130E9422706C2F8EE053
:10BAC00090E10E94657D80E00E94BF6F63E08091FD
:10BAD00069131BDE8EE090E10E941D7DEC018EE07B
:10BAE00090E10E941D7D20E030E0382FC9018C2BB1
:10BAF0009D2BDF91CF9108950F931F93CF93DF93E9
:10BB0000CDB7DEB761970FB6F894DEBF0FBECDBFDD
:10BB10008C01462FBE01665F7F4F61DD811105C03C
:10BB200060E070E08EEF92EC4BC0AE014F5F5F4F74
:10BB3000BE01665F7F4FC80147DC882361F12A811F
:10BB400030E0C901982F8827990F990F990F6981C3
:10BB500028E0629FB00111249C01262B372B8A8597
:10BB60008031E1F4688570E08F81AB01481B510999
:10BB7000CA019695982F8827979587950E94F3B5C7
:10BB800060517109207F53E0220F331F5A95E1F76E
:10BB9000620F731F04C060E874EE01C0B901613820
:10BBA00054EE75070CF4BCCF072E000C880B990BD4
:10BBB0000E942EB120E030E040E05CE30E948DB1B5
:10BBC00061960FB6F894DEBF0FBECDBFDF91CF9167
:10BBD0001F910F9108959F92AF92BF92CF92DF92E3
:10BBE000EF92FF920F931F93CF93DF93CDB7DEB702
:10BBF00061970FB6F894DEBF0FBECDBF8C018CE00D
:10BC0000F8018183C12CD12C2FE5E22E3FE7B32E22
:10BC10004FE1A42E5FE3952EF801848190E0C816D1
:10BC2000D9060CF09DC04C2DBE01665F7F4FC80148
:10BC3000D6DCF8018181893038F0F82EFCE0F81765
:10BC400028F49CE0F92E02C089E0F82E8A85803124
:10BC500031F0BE01665F7F4FC80112DC01C08CE08D
:10BC6000F81609F479C0AE014F5F5F4FBE01665F01
:10BC70007F4FC801A9DB882309F46EC08A85803113
:10BC800009F46AC08BE0F81651F0ECE0FE1629F0DA
:10BC9000FAE0FF1206C09D8205C0BD8203C0ED829E
:10BCA00001C0AD82F801868197810E941E7EBE018F
:10BCB000665F7F4FF8018681978167DB40E06EE425
:10BCC000F801868197810E94EB7D40E06B81F8014D
:10BCD000868197810E94EB7D40E06C81F80186812E
:10BCE00097810E94EB7D8A85803139F040E06D813B
:10BCF000F801868197810E94EB7DF801868197810A
:10BD00000E941E7EBE01665F7F4FF801868197818B
:10BD10003CDBF801408168E4868197810E94EB7DDD
:10BD200064E170E080E090E00E940189F801808188
:10BD3000882331F06AE070E080E090E00E940189A1
:10BD4000F801868197810E941E7EF80181818F15FE
:10BD500008F48F2DF8018183FFEFCF1ADF0A5CCF43
:10BD600061960FB6F894DEBF0FBECDBFDF91CF91C5
:10BD70001F910F91FF90EF90DF90CF90BF90AF9009
:10BD80009F9008958F929F92AF92BF92CF92DF9231
:10BD9000EF92FF920F931F93CF93DF93EC018E816D
:10BDA0009F810E941E7E40E06CEC8E819F810E94EC
:10BDB000EB7D488164E48E819F810E94EB7D8A81C6
:10BDC000882309F442C0E981E950E33040F4F0E00F
:10BDD000EE0FFF1FEB5CFA4F0081118102C00EEEE7
:10BDE00012E08B818823F9F0888181111CC00E94A8
:10BDF0005D8A4B015C016801110FEE08FF088E811E
:10BE00009F810E94987D813001F10E945D8ADC0152
:10BE1000CB018C199D09AE09BF0988159905AA05A2
:10BE2000BB0568F312C0B801110F880B990BDF91A5
:10BE3000CF911F910F91FF90EF90DF90CF90BF9027
:10BE4000AF909F908F900C940189DF91CF911F91BB
:10BE50000F91FF90EF90DF90CF90BF90AF909F90A9
:10BE60008F900895EF92FF920F931F93CF93DF93DC
:10BE7000CDB7DEB728970FB6F894DEBF0FBECDBFA3
:10BE80008C01DC011696ED91FC91179713861586AF
:10BE90001486DF011B9633961E92EA17FB07E1F723
:10BEA000F80114821582EE24E394BE016F5F7F4F88
:10BEB000D80116968D919C9117970FDB882309F472
:10BEC00071C067E0CE01019648DA98858913EDCFFD
:10BED000F8018081811123C0868197810E941E7E96
:10BEE000BE016F5F7F4FD80116968D919C91179779
:10BEF0004CDA40E064EBF801868197810E94EB7D8B
:10BF0000D80116968D919C9117970E94987DF82ED6
:10BF1000F801868197810E941E7EFF20A1F1D80141
:10BF20001196FC9089818031C9F1BE016F5F7F4F0E
:10BF3000C801A6DA8F1518F4F80181810AC0898139
:10BF4000803111F48CE005C0BE016F5F7F4FC801E6
:10BF500097DAD80111968C93119714968C911497B7
:10BF60008F5F14968C938981883281F030F4803110
:10BF700069F0823209F099CF09C08B3339F08234ED
:10BF800009F093CF03C0F801E082C9CFD80115961C
:10BF90008C9115978F5F15968C9387CFBCE0BF155A
:10BFA00058F2D0CF28960FB6F894DEBF0FBECDBFA3
:10BFB000DF91CF911F910F91FF90EF9008956F92B5
:10BFC0007F928F929F92AF92BF92CF92DF92EF9229
:10BFD000FF920F931F93CF93DF93CDB7DEB72C97CC
:10BFE0000FB6F894DEBF0FBECDBF7C015B014A01E6
:10BFF00064E67AE00E94295764E67AE0CE0107966B
:10C000000E942957C12CD12C35018FEF681A780A6C
:10C010008E010F5F1F4FC814D9040CF084C0F701C4
:10C02000848195818615970508F07DC0B501C8010A
:10C030000E94058EB801CE0107960E94E255C80104
:10C040000E94C55664E170E080E090E00E940189A2
:10C050008B859C85892B61F4B501C8010E94A38C56
:10C06000B801CE0107960E94E255C8010E94C5564C
:10C070008B859C85892B79F067E278E08F819885A4
:10C080000E946CB8892BD9F4F701248135812115E0
:10C09000310569F514C064E170E080E090E00E9431
:10C0A0000189F701848195818A159B0520F4EFEFC2
:10C0B000CE1ADE0AB0CFF5E1CF0ED11CACCFBE0157
:10C0C000695F7F4FC7010E94DC55F2E3CF1AD108A8
:10C0D000B701C8010E94215742E350E06FEF7FEFA4
:10C0E000C8010E944990C8010E94C556DACF22308B
:10C0F000310530F464E67AE0C7010E949B56E5CF33
:10C100002150310940E050E0B701C8010E943D577D
:10C110000E151F0521F0B801C7010E94E255C801A4
:10C120000E94C556D2CFCE0107960E94C556C701C0
:10C130002C960FB6F894DEBF0FBECDBFDF91CF9126
:10C140001F910F91FF90EF90DF90CF90BF90AF9035
:10C150009F908F907F906F900895AF92BF92CF92F3
:10C16000DF92EF92FF920F931F93CF93DF93CDB7A0
:10C17000DEB72C970FB6F894DEBF0FBECDBF80910F
:10C18000D30C811102C00E94A141809105029091BF
:10C190000602029751F080919D0C90919E0C0097A1
:10C1A00009F48AC1039709F487C16FE571E18BE750
:10C1B00092E10E9456566BE772E1CE0101960E9411
:10C1C000215744E150E060E070E0CE0101960E940A
:10C1D0009192CE0101960E94C55660E571E18BE710
:10C1E00092E10E9456566BE772E1CE0101960E94E1
:10C1F000215744E150E06FEF7FEFCE0101960E949E
:10C200004990CE0101960E94C55687E050DC8C0112
:10C2100086E04DDCBC0180E090E00E942CB12AE079
:10C2200037ED43EA5CE30E948DB123E333E948E84C
:10C2300053E40E94B7B26B017C0184E0A82EB12CBC
:10C2400020E030E048EC52E4C701B6010E946DB432
:10C2500018160CF581E0A81AB10809F4F3C064E6D9
:10C2600070E080E090E00E94018986E020DCBC0163
:10C2700080E090E00E942CB12AE037ED43EA5CE3D5
:10C280000E948DB123E333E948E853E40E94B7B23A
:10C290006B017C01D5CFB80180E090E00E942CB109
:10C2A0002AE037ED43EA5CE30E948DB123E333E9F2
:10C2B00048E853E40E94B7B2AB01BC0121E0CE01D3
:10C2C00001960E94CA5660E07AE0CE0107960E946D
:10C2D0002957BE016F5F7F4FCE0107960E944556DA
:10C2E000BC0181E892E10E94B056CE0107960E94FF
:10C2F000C556CE0101960E94C55661E872E1CE0195
:10C3000001960E94215742E350E06FEF7FEFCE018C
:10C3100001960E944990CE0101960E94C5566AE09E
:10C320007AE0CE0101960E942957CE0101960E9423
:10C33000C590CE0101960E94C55669E07AE081E879
:10C3400092E10E94CE5521E0B701A601CE010196EF
:10C350000E94CA5662EA7AE0CE0107960E942957E7
:10C36000BE016F5F7F4FCE0107960E944556BC010C
:10C3700087E892E10E94B056CE0107960E94C5560A
:10C38000CE0101960E94C55666E67CE0CE0101967C
:10C390000E94295767E872E1CE0101960E94455636
:10C3A000BC018BE792E10E94B056CE0101960E943B
:10C3B000C5566BE772E1CE0101960E9421574AE013
:10C3C00050E060E070E0CE0101960E943693CE010D
:10C3D00001960E94C5566AE07AE0CE0101960E945D
:10C3E0002957CE0101960E94C590CE0101960E9468
:10C3F000C55669E07AE087E892E10E94CE5567E889
:10C4000072E1CE0101960E94215766E67CE0CE01E2
:10C4100001960E942E5661E872E10E944556BC01C9
:10C4200081E892E10E94B056CE0101960E94C55665
:10C4300080919D0C90919E0C039709F006C184E0B9
:10C4400090E0FFC065E471E18BE792E10E945656EF
:10C450006BE772E1CE0101960E9421574AE050E05D
:10C4600060E070E0CE0101960E949192CE010196AB
:10C470000E94C5566EEE79E0CE0101960E942957C2
:10C480006BE772E1CE0101960E944556BC0181E83E
:10C4900092E10E94B056CE0101960E94C55680914D
:10C4A0009D0C90919E0C049721F410929E0C10927A
:10C4B0009D0C81E090E018C187E39EE00E94E3902C
:10C4C00064E670E080E090E00E94018965E871E137
:10C4D0008BE792E10E9456566BE772E1CE0101961E
:10C4E0000E94215744E150E060E070E0CE010196E7
:10C4F0000E949192CE0101960E94C55666E771E1B5
:10C500008BE792E10E9456566BE772E1CE010196ED
:10C510000E94215744E150E06FEF7FEFCE0101967A
:10C520000E944990CE0101960E94C5568CE40E945B
:10C5300001916B017C0104E010E0A7019601C701A5
:10C54000B6010E94B7B5811192C021E0B701A601E2
:10C55000CE0107960E94CA5660E07AE0CE010196AD
:10C560000E942957BE01695F7F4FCE0101960E944C
:10C570004556BC0181E892E10E94B056CE01019679
:10C580000E94C556CE0107960E94C55661E872E129
:10C59000CE0101960E94215742E350E06FEF7FEFFA
:10C5A000CE0101960E944990CE0101960E94C55687
:10C5B0006AE07AE0CE0101960E942957CE010196E9
:10C5C0000E94C590CE0101960E94C55669E07AE0AE
:10C5D00081E892E10E94CE5586E60E9401916B01AE
:10C5E0007C0104E010E0A7019601C701B6010E949A
:10C5F000B7B5882309F47DC00150110909F0E2C0E4
:10C6000064E67AE087E892E10E949B5667E872E16F
:10C61000CE0101960E94215766E67CE0CE0101968C
:10C620000E942E5661E872E10E944556BC0181E8E5
:10C6300092E10E94B056CE0101960E94C55683E059
:10C6400090E090939E0C80939D0C64E670E080E0F7
:10C6500090E00E9401898091D30C882309F4BEC028
:10C6600060E273E080E090E00E940189B7C0015071
:10C67000110909F09BC06BE671E18BE792E10E9422
:10C6800056566BE772E1CE0101960E9421574AE0AF
:10C6900050E060E070E0CE0101960E949192CE01E0
:10C6A00001960E94C5566EEE79E0CE0101960E9479
:10C6B00029576BE772E1CE0101960E944556BC01F5
:10C6C00081E892E10E94B056CE0101960E94C556C3
:10C6D00080919D0C90919E0C039721F410929E0CDA
:10C6E00010929D0C82E090E09093060280930502E8
:10C6F000ACCF21E0B701A601CE0107960E94CA5631
:10C7000062EA7AE0CE0101960E942957BE01695F74
:10C710007F4FCE0101960E944556BC0187E892E109
:10C720000E94B056CE0101960E94C556CE010796D2
:10C730000E94C55666E67CE0CE0101960E9429570C
:10C7400067E872E1CE0101960E944556BC018BE775
:10C7500092E10E94B056CE0101960E94C5566BE749
:10C7600072E1CE0101960E9421574AE050E06FEF3E
:10C770007FEFCE0101960E943693CE0101960E9472
:10C78000C5566AE07AE0CE0101960E942957CE0193
:10C7900001960E94C590CE0101960E94C55669E09F
:10C7A0007AE087E892E10E94CE5530CF68EC70E0E5
:10C7B00080E090E00E9401898CE40E9401916B016D
:10C7C0007C01BBCE68EC70E080E090E00E940189C3
:10C7D00086E60E9401916B017C0105CF2C960FB675
:10C7E000F894DEBF0FBECDBFDF91CF911F910F91A7
:10C7F000FF90EF90DF90CF90BF90AF9008952F9271
:10C800003F924F925F926F927F928F929F92AF92E0
:10C81000BF92CF92DF92EF92FF920F931F93CF932D
:10C82000DF93CDB7DEB7C554D1090FB6F894DEBF9C
:10C830000FBECDBF2B013C0169017A010E945D8AC8
:10C8400022966CAF7DAF8EAF9FAF229720E9421644
:10C8500021E052066104710434F090E9492E552418
:10C860005394612C712C30E1C31637E2D306E104F6
:10C87000F1042CF4CDA6DEA6EFA6F8AA08C080E14C
:10C8800097E2A0E0B0E08DA79EA7AFA7B8AB8091DC
:10C89000D30C882321F0CDA6DEA6EFA6F8AA229617
:10C8A0006CAD7DAD8EAD9FAD229728EE33E040E0BC
:10C8B00050E00E945AB226962CAF3DAF4EAF5FAF0C
:10C8C000269791E09DAB19A61AA61BA61CA68E0161
:10C8D000035F1F4FCC24DD247601C418D508E60879
:10C8E000F708C9AADAAAEBAAFCAAC9A4DAA4EBA49D
:10C8F000FCA42DA53EA54FA558A9C216D306E40653
:10C90000F5060CF02BC3C701B6010E942EB120E042
:10C9100030E04AE754E40E947EB3AB01BC0123E05F
:10C92000C8010E94CA56B8018BE792E10E94E25505
:10C93000C8010E94C5568DA59EA5AFA5B8A90A97A6
:10C94000A105B1058CF426964CAD5DAD6EAD7FAD05
:10C950002697C8010E946870B8018BE792E10E9497
:10C96000E255C8010E94C556CE0101963DD868E344
:10C9700071E181E892E10E945656DE0111961D0197
:10C98000C12CD12C7601F10181909190A190B190B0
:10C990001F01A5019401C501B4010E948DB19B0145
:10C9A000AC01C701B6010E94B8B26B017C0123E063
:10C9B000B501A401C8010E94CA56B801CE01439630
:10C9C0000E94215766E67CE0CE0143960E942E56D7
:10C9D000BC0181E892E10E94DC55CE0143960E94A1
:10C9E000C556C8010E94C5560215130561F6C70158
:10C9F000B6010E9476B56B017C01FDE24F16F1E0B5
:10CA00005F066104710434F00E94A14160E080E09F
:10CA10000E943D7023E0B701A601CE0143960E941B
:10CA2000CA566CE879E0C8010E9429576BE772E1A9
:10CA3000C8010E9445566CE07AE00E942E56BE0165
:10CA40006D5E7F4F0E94455661E17AE00E942E564E
:10CA5000BC0181E892E10E94DC55C8010E94C556E4
:10CA6000CE0143960E94C5562DEC3CEC4CE45FE3AE
:10CA7000C701B6010E946DB429813A814B815C8166
:10CA80002DA33EA34FA358A718160CF0ABC12AE95B
:10CA900039E949E95FE3C701B6010E9428B187FF80
:10CAA000A1C1CDA8CC2009F49DC189849A84AB840E
:10CAB000BC8420E030E0A901C501B4010E9428B186
:10CAC000CD80DE80EF80F884882309F12DA13EA17E
:10CAD0004FA158A5CA01B9010E948DB16EAB7FABC1
:10CAE00088AF99AFA7019601C701B6010E948DB129
:10CAF0009B01AC016EA97FA988AD99AD0E94B8B227
:10CB00000E9476B5A50194010E942BB304C06BED81
:10CB10007FE089EC9FE320EE3EE245E652E40E948E
:10CB20008DB16EAB7FAB88AF99AF20E030E0A9014B
:10CB3000C701B6010E9428B1882309F12DA13EA1A9
:10CB40004FA158A5CA01B9010E948DB16AAF7BAF50
:10CB50008CAF9DAFA5019401C501B4010E948DB1B8
:10CB60009B01AC016AAD7BAD8CAD9DAD0E94B8B2AE
:10CB70000E9476B5A70196010E942BB304C06BED0D
:10CB80007FE089EC9FE320EE3EE245E652E40E941E
:10CB90008DB16AAF7BAF8CAF9DAF20E030E0A901D3
:10CBA0006DA17EA18FA198A50E9428B18823F9F0DC
:10CBB000A5019401C501B4010E948DB14B015C0136
:10CBC000A7019601C701B6010E948DB19B01AC017E
:10CBD000C501B4010E94B8B20E9476B52DA13EA154
:10CBE0004FA158A50E942BB36B017C0108C08BEDAF
:10CBF000C82E8FE0D82E89ECE82E8FE3F82E6DE852
:10CC000079E0C8010E9429576BE772E1C8010E94D0
:10CC1000455664E17AE00E942E56BC0181E892E11B
:10CC20000E94B056C8010E94C5566DE879E0C8015F
:10CC30000E9429576BE772E1C8010E9445566EE2D7
:10CC40007AE00E942E56BC018BE792E10E94B0561A
:10CC5000C8010E94C55621E04EA95FA968AD79AD13
:10CC6000CE014F960E94CA5621E04AAD5BAD6CAD35
:10CC70007DADCE0149960E94CA5620EE3EE245E6C1
:10CC800052E4C701B6010E948DB1AB01BC0121E0A5
:10CC9000C8010E94CA56B801CE0143960E9421578E
:10CCA00066E67CE0CE0143960E942E56BE01675E8A
:10CCB0007F4F0E94455666E67CE00E942E56BE01DC
:10CCC000615E7F4F0E944556BC0185E792E10E945C
:10CCD000B056CE0143960E94C556C8010E94C55663
:10CCE000CE0149960E94C556CE014F960E94C55668
:10CCF0002DE2421621E052066104710474F469A524
:10CD00007AA58BA59CA525E030E040E050E00E948C
:10CD10005AB2672B682B692BC1F56BE772E1C8012A
:10CD20000E94215745E050E06FEF7FEFC8010E945D
:10CD30003693C8010E94C55667E37AE0C8010E9495
:10CD4000295745E050E061EF7FEFC8010E949192C2
:10CD5000C8010E94C55664E67AE0C8010E942957BE
:10CD6000C8010E94C590C8010E94C55665E772E1DE
:10CD7000C8010E94215745E050E060E070E0C80122
:10CD80000E944990C8010E94C55665E772E181E89A
:10CD900092E10E94DC553FE14316510461047104A5
:10CDA00034F4C9A4DAA4EBA4FCA4F7FC10C061E835
:10CDB00072E1C8010E942157C8017AD3C8010E94BC
:10CDC000C55664E67AE081E892E10E949B56B20182
:10CDD000C30177FE04C069A97AA98BA99CA90E9406
:10CDE0000189A9C023E04DA15EA16FA178A5CE0164
:10CDF00043960E94CA566DE879E0C8010E942957FF
:10CE00006BE772E1C8010E94455669E37AE00E942F
:10CE10002E56BE016D5E7F4F0E94455662E17AE05C
:10CE20000E942E56BC018BE792E10E94B056C801C9
:10CE30000E94C556CE0143960E94C55649855A8523
:10CE40006B857C8523E0CE0149960E94CA564D81B0
:10CE50005E816F81788523E0C8010E94CA56B801BF
:10CE6000CE0143960E9421576EE37AE0CE014396AD
:10CE70000E942E56BE01675E7F4F0E94455662E1BA
:10CE80007AE00E942E56BC0185E792E10E94B056DE
:10CE9000CE0143960E94C556C8010E94C556CE01D8
:10CEA00049960E94C5562DE2421621E052066104C1
:10CEB000710474F469A57AA58BA59CA525E030E0E2
:10CEC00040E050E00E945AB2672B682B692BF1F4C6
:10CED0006BE772E1C8010E9421574AE050E06FEF12
:10CEE0007FEFC8010E943693C8010E94C55665E7CE
:10CEF00072E1C8010E9421574AE050E060E070E012
:10CF0000C8010E944990C8010E94C55661E872E1BB
:10CF1000C8010E942157C801CBD2C8010E94C55642
:10CF200064E67AE081E892E10E949B56C301B20177
:10CF30000E9401891DAA0E945D8A6B017C012296D4
:10CF40002CAD3DAD4EAD5FAD2297C21AD30AE40AB7
:10CF5000F50AC9A6DAA6EBA6FCA6C7CC6BE772E178
:10CF6000CE010D960E9421574AE050E06FEF7FEF0F
:10CF7000CE010D960E949192CE010D960E94C5564B
:10CF8000CDA8CC20B1F167E37AE0CE010D960E94E6
:10CF9000295745E050E061EF7FEFCE010D960E94EA
:10CFA0009192CE010D960E94C5568091D30C882394
:10CFB00091F060E371E1CE010D960E94195745E0B2
:10CFC00050E060E070E0CE010D960E949192CE019B
:10CFD0000D960E94C55664E67AE0CE010D960E9439
:10CFE0002957CE010D960E94C590CE010D960E9444
:10CFF000C55665E772E1CE010D960E9421574AE0C1
:10D0000050E06FEF7FEFCE010D960E944990CE0168
:10D010000D960E94C556CB5BDF4F0FB6F894DEBF6E
:10D020000FBECDBFDF91CF911F910F91FF90EF9079
:10D03000DF90CF90BF90AF909F908F907F906F9038
:10D040005F904F903F902F9008958F929F92AF9254
:10D05000BF92CF92DF92EF92FF920F931F93CF93E5
:10D06000DF938C01862F0B30110509F06FC0909172
:10D07000E212992309F0F89462E10E948F5B2091FB
:10D08000E212222309F07894009709F072C0E09030
:10D09000DD12F090DE126F2D70E080E090E00E94D3
:10D0A0002EB12DEC3CEC4CEC5DE30E948DB14B01BC
:10D0B0005C016E2D70E080E090E00E942EB19B013B
:10D0C000AC01C501B4010E94B8B26093D51270934F
:10D0D000D6128093D7129093D812C091DF12D091BC
:10D0E000E0126C2F6F7770E080E090E00E942EB12C
:10D0F0004B015C016D2F70E080E090E00E942EB14A
:10D100002DEC3CEC4CEC5DE30E948DB19B01AC013D
:10D11000C501B4010E94B8B2C7FD09C06093D9121D
:10D120007093DA128093DB129093DC120BC0DC0157
:10D13000CB01B0588093D9129093DA12A093DB12EE
:10D14000B093DC12FE0CCF0DCD0F71C0063111056E
:10D1500009F0B4C09091E212992309F0F89461E0CB
:10D160000E948F5B2091E212222309F078940097AD
:10D17000A9F040E050EC69E774EC4093D51250936D
:10D18000D6126093D7127093D8124093D91250934D
:10D19000DA126093DB127093DC1295C0F090DE120D
:10D1A000D091DD126091DD127091DE127627672733
:10D1B000762780E090E00E942CB12DEC3CEC4CEC0A
:10D1C0005DE30E948DB16093D5127093D612809367
:10D1D000D7129093D812E090E012C091DF128C2FFA
:10D1E0008F776E2D70E0782B80E090E00E942CB15C
:10D1F0002DEC3CEC4CEC5DE30E948DB1C7FD09C009
:10D200006093D9127093DA128093DB129093DC1240
:10D210000BC0DC01CB01B0588093D9129093DA1285
:10D22000A093DB12B093DC12DF0DED0ECE0D8091DA
:10D23000E112C81346C0C090D512D090D612E0902B
:10D24000D712F090D81220E030E048EC52E4C70149
:10D25000B6010E946DB418161CF0C0E0D0E002C008
:10D26000CBEFDFEF20E030E0A901C701B6010E945B
:10D2700028B187FF02C0CAEFDFEFC090D912D0906B
:10D28000DA12E090DB12F090DC1220E030E048ECA3
:10D2900052ECC701B6010E9428B187FF02C0C9EF56
:10D2A000DFEF20E030E040EF52E4C701B6010E941A
:10D2B0006DB41816ACF4C8EFDFEF12C0CFEFDFEF9C
:10D2C0000FC08FEF9FEF8F3FFFEF9F0709F4D3C091
:10D2D000009709F4B0CF029609F4D9C0CCEFDFEF84
:10D2E0000C30110509F0D6C08CE5ACD680E090E09A
:10D2F000A4D6A1D665E08CE50E94855BC82FD0E05E
:10D300002097A1F0C530D105A4F008EE1CE08EE016
:10D3100090E10E941D7DF80180870F5F1F4FC801BB
:10D32000885E9C408C179D0794F306C0CEEFDFEF1C
:10D33000B1C0CDEFDFEFAEC0C091F00C0091F10CA9
:10D34000602F70E080E090E00E942EB12DEC3CEC6C
:10D350004CEC5DE30E948DB16B017C016C2F70E0A1
:10D3600080E090E00E942EB19B01AC01C701B601A4
:10D370000E94B8B26093E80C7093E90C8093EA0CB9
:10D380009093EB0CD091F20C1091F30C6D2F6F7702
:10D3900070E080E090E00E942EB16B017C01612F73
:10D3A00070E080E090E00E942EB12DEC3CEC4CEC63
:10D3B0005DE30E948DB19B01AC01C701B6010E94E3
:10D3C000B8B2D7FF5BC0DC01CB01B0588093EC0C46
:10D3D0009093ED0CA093EE0CB093EF0C8C2F800F7C
:10D3E000C82FCD0FC10F8091F40CC81344C0C0905A
:10D3F000E80CD090E90CE090EA0CF090EB0C20E007
:10D4000030E048EC52E4C701B6010E946DB4181632
:10D410001CF0C0E0D0E002C0CBEFDFEF20E030E056
:10D4200040EA50E4C701B6010E9428B187FF02C05C
:10D43000CAEFDFEFC090EC0CD090ED0CE090EE0C5A
:10D44000F090EF0C20E030E040EF51ECC701B60166
:10D450000E9428B187FF02C0C9EFDFEF20E030E073
:10D4600040EF52E4C701B6010E946DB4181694F45F
:10D47000C8EFDFEF0FC0CFEFDFEF0CC06093EC0C15
:10D480007093ED0C8093EE0C9093EF0CA7CFCEEF42
:10D49000DFEF26CFCE01DF91CF911F910F91FF904B
:10D4A000EF90DF90CF90BF90AF909F908F900895B6
:10D4B000CF93DF93FC0124813581232B89F0EC018C
:10D4C000BC018AE99DE04AD56EE170E080E090E021
:10D4D0000E940189BE0181E79FE0DF91CF913EC5A7
:10D4E000DF91CF910895CF92DF92EF92FF92CF9389
:10D4F000C0911B11C43014F5C1300CF04DC0C111E6
:10D5000079C00E942477BC01990F880B990B0E9467
:10D510002EB120E030E040EA50E40E948DB120E0DE
:10D5200030EC4FE754E40E947EB320911C113091FF
:10D530001D1140911E1150911F1159C0C43009F0A6
:10D5400059C00E942477BC01990F880B990B0E9447
:10D550002EB120E030E040EA50E40E948DB120E09E
:10D5600030EC4FE754E40E947EB320E030E040EA24
:10D5700050E40E947EB320E030E040E851E40E9495
:10D580008DB120E030E040E850E40E94B8B220E0E5
:10D5900030E04AE754E42BC00E942477BC01990F85
:10D5A000880B990B0E942EB12AE137E64CE950E432
:10D5B0000E948DB120911C1130911D1140911E11BE
:10D5C00050911F110E94B7B26B017C01EC2FEE0F3E
:10D5D000FF0BE55CFA4F60817181072E000C880B10
:10D5E000990B0E942EB19B01AC01C701B6010E94AC
:10D5F0007EB303C060E070E0CB01CF91FF90EF906D
:10D60000DF90CF9008958F929F92AF92BF92CF926A
:10D61000DF92EF92FF92CF93DF93CDB7DEB72C97D7
:10D620000FB6F894DEBF0FBECDBF66E472E1CE0147
:10D6300001960E9419574CE251E06FEF7FEFCE0147
:10D6400001960E944990CE0101960E94C5566091B4
:10D65000B7027091B8028091290290912A02F5DCFC
:10D6600084E1882E912CA12CB12CE12CF12C2FEFF0
:10D67000E21AF20AC501B4010E9401896091B70261
:10D680007091B8028091290290912A02DEDC23E099
:10D69000E216F10434F02AE0E216F10444F4892B96
:10D6A00049F084E1880E911CA11CB11CE0CF892BAC
:10D6B00009F089C18091290290912A028B3091054D
:10D6C000C9F48091D9129091DA12A091DB12B09135
:10D6D000DC128093F90C9093FA0CA093FB0CB0939E
:10D6E000FC0C8091D5129091D612A091D712B091D6
:10D6F000D8121DC08631910521F30C9701F5809158
:10D70000EC0C9091ED0CA091EE0CB091EF0C80938D
:10D71000F90C9093FA0CA093FB0CB093FC0C809145
:10D72000E80C9091E90CA091EA0CB091EB0C80937D
:10D73000F50C9093F60CA093F70CB093F80C409175
:10D74000F90C5091FA0C6091FB0C7091FC0C21E0EB
:10D75000CE0107960E94CA5662EA7AE0CE0101968F
:10D760000E942957BE01695F7F4FCE0101960E943A
:10D770004556BC0181E892E10E94B056CE01019667
:10D780000E94C556CE0107960E94C5564091F50CE1
:10D790005091F60C6091F70C7091F80C21E0CE01DD
:10D7A00007960E94CA5665E476E0CE0101960E9473
:10D7B0002957BE01695F7F4FCE0101960E944556F1
:10D7C000BC0181E892E10E94DC55CE0101960E94E5
:10D7D000C556CE0107960E94C55667E076E081E8FF
:10D7E00092E10E94CE5564E67AE0CE0101960E9455
:10D7F000295744E150E060E070E0CE0101960E94BC
:10D800009192CE0101960E94C556C090F90CD0901D
:10D81000FA0CE090FB0CF090FC0C20E030E0A90149
:10D82000C701B6010E946DB420E030E040E05FE344
:10D8300087FD05C0C701B6010E94B8B204C0C70188
:10D84000B6010E94B7B20E9417B4AB01BC01CE0171
:10D8500001963ED4BE016F5F7F4F8BE792E10E943D
:10D86000E255CE0101960E94C55660E087E005D4DE
:10D870006BE772E18CE793E10E9487576FED8CE7CD
:10D8800093E10E9480576BE476E08CE793E10E947D
:10D8900060586091F50C7091F60C8091F70C9091A6
:10D8A000F80C0E9417B44AE050E08CE793E10E9424
:10D8B000165867E076E08CE793E10E94605864E6D2
:10D8C00070E080E090E00E940189C090F90CD09057
:10D8D000FA0CE090FB0CF090FC0C20E030E040EF04
:10D8E00051E4C701B6010E946DB487FD03C067E330
:10D8F00072E154C020E030E040ED51E4C701B601D0
:10D900000E946DB487FD1FC067E272E1CE010196EF
:10D910000E9419574AE050E06FEF7FEFCE01019669
:10D920000E944990CE0101960E94C55680914702FF
:10D93000882331F06CED75E080E090E00E94018971
:10D9400067E172E12BC020E030E040EB51E4C70119
:10D95000B6010E946DB487FD03C069E072E11EC08C
:10D960006AEF71E1CE0101960E9419574AE050E03A
:10D970006FEF7FEFCE0101960E944990CE01019694
:10D980000E94C55680914702882331F06CED75E006
:10D9900080E090E00E9401896CEE71E1CE01019679
:10D9A0000E9419574AE050E06FEF7FEFCE010196D9
:10D9B0000E944990CE0101960E94C55662E370E034
:10D9C00080E090E0DCC00E94A1416EE170E080E068
:10D9D00090E00E9401890E94709A6B017C0164E6CC
:10D9E00070E080E090E00E94018962EA7AE081E8DC
:10D9F00092E10E949B5621E0B701A601CE0101965B
:10DA00000E94CA56BE016F5F7F4F81E892E10E947B
:10DA1000DC55CE0101960E94C55661E872E1CE0147
:10DA200001960E9421574AE050E060E070E0CE018C
:10DA300001960E949192CE0101960E94C556809156
:10DA40002E05882379F080912D05882359F06FEDFC
:10DA50008CE793E10E9480576AE07AE08CE793E1DB
:10DA60000E94605869E07AE081E892E10E94CE5518
:10DA7000C092F90CD092FA0CE092FB0CF092FC0CE4
:10DA800020E030E040EF51E4C701B6010E946DB4E0
:10DA900087FD03C06CED71E154C020E030E040ED43
:10DAA00051E4C701B6010E946DB487FD1FC06CEC44
:10DAB00071E1CE0101960E9419574AE050E06FEFE4
:10DAC0007FEFCE0101960E944990CE0101960E94FF
:10DAD000C55680914702882331F06CED75E080E0F7
:10DAE00090E00E9401896CEB71E12BC020E030E0F6
:10DAF00040EB51E4C701B6010E946DB487FD03C03D
:10DB00006EEA71E11EC06FE971E1CE0101960E94DB
:10DB100019574AE050E06FEF7FEFCE0101960E9467
:10DB20004990CE0101960E94C556809147028823F4
:10DB300031F06CED75E080E090E00E94018961E9D0
:10DB400071E1CE0101960E9419574AE050E06FEF53
:10DB50007FEFCE0101960E944990CE0101960E946E
:10DB6000C5566CE271E080E090E00E9401898091EE
:10DB70004702882331F068EE73E080E090E00E9475
:10DB800001892C960FB6F894DEBF0FBECDBFDF9192
:10DB9000CF91FF90EF90DF90CF90BF90AF909F908C
:10DBA0008F900895DF92EF92FF920F931F93CF9380
:10DBB000DF93CDB7DEB762970FB6F894DEBF0FBE26
:10DBC000CDBF8C011092FD0C64E67AE0CE010D967B
:10DBD0000E942957FF24F39481E79FE00E947F521F
:10DBE0002091FD0C18161906DCF5211139C081E7CA
:10DBF0009FE00E945D528A3041F08D3031F0682FF5
:10DC0000CE010D960E94BB5524C089899A89892B23
:10DC100001F1F092FD0C61E47AE0CE0101960E94E0
:10DC20002957BE01635F7F4FCE0101960E94455682
:10DC3000BC01CE0107960E942157CE0107960E9493
:10DC40006592CE0107960E94C556CE0101960E94AC
:10DC5000C5566AE070E080E090E00E940189BCCF88
:10DC6000211184C0E12CF12CDD24D3948AE99DE0BC
:10DC70000E947F521816190614F58AE99DE00E9449
:10DC80005D528A3079F08D3069F09091FD0C9111E0
:10DC900009C0682FCE010D960E94BB558FEFE81A80
:10DCA000F80A06C089899A89892B11F0D092FD0C57
:10DCB00065E070E080E090E00E940189D7CF64E1E8
:10DCC00070E080E090E00E940189EF28C9F1898925
:10DCD0009A89892BA9F180911F14882359F16FE942
:10DCE00079E0CE0101960E942957BE016F5F7F4FF8
:10DCF000CE010D960E94F187F82ECE0101960E946A
:10DD0000C556F11017C06AE47AE081E79FE00E94EF
:10DD10006058BE01635F7F4FCE0101960E9421577C
:10DD2000BE016F5F7F4F81E79FE018D1CE01019662
:10DD30000E94C55664E170E080E090E00E94018995
:10DD40008091FD0C811112C089899A89892B71F407
:10DD500064E670E080E090E00E9401890E945D8AA4
:10DD600064E67AE0C8010E94295751C089899A89DE
:10DD7000019709F046C06EED75E0CE0107960E944E
:10DD80002957BE01695F7F4FCE010D960E94F18732
:10DD9000811116C06CE877E0CE0101960E942957E8
:10DDA000BE016F5F7F4FCE010D960E94F187FF2469
:10DDB000F3948111F12CCE0101960E94C55601C049
:10DDC000F12CCE0107960E94C556FF20A1F040E03D
:10DDD00050E0BE01635F7F4FCE0101960E94EC418F
:10DDE000BE016F5F7F4F8DE892E10E94E255CE0148
:10DDF00001960E94C55664E170E080E090E00E94C8
:10DE00000189BE01635F7F4FC8010E941157CE0197
:10DE10000D960E94C556C80162960FB6F894DEBFF3
:10DE20000FBECDBFDF91CF911F910F91FF90EF906B
:10DE3000DF900895DF92EF92FF920F931F93CF939D
:10DE4000DF93CDB7DEB72C970FB6F894DEBF0FBEC9
:10DE5000CDBF8C011092FD0C64E67AE0CE010796EE
:10DE60000E942957E12CF12CDD24D3948AE99DE00E
:10DE70000E947F521816190614F58091FD0C81112D
:10DE80001EC08AE99DE00E945D528A3059F08D30B3
:10DE900049F0682FCE0107960E94BB558FEFE81A14
:10DEA000F80A06C08B859C85892B11F0D092FD0C59
:10DEB0006FE070E080E090E00E940189D7CF62E3DC
:10DEC00070E080E090E00E940189EF2851F08AE93B
:10DED0009DE00E941D5364E670E080E090E00E94A7
:10DEE00001898091FD0C81110AC08B859C85892B4D
:10DEF00031F464E67AE0C8010E94295718C0809185
:10DF00001F14882371F0BE01695F7F4FCE01019617
:10DF10000E942157CE010196CBDACE0101960E94D4
:10DF2000C556BE01695F7F4FC8010E941157CE01DF
:10DF300007960E94C556C8012C960FB6F894DEBF0E
:10DF40000FBECDBFDF91CF911F910F91FF90EF904A
:10DF5000DF90089562E67AE00C94B9570F931F930F
:10DF6000CF93DF93EC010E9487578C01CE01F2DF43
:10DF7000800F911FDF91CF911F910F910895282F4E
:10DF80003091990D313208F04AC08091760D81119F
:10DF9000FCCF9091881342E04093760D2093750D4D
:10DFA0002FEF2093740D1092730D3093720DE9E7EB
:10DFB000FDE0A2E5BDE020E0321721F041914D9354
:10DFC0002F5FFACF1092510D2091510D990F922B86
:10DFD0009093510D9091500D913061F41092500D2D
:10DFE0009091510D9093BB009091BC0093FDF8CFA0
:10DFF00095EC01C095EE9093BC009091760D923017
:10E00000E1F39091740D9F3F79F08091740D80320F
:10E0100041F08091740D803331F084E005C081E0DF
:10E0200003C082E001C083E01092780D1092990D38
:10E030001092770D089581E0A2CF682F8EE090E1D5
:10E040000C94657D91E09093770D809388131092E6
:10E05000780D1092990D0895CF93C82F682F607F87
:10E060008CE793E10E94937E80E1C89FB001112468
:10E070008CE793E1CF910C94937ECF93DF93CDB750
:10E08000DEB728970FB6F894DEBF0FBECDBF98E07D
:10E09000E3E4F5E0DE01119601900D929A95E1F727
:10E0A00090918513961710F46FEF690FFE0131966A
:10E0B000E60FF11DE60FF11D9081890F806828960B
:10E0C0000FB6F894DEBF0FBECDBFDF91CF91C4CFA6
:10E0D0000F931F93CF93DF93CDB7DEB7A2970FB601
:10E0E000F894DEBF0FBECDBF8C01CB01BA01F801A1
:10E0F0001182108213821282158214822AE0AE01EC
:10E100004F5F5F4F0E94FAACBE016F5F7F4FC80147
:10E110000E949B56A2960FB6F894DEBF0FBECDBFED
:10E12000DF91CF911F910F9108950F931F93CF937C
:10E13000DF93EC010E94B9578C01CE010BDF800FF9
:10E14000911FDF91CF911F910F910895CF92DF9290
:10E15000EF92FF92CF93DF936B017C0197FF15C085
:10E160006DE281E79FE00E948057EC01442755272C
:10E17000BA014C195D096E097F092AE081E79FE029
:10E180000E94CE57C80FD91F08C02AE0AB01BC01BE
:10E1900081E79FE00E94CE57EC0181E79FE0DADE45
:10E1A0008C0F9D1FDF91CF91FF90EF90DF90CF906C
:10E1B00008958F929F92AF92BF92CF92DF92EF928B
:10E1C000FF920F931F93CF93DF936B017C01142F6A
:10E1D0009B01AC010E94B7B5882319F065E67AE08F
:10E1E00027C046015701E894B7F82FEF3FEF4FE7FC
:10E1F0005FE7C501B4010E94B7B581110DC02FEFD3
:10E200003FEF4FE75FE7C501B4010E9428B1181640
:10E210001CF469E67AE00CC02FEF3FEF4FE75FE4B4
:10E22000C701B6010E946DB4181694F46DE67AE049
:10E2300081E79FE0DF91CF911F910F91FF90EF90C9
:10E24000DF90CF90BF90AF909F908F900C94B95774
:10E250002FEF3FEF4FE75FECC701B6010E9428B1F7
:10E2600087FDE4CF20E030E0A901C701B6010E949C
:10E2700028B187FF0BC06DE281E79FE00E948057C5
:10E28000EC01F7FAF094F7F8F09402C0C0E0D0E0A7
:10E2900000E060E070E080E09FE3101741F020E0D4
:10E2A00030E040E251E40E947EB30F5FF6CFA70159
:10E2B00096010E94B8B26B017C010E941CB44B0114
:10E2C0005C012AE0AB01BC0181E79FE00E94CE57D0
:10E2D000C80FD91F1123C9F1C501B4010E942CB187
:10E2E0009B01AC01C701B6010E94B7B26B017C0172
:10E2F0006EE281E79FE00E948057C80FD91F20E09F
:10E3000030E040E251E4C701B6010E948DB14B01FB
:10E310005C010E941CB46B01E12CF12C2AE0B701D6
:10E32000A60181E79FE00E94CE57C80FD91FC70101
:10E33000B6010E942CB19B01AC01C501B4010E9441
:10E34000B7B26B017C011150D1F6CE01DF91CF91B4
:10E350001F910F91FF90EF90DF90CF90BF90AF9003
:10E360009F908F9008952F923F924F925F926F925D
:10E370007F928F929F92AF92BF92CF92DF92EF9255
:10E38000FF920F931F93CF93DF93CDB7DEB72897FC
:10E390000FB6F894DEBF0FBECDBFC090000DD09079
:10E3A000010D4091020D5091030DC416D5062CF4B9
:10E3B0003C2D2D2D6A01432F522FE4E0FDE060E05B
:10E3C00070E0CB01019111910417150754F44A0133
:10E3D000550FAA08BB08680D791D8A1D9B1DA80151
:10E3E00015C0C016D10654F40D2C000CEE08FF0821
:10E3F0006C0D7D1D8E1D9F1D680108C0012E000C37
:10E40000220B330B600F711F821F931F2DE0E0352D
:10E41000F207C1F60E942EB120E030E048E152E45C
:10E420000E947EB38B0188879F8380E0E82E8DE079
:10E43000F82E812C912C5401D7016D917D917D0195
:10E44000072E000C880B990B0E942EB1980148856D
:10E450005F810E94B7B29B01AC010E948DB19B010C
:10E46000AC01C501B4010E94B8B24B015C01E0E50A
:10E47000FDE0EE15FF0501F720E030E04CE152E44D
:10E480000E947EB30E9476B56B017C0120E030E0F3
:10E4900040E85FE30E946DB418160CF069C020E0FC
:10E4A0003DE03A832983212C312C412C512C32011F
:10E4B000A981BA818D919D91BA83A9839C01990FFD
:10E4C000440B550B2B833C834D835E83CA01B901FA
:10E4D0000E942EB1980148855F810E94B7B24B011E
:10E4E0005C0120E030E0A9010E946DB4181624F010
:10E4F000B7FAB094B7F8B094A7019601C501B4017A
:10E500000E9428B187FF0BC08B819C81AD81BE81A9
:10E51000480E591E6A1E7B1E9FEF291A390AA0E574
:10E52000BDE0E981FA81AE17BF0711F620E030E0C7
:10E5300040EC5FE3C701B6010E948DB16B017C0125
:10E54000F5E02F1631040CF4AACFC301B2010E94EA
:10E550002EB16B017C01B101330C880B990B0E9429
:10E560002EB19B01AC01C701B6010E947EB303C06E
:10E57000B80188859F816B017C01C701B60128968F
:10E580000FB6F894DEBF0FBECDBFDF91CF911F91C4
:10E590000F91FF90EF90DF90CF90BF90AF909F9042
:10E5A0008F907F906F905F904F903F902F90089545
:10E5B0004F925F926F927F928F929F92AF92BF9293
:10E5C000CF92DF92EF92FF921F93CF93DF93CDB75D
:10E5D000DEB728970FB6F894DEBF0FBECDBF4B0154
:10E5E0005C0111E0612E712C9301220F331F220F69
:10E5F000331F3A832983F901ED57FD4FC080D18045
:10E60000E280F380A5019401C701B6010E9428B100
:10E6100087FF02C01F5FE6CFA5019401C701B601C5
:10E620000E9428B149815A8145595D4F5E834D83CF
:10E63000811106C0FA0160817181828193814DC090
:10E64000F1E06F1AF0EC7F0AC301880F991F880F61
:10E65000991FFC01ED57FD4F20813181428153818B
:10E6600029833A834B835C83FC01E559FD4F40804D
:10E67000518062807380A3019201ED81FE816081EF
:10E680007181828193810E94B7B26D837E838F8373
:10E69000988729813A814B815C81C501B4010E9430
:10E6A000B7B29B01AC016D817E818F8198850E94FC
:10E6B0008DB14B015C0129813A814B815C81C7019D
:10E6C000B6010E94B7B29B01AC01C501B4010E9422
:10E6D0007EB3A30192010E94B8B228960FB6F894B7
:10E6E000DEBF0FBECDBFDF91CF911F91FF90EF90A6
:10E6F000DF90CF90BF90AF909F908F907F906F9062
:10E700005F904F9008950F931F930E945D8A6093CE
:10E710003F0E7093400E8093410E9093420E87E31C
:10E720009EE00E945D5297FF1FC00E945D8A00918B
:10E730003F0E1091400E2091410E3091420EDC01AF
:10E74000CB01801B910BA20BB30B00913B0E1091E0
:10E750003C0E20913D0E30913E0E80179107A2078E
:10E76000B307E8F28FEF9FEF1F910F910895CF92BB
:10E77000DF92EF92FF92CF93DF93EC016A017B016E
:10E78000E889F98982E080834115514E6105710560
:10E79000B1F060E079E08DE390E0A70196010E947E
:10E7A00086B2DA01C9010197A109B109B695A79509
:10E7B000979587959C01211580E13807A8F0E88995
:10E7C000F989108260E874E88EE190E0A701960173
:10E7D0000E9486B2DA01C9010197A109B109B69573
:10E7E000A795979587959C01EC85FD853083EE85EF
:10E7F000FF852083188EEC89FD8986E08083EA8975
:10E80000FB89808180618083EA89FB8980818860BF
:10E810008083EA89FB89808180688083EA89FB891B
:10E8200080818F7D8083DF91CF91FF90EF90DF908B
:10E83000CF9008950F931F93CF93DF931F921F9252
:10E84000CDB7DEB70EEF1CE0F80160818EED93E0EE
:10E850009A838983CE0101960E94D341F801618198
:10E860008FED93E09A838983CE0101960E94D34174
:10E87000C8010F900F90DF91CF911F910F910895D4
:10E88000EF92FF920F931F93CF93DF931F921F92EC
:10E89000CDB7DEB70BE711E18B5791417C01C70182
:10E8A000800F911FF80161918F019A838983CE01B6
:10E8B00001960E94D341F1E105381F0781F78BE7EC
:10E8C00091E10F900F90DF91CF911F910F91FF90E9
:10E8D000EF900895EF92FF920F931F93CF93DF93E2
:10E8E0001F921F92CDB7DEB70CEE10E18C5E904107
:10E8F0007C01C701800F911FF80161918F019A83FC
:10E900008983CE0101960E94D341F1E102371F07AE
:10E9100081F78CEE90E10F900F90DF91CF911F91D6
:10E920000F91FF90EF900895EF92FF920F931F9336
:10E93000CF93DF931F921F92CDB7DEB70BE711E1A4
:10E940008B5791417C01C701800F911FF8016191A4
:10E950008F019A838983CE0101960E94D341F2E10F
:10E9600005371F0781F78BE791E10F900F90DF913B
:10E97000CF911F910F91FF90EF90089581E08093C8
:10E980002D0580912E05882341F088E08093871320
:10E9900060E08CE793E10C94807E089580912E05D1
:10E9A00081110EC081E080932E0580932D0580910A
:10E9B0008213982F9460909382138C604DDB17C064
:10E9C00080912D05882399F01092871360E08CE7E1
:10E9D00093E10E94807E10922D05809182138B7F9F
:10E9E00080938213886038DB10922E050895C6CF7D
:10E9F0002F923F924F925F926F927F928F929F924F
:10EA0000AF92BF92CF92DF92EF92FF920F931F933C
:10EA1000CF93DF93CDB7DEB766970FB6F894DEBF1E
:10EA20000FBECDBF1C0184ED9EE00E94E39040E844
:10EA300055E260E070E084ED9EE099DE64E670E00F
:10EA400080E090E00E9401898CED95E0A0E0B0E0CC
:10EA50008093D80E9093D90EA093DA0EB093DB0E6C
:10EA600064E670E080E090E00E9401898FEF8A8781
:10EA700081E08B8786E88C871D861E861F86188A14
:10EA8000198A89E78A8BC101880F991F9E8B8D8B0C
:10EA9000C12CD12CE12CF12C412C512C320184EDD4
:10EAA0009EE0E214F3046CF5ED89FE89CE16DF06D4
:10EAB00044F50E944E5208974CF049E050E0BE01E8
:10EAC000665F7F4F84ED9EE00E94245265E070E017
:10EAD00080E090E00E94018900E010E0812C912C00
:10EAE000540184ED9EE00E947F52892B31F4F4E0C2
:10EAF0008F169104A104B104ACF50230110594F510
:10EB000035C00E94E390E114F10409F47101C301DE
:10EB1000B2010E942EB14B015C01B701FF0C880BC2
:10EB2000990B0E942EB19B01AC01C501B4010E945A
:10EB30007EB366960FB6F894DEBF0FBECDBFDF91F1
:10EB4000CF911F910F91FF90EF90DF90CF90BF90EA
:10EB5000AF909F908F907F906F905F904F903F907D
:10EB60002F9008958FEFC81AD80A99CF84ED9EE0B0
:10EB70000E947F52892B69F084ED9EE00E945D52D5
:10EB8000E1E0F0E0EC0FFD1FE00FF11F80830F5F6D
:10EB90001F4F65E070E080E090E00E940189023044
:10EBA000110569F599818A85981329C09A818C8508
:10EBB000981325C0CE0103969C8B8B8B84ED9EE031
:10EBC0000E947F52892B31F494E089169104A104AC
:10EBD000B1043CF509301105C1F48B8190E0982F08
:10EBE00088272C81820F911D092E000CAA0BBB0BCC
:10EBF000480E591E6A1E7B1EEFEFEE1AFE0AFFEF4B
:10EC00008F1A9F0AAF0ABF0A6CCF84ED9EE00E9464
:10EC10005D52EB89FC898193FC8BEB8B0F5F1F4F5F
:10EC2000CDCF0430110544F3D8CF2F923F924F92AD
:10EC30005F926F927F928F929F92AF92BF92CF928C
:10EC4000DF92EF92FF920F931F93CF93DF936C01AC
:10EC5000CFEAD5E089E0882E82E0982E0CEE10E114
:10EC6000EE24E394F12C22E1222E312C33E1432EC9
:10EC7000512C40E1642E712C51E1A52EB12C8091D4
:10EC80000702909108028E159F050CF4CAC021E07E
:10EC9000C216D10439F4F80182AD93ADF401918329
:10ECA00080830AC0F2E0CF16D10431F4F4018081F0
:10ECB0009181F80193AF82AFF40180819181009737
:10ECC00039F48A819B819093BA028093B90222C061
:10ECD0008130910539F48A819B819093B8028093A9
:10ECE000B70218C08230910539F48A819B819093D4
:10ECF000B6028093B5020EC0039761F48A819B81AE
:10ED00009093B4028093B30264E67AE08FEC92E1D0
:10ED10000E949B56F401819191914F01843091059D
:10ED200039F42A813B81309362022093610212C040
:10ED30008530910539F42A813B8130935A02209322
:10ED4000590208C086309105C9F00EC08A3091057D
:10ED500009F448C08531910589F42A813B813093BB
:10ED60005E0220935D023EC08730910579F72A81CB
:10ED70003B813093600220935F020AC08631910587
:10ED800039F42A813B8130935C0220935B022AC0D4
:10ED90008731910539F52A813B812830310549F4C5
:10EDA0007092030260920202B0920102A0920002ED
:10EDB00019C02730310549F4309203022092020233
:10EDC00050920102409200020DC02630310551F4EC
:10EDD00021E030E0309303022093020210920102FE
:10EDE000109200029C012B5031092A30310590F419
:10EDF0002A813B813093B4022093B30239E1389FDA
:10EE0000B001399F700D112465547D4F8FEC92E154
:10EE10000E949B568FEFE81AF80A22960E5F1F4F4A
:10EE20002ECFDF91CF911F910F91FF90EF90DF9048
:10EE3000CF90BF90AF909F908F907F906F905F909A
:10EE40004F903F902F9008957F928F929F92AF9214
:10EE5000BF92CF92DF92EF92FF920F931F93CF93C7
:10EE6000DF93782E8AE0A82EB12CEE24EA9493E06A
:10EE7000F92E88248A9423E0922E00E010E0C12C21
:10EE8000D12CC0E0D0E0872D0E94B788C816D906E3
:10EE900028F00817190718F48C0101C06C018815B7
:10EEA000990528F08E159F0518F47C0101C04C01CE
:10EEB000C80FD91F65E070E080E090E00E940189F2
:10EEC00081E0A81AB108F9F60C0D1D1DCE01801BBA
:10EED000910B8E199F098819990966E070E00E94CC
:10EEE000DFB5CB01DF91CF911F910F91FF90EF9094
:10EEF000DF90CF90BF90AF909F908F907F900895BC
:10EF00004F925F926F927F92AF92BF92CF92DF92B9
:10EF1000FF920F931F93CF93DF9300D000D0CDB714
:10EF2000DEB75C0184ED9EE00E94E39040E052EC8D
:10EF300061E070E084ED9EE01ADC8CED95E0A0E0ED
:10EF4000B0E08093D80E9093D90EA093DA0EB093D0
:10EF5000DB0E64E670E080E090E00E940189C12C45
:10EF6000D12CF12CCA14DB040CF051C065E070E028
:10EF700080E090E00E94018900E010E0412C512CDB
:10EF80003201F1100FC084ED9EE00E947F52892B68
:10EF900031F485E148165104610471041CF4033016
:10EFA000110554F08FEFC81AD80A64E670E080E0CB
:10EFB00090E00E940189D6CF84ED9EE00E947F52AE
:10EFC000892B69F084ED9EE00E945D52E1E0F0E063
:10EFD000EC0FFD1FE00FF11F80830F5F1F4F65E0F7
:10EFE00070E080E090E00E940189023011054CF051
:10EFF00089818B3B31F4FF24F3948A818A3A09F0AA
:10F00000F12C8FEF481A580A680A780ABACF8F2D68
:10F0100026960FB6F894DEBF0FBECDBFDF91CF911D
:10F020001F910F91FF90DF90CF90BF90AF907F9096
:10F030006F905F904F9008951F93CF93DF93182F99
:10F04000C0E0DDE0812F0E94B788899399936CE33B
:10F0500070E080E090E00E9401898DE0C035D80723
:10F0600089F781D920E030E040EA50E40E948DB178
:10F0700020E030E040E85AE30E948DB1DF91CF916B
:10F080001F9108954F925F926F927F928F929F92FD
:10F09000AF92BF92CF92DF92EF92FF92CF93DF9326
:10F0A000CDB7DEB768970FB6F894DEBF0FBECDBF01
:10F0B0006B017C010E945D8A698B7A8B8B8B9C8BA8
:10F0C00087E39EE00E94E39061E0809102020E944B
:10F0D0007B8860E0809100020E947B880E94709A89
:10F0E0000E94D04A0E94ED4A6D877E878F87988B59
:10F0F0000E94DC884B015C016AE070E080E090E0F7
:10F100000E94018961E77AE081E892E10E949B56C2
:10F1100020E030E04AE754E4C701B6010E948DB117
:10F120006D8B7E8B8F8B988F412C512C3201C12C93
:10F13000D12C7601C701B6010E942EB12D893E89DE
:10F140004F89588D0E9428B187FF85C10E945D8A32
:10F1500029893A894B895C89621B730B840B950B57
:10F160000E942CB120E030E04AE754E40E947EB3D4
:10F17000AB01BC0123E0CE0101960E94CA56BE013C
:10F180006F5F7F4F8BE792E10E94E255CE010196BF
:10F190000E94C5560E94ED4A6B017C010E94DC88EA
:10F1A0009B01AC01281939094A095B0949015A0137
:10F1B00031ED831637E09306A104B1040CF441C08D
:10F1C00020E030E0A901C701B6010E946DB4181615
:10F1D0005CF426EA3BE944EC5BE3C701B6010E941C
:10F1E00028B187FF0BC02DC026EA3BE944EC5BEB5E
:10F1F000C701B6010E946DB418161CF1C501B40117
:10F2000028EE33E040E050E00E945AB2CA01B90152
:10F210000E942EB14B015C012D853E854F8558899A
:10F22000C701B6010E94B7B220E030E04AE754E4DB
:10F230000E948DB1A50194010E947EB34B015C0137
:10F2400003C0812C912C54016BE772E1CE01019631
:10F250000E9421576EED75E0CE0101960E942E5658
:10F26000BC018BE792E10E94B056CE0101960E944C
:10F27000C55623E0B701A601CE0101960E94CA56E9
:10F28000BE016F5F7F4FCE0107960E9421576CE54C
:10F2900079E0CE0107960E942E56BC0185E792E1E7
:10F2A0000E94B056CE0107960E94C556CE01019627
:10F2B0000E94C55622E0B501A401CE0107960E9426
:10F2C000CA566DE879E0CE0101960E9429576BE796
:10F2D00072E1CE0101960E9445566FE87AE00E94E5
:10F2E0002E5665E772E10E94455661EE75E00E9478
:10F2F0002E56BE01695F7F4F0E9445566CED75E04A
:10F300000E942E56BC0181E892E10E94DC55CE019C
:10F3100001960E94C556CE0107960E94C55620E070
:10F3200030E0A901C501B4010E946DB487FD06C09B
:10F3300066E67CE085E792E10E94CE5522E0B501C9
:10F34000A401CE0101960E94CA56BE016F5F7F4F95
:10F35000CE0107960E9421576CED75E0CE0107960D
:10F360000E942E56BC0185E792E10E94DC55CE0139
:10F3700007960E94C556CE0101960E94C55661E8C7
:10F3800072E1CE0101960E942157CE0101960E94A2
:10F39000586ACE0101960E94C556C301B20125E00C
:10F3A00030E040E050E00E945AB2672B682B692B96
:10F3B00021F56CE772E1CE0101960E94195745E0F4
:10F3C00050E060E070E0CE0101960E949192CE0183
:10F3D00001960E94C55665E772E1CE0101960E9432
:10F3E000215745E050E06FEF7FEFCE0101960E947C
:10F3F0004990CE0101960E94C55664E67AE081E804
:10F4000092E10E949B5665E070E080E090E00E94EF
:10F4100001890E945D8A6B017C0129893A894B89A7
:10F420005C89C21AD30AE40AF50A0E94ED4A6D8784
:10F430007E878F87988B0E94DC884B015C016AE095
:10F4400070E080E090E00E9401893FEF431A530A88
:10F45000630A730A6FCE60E0809102020E947B888B
:10F4600068960FB6F894DEBF0FBECDBFDF91CF9187
:10F47000FF90EF90DF90CF90BF90AF909F908F90D4
:10F480007F906F905F904F9008954F925F926F9230
:10F490007F92AF92BF92CF92DF92EF92FF920F9343
:10F4A0001F93CF93DF93CDB7DEB7EA970FB6F894EB
:10F4B000DEBF0FBECDBFF82E64E67AE0CE01C59662
:10F4C0000E9429578E010B5E1F4F6F2DC801EDD38F
:10F4D00018870F831D821E82198289E08A8381E04A
:10F4E0008B838C831C8A1B8ACE0101960E94325F1B
:10F4F000CE0101960E94C25ECE0101960E94EB5D94
:10F500000E8110E00330110509F46EC162E772E16B
:10F51000CE01C5960E94565664E67AE081E892E1F3
:10F520000E949B56BE016B5C7F4FCE0183960E946A
:10F5300021574AE050E060E070E0CE0183960E94DF
:10F540009192CE0183960E94C55661E080E00E94B0
:10F550003D7062EA7AE0CE01C5960E949B568FE923
:10F56000A82E8CE0B82ECC24C394D12CE12CF12C05
:10F57000E016F1060CF0EEC06E2DCE0101960E9451
:10F580007C5DF50121913191419151915F010E9482
:10F59000B8B22B013C0120E030E04CEF52EC0E946D
:10F5A00028B187FF24C0B601CE0189960E945A5B1C
:10F5B00061EE77E0CE0183960E942957BE01675D18
:10F5C0007F4FCE0183960E94455663E97AE00E9400
:10F5D0002E56BC0181E892E10E94DC55CE01839653
:10F5E0000E94C556CE0189960E94C55648C022E0A9
:10F5F000B301A201CE018F960E94CA56B601CE0178
:10F6000089960E945A5B61EE77E0CE0183960E9454
:10F610002957BE01675D7F4FCE0183960E944556F4
:10F6200069E67BE00E942E56BE01615D7F4F0E941D
:10F630004556BC0185E792E10E94B056CE01839603
:10F640000E94C556CE0189960E94C556CE018F965E
:10F650000E94C55665E772E1CE0183960E9421574C
:10F6600066E67CE0CE0183960E942E56BC0181E8BE
:10F6700092E10E94DC55CE0183960E94C55601306E
:10F68000110559F4E114F10409F05DC061E872E17B
:10F69000CE01C5960E94B05656C00230110511F534
:10F6A00022E0B301A201CE0183960E94CA56BE0198
:10F6B0006D5D7F4FCE0189960E94215766E67CE002
:10F6C000CE0189960E942E56BC01CE01C5960E949D
:10F6D000DC55CE0189960E94C556CE0183960E94C4
:10F6E000C55631C00330110571F165E772E1CE01F5
:10F6F00083960E94215744E150E06FEF7FEFCE01E7
:10F7000083960E944990CE0183960E94C5566AE076
:10F710007AE0CE0183960E942957CE0183960E94FB
:10F72000C590CE0183960E94C55680912E058823F0
:10F7300051F080912D05882331F060ED77E080E075
:10F7400090E00E940189FFEFEF1AFF0A8FEFC81ABD
:10F75000D80A0ECFCE01C5960E941B5581E892E1D2
:10F760000E941B5501151105C9F46FE572E181E88E
:10F7700092E10E94565664E572E1CE0183960E94A2
:10F7800019574AE050E06FEF7FEFCE0183960E9459
:10F790004990CE0183960E94C556EBC004301105F6
:10F7A0000CF000C1BE016B5C7F4FCE0183960E94BE
:10F7B00021574AE050E06FEF7FEFCE0183960E9421
:10F7C0004990CE0183960E94C5566AE07AE0CE0148
:10F7D00083960E942957CE0183960E94C590CE0140
:10F7E00083960E94C556DEC06FE97AE0CE01C596C9
:10F7F0000E949B56BE016B5C7F4FCE0183960E9498
:10F8000021574AE050E060E070E0CE0183960E940C
:10F810009192CE0183960E94C55664E67AE081E813
:10F8200092E10E949B5661E872E1CE01C5960E946A
:10F83000B05600E010E0602FCE0101960E947C5D82
:10F840006B017C0122E0AB01BC01CE018396011566
:10F85000110551F40E94CA56BE016D5D7F4F8CE7C1
:10F8600093E10E94875718C00E94CA56BE016D5D81
:10F870007F4FCE0189960E94215766E67CE0CE013B
:10F8800089960E942E56BC01CE01C5960E94DC5579
:10F89000CE0189960E94C556CE0183960E94C55618
:10F8A00022E0B701A601CE0183960E94CA56BE018E
:10F8B0006D5D7F4FCE0189960E94215766E67CE000
:10F8C000CE0189960E942E56BC0181E892E10E94E9
:10F8D000DC55CE0189960E94C556CE0183960E94C2
:10F8E000C5560F5F1F4F0330110509F0A4CFCE019D
:10F8F000C5960E941B55BE016B5C7F4FCE0183965F
:10F900000E9421574AE050E06FEF7FEFCE018396CF
:10F910000E944990CE0183960E94C5566AE07AE023
:10F92000CE0183960E942957CE0183960E94C590EE
:10F93000CE0183960E94C55681E892E10E941B5534
:10F9400065EA7AE0CE0183960E94295761E872E168
:10F95000CE0183960E9445566FEA7AE00E942E56A9
:10F96000BC0181E892E10E94B056CE0183960E94CC
:10F97000C556CE01C5960E94C556EA960FB6F894B4
:10F98000DEBF0FBECDBFDF91CF911F910F91FF90D2
:10F99000EF90DF90CF90BF90AF907F906F905F908F
:10F9A0004F9008956FEA7AE081E892E10E94CE5587
:10F9B000E0CF85ED8093BC008091BC0084FDFCCF3E
:10F9C0001092760D08954091A913262F30E0240F50
:10F9D000311D21323105DCF42091760D2430C9F43B
:10F9E000FC0180E090E0861758F43091A913219132
:10F9F000DC01A757BC4EA30FB11D2C930196F3CF8A
:10FA00008091A913680F6093A91380E0089581E0A5
:10FA1000089582E00895089508950895E091F613F9
:10FA20008091F513E81730F4F0E0E950FC4E808146
:10FA300090E008958FEF9FEF08959091F6138091D5
:10FA4000F513981750F4E92FF0E0E950FC4E2081AF
:10FA500030E09F5F9093F61302C02FEF3FEFC90194
:10FA600008958091F51390E02091F613821B91097F
:10FA70000895CF92DF92EF92FF920F931F93CF934F
:10FA8000DF937C01CB018A012091770D222389F03D
:10FA9000EB016B01C40ED51ECC15DD0561F069913B
:10FAA000D701ED91FC910190F081E02DC7011995EE
:10FAB000F3CF642F88DFC801DF91CF911F910F91A1
:10FAC000FF90EF90DF90CF900895CF93DF931F9238
:10FAD000CDB7DEB769832091770D2223D1F0209135
:10FAE000990D203240F021E030E0FC013383228385
:10FAF00080E090E014C08091780DE82FF0E0E758A6
:10FB0000F24F998190838F5F8093780D8093990D48
:10FB100004C061E0CE01019656DF81E090E00F90D5
:10FB2000DF91CF91089580E090E008950C94DDB6C8
:10FB3000FC0190810180F281E02DF8948181892B74
:10FB400081832281892F809528232283A7E0B0E03A
:10FB50001197F1F7218182238183A3E2B0E011970D
:10FB6000F1F780817894EFECF0E03197F1F798238A
:10FB700081E009F480E00895FC0190810180F28128
:10FB8000E02D892F809560FF12C0F8942281822396
:10FB900082838181892B8183A3E2B0E01197F1F701
:10FBA0008281982B9283789487ED90E011C0F8942D
:10FBB0002281822382838181892B8183AFEFB0E010
:10FBC0001197F1F78281982B928378948FE090E0DF
:10FBD0000197F1F70895DF92EF92FF920F931F9331
:10FBE000CF93DF93EC01D62EE42E08E010E0FF2443
:10FBF000F39461E08D2D8F2109F460E0CE01BCDF2C
:10FC0000FF0C01501109A9F7E11010C0F894E98127
:10FC1000FA8191818881809589238183E981FA81A4
:10FC2000928188818095892382837894DF91CF9116
:10FC30001F910F91FF90EF90DF900895DC012C91C0
:10FC40001196ED91FC911297F8948181922F9095E5
:10FC50008923818378948DE743E050E0815021F13E
:10FC6000DA011197F1F730813223C1F3F8948281E0
:10FC7000892382838181822B81837894ABE7B7E0EB
:10FC80001197F1F7F89481819823918383E191E0B2
:10FC90000197F1F78081282381E009F080E07894D2
:10FCA000E3E6F6E03197F1F708951F93CF93DF93E2
:10FCB000EC01162F60E0812F0E947B88612F70E09D
:10FCC000FB01E05BFC4EE491E883FB01E65FFC4E48
:10FCD000E491F0E0EE0FFF1FE051FD4E859194910D
:10FCE0009A8389831B861D861C86FE013B9623967C
:10FCF0001292EC17FD07E1F7DF91CF911F91089564
:10FD00001F93CF93DF93EC01162F8C810E942270FA
:10FD10006B85812F862B90E00E941D70DF91CF9123
:10FD20001F910C941B700F931F93CF938C01C62FC0
:10FD3000E7DF6C2F6460C801E3DF6C2F6B7FC801C5
:10FD4000DFDF83EC90E00197F1F7CF911F910F91E6
:10FD500008950F931F93CF938C01C62F607F61602E
:10FD6000E2DF80E1C89FB00111246160C801DBDFE0
:10FD700081E090E0CF911F910F9108951F920F9213
:10FD80000FB60F9211240BB60F922F933F934F9300
:10FD90005F936F937F938F939F93AF93BF93EF93F3
:10FDA000FF9380911B100E94258820911E10309196
:10FDB0001F102F5F3F4F30931F1020931E10909104
:10FDC0001D10953618F096E090931A1090911A1025
:10FDD0009430C9F128F4923069F09330D1F05EC0CC
:10FDE000953009F451C0963009F058C091E09093D5
:10FDF000EA1051C0811152C020911E1030911F1085
:10FE00002436310508F442C01092EA1010921D10F9
:10FE10001CC0813009F042C0E0911D1091E09E0F9E
:10FE200090931D10F0E020911E1030911F10EE0FE6
:10FE3000FF1FE05EFF4E3183208310921F1010924F
:10FE40001E1094E029C0811117C0E0911D1091E0AF
:10FE50009E0F90931D10F0E020911E1030911F1006
:10FE6000EE0FFF1FE05EFF4E3183208310921F10C4
:10FE700010921E1093E010C020911E1030911F10A0
:10FE80002536310558F007C0811108C010921F10A7
:10FE900010921E1003C095E090931A1090911C10C0
:10FEA000992329F0811102C02F9A01C02F98FF9148
:10FEB000EF91BF91AF919F918F917F916F915F91E2
:10FEC0004F913F912F910F900BBE0F900FBE0F904F
:10FED0001F901895CF92DF92EF92FF92CF93DF930E
:10FEE000EC01072E000C880B990B0E942EB16B01C0
:10FEF0007C0120E030E040E45FE30E948DB120E02F
:10FF000030E048E452E40E947EB30E9417B4C61762
:10FF1000D707D4F020E030E040EA5FE3C701B60144
:10FF20000E948DB120E030E048E452E40E947EB3AC
:10FF300020E030E040E85FE30E94B8B20E9417B4CE
:10FF400021E06C177D070CF420E0822F90E0DF9118
:10FF5000CF91FF90EF90DF90CF9008950F931F9374
:10FF6000CF93DF93082F63E476E081E79FE00E9460
:10FF70006058C7E0D0E010E0B8010C2E02C07595C3
:10FF800067950A94E2F76170772742E050E081E7D5
:10FF90009FE00E941658219778F7DF91CF911F912B
:10FFA0000F9108951F920F920FB60F9211240BB666
:10FFB0000F922F933F934F935F936F937F938F9302
:10FFC0009F93AF93BF93EF93FF938091B900887F86
:10FFD000803609F49CC068F5883209F45BC090F45F
:10FFE000803109F454C038F4882309F4F6C088300D
:10FFF00009F44DC0F5C0883109F44CC0803209F4D1
:020000021000EC
:100000005DC0EEC0803409F468C048F4803309F460
:1000100055C0883309F0E4C08093740DD8C0803592
:1000200009F44FC0883509F45DC0883409F0D8C0A0
:10003000D6C0883909F4C7C0A8F4883709F467C066
:1000400038F4883609F463C0803709F460C0C8C04A
:10005000883809F4B8C0803909F45FC0803809F0E5
:10006000BFC05BC0803B09F486C038F4803A09F415
:1000700066C0883A09F47FC0B3C0803C09F4A7C0C9
:10008000883C09F4A4C0883B09F48AC0A9C08091C7
:10009000510D10C09091730D8091720D981770F5ED
:1000A000E091730D81E08E0F8093730DF0E0EE5AB6
:1000B000F24F80818093BB0085EC86C08093740DE5
:1000C0008EC0E091730D81E08E0F8093730D80914F
:1000D000BB00F0E0EE5AF24F80839091730D809157
:1000E000720D6EC0E091730D81E08E0F8093730DE1
:1000F0008091BB00F0E0EE5AF24F80838091750D45
:1001000081116DC081E08093500D84EA61C083E06D
:100110008093760D1092CB13CFCF8091CB1380328A
:1001200008F051C0E091CB1381E08E0F8093CB1388
:100130008091BB00F0E0E555FC4E8083BDCF85EC9F
:100140008093BC001092760D8091CB13803230F4F6
:10015000E091CB13F0E0E555FC4E10826091CB139B
:1001600070E0E091E40CF091E50C8BEA93E11995D5
:100170001092CB1335C084E08093760D1092AA13B1
:100180001092A913E091E60CF091E70C199580917B
:10019000A913811105C081E08093A91310928913DE
:1001A000E091AA1381E08E0F8093AA13F0E0E75745
:1001B000FC4E80818093BB009091AA138091A9137B
:1001C000981708F479CF85E88093BC0009C085ECC6
:1001D0008093BC001092760D03C01092740DE9DB81
:1001E000FF91EF91BF91AF919F918F917F916F910F
:1001F0005F914F913F912F910F900BBE0F900FBECB
:100200000F901F9018950895ECEEF0E114A215A23E
:1002100016A217A210A611A612A613A681E084A703
:1002200029E130E036A725A787A780E090E0A0EA83
:10023000B0E480AB91ABA2ABB3AB80E090E0A8EAB6
:10024000B1E484AB95ABA6ABB7AB8093250290939A
:100250002602A0932702B093280280E090E0A0E855
:10026000BFE38093361190933711A0933811B09368
:1002700039118093210290932202A0932302B0931C
:10028000240210926311109262118BE090E090931F
:1002900065118093641190932A0280932902109231
:1002A000C80C1092C70C80E090E00C946A74AF9276
:1002B000BF92CF92DF92EF92FF920F931F93CF9353
:1002C000DF93CDB7DEB7A4970FB6F894DEBF0FBEAD
:1002D000CDBF8091CC13882319F01092CC138EC51A
:1002E00080919D1290919E12049708F03FC067E2A2
:1002F00078E0CE0101960E942957BE016F5F7F4FC3
:1003000089E992E16ED6182FCE0101960E94C5565A
:10031000112361F161E070E089E992E10E947B556F
:1003200080330CF4845E6AE270E0681B710987FD1B
:100330007395CE0101960E945A5BBE016F5F7F4F9D
:1003400089E992E10E94E255CE0101960E94C556CC
:1003500069E972E18DE892E10E94B05689E992E183
:100360000E941055CB010E94D70A48C566E777E086
:10037000CE0107960E942957BE01695F7F4F89E928
:1003800092E12FD6811115C06CE777E0CE0101967E
:100390000E942957BE016F5F7F4F89E992E121D604
:1003A00011E0811101C010E0CE0101960E94C556F6
:1003B00001C011E0CE0107960E94C556112309F431
:1003C00082C362EC7AE0CE0101960E942957CE01E9
:1003D00001960E94586ACE0101960E94C5566EECA5
:1003E0007AE0CE0107960E94295760E773E1CE01BB
:1003F00007960E944556BC01CE0101960E942157E6
:10040000CE0101960E94586ACE0101960E94C556FF
:10041000CE0107960E94C556609143027091440236
:1004200080914502909146020E942EB120E030E07A
:1004300048EC52E40E947EB3AB01BC0122E0CE0145
:1004400007960E94CA5664EE7AE0CE010D960E948D
:100450002957BE01695F7F4FCE010D960E94455618
:1004600064E978E00E942E56BC01CE0101960E94FC
:100470002157CE0101960E94586ACE0101960E9432
:10048000C556CE010D960E94C556CE0107960E9414
:10049000C55640913F0250914002609141027091D7
:1004A000420224E0CE0107960E94CA5669EF7AE024
:1004B000CE010D960E942957BE01695F7F4FCE0184
:1004C0000D960E944556BC01CE0101960E9421570F
:1004D000CE0101960E94586ACE0101960E94C5562F
:1004E000CE010D960E94C556CE0107960E94C556B4
:1004F000409133025091340260913502709136027E
:1005000022E0CE0107960E94CA5640912B025091DC
:100510002C0260912D0270912E0223E0CE010D96E7
:100520000E94CA56409137025091380260913902B8
:1005300070913A0222E0CE0143960E94CA56409141
:100540002F0250913002609131027091320223E00B
:10055000CE0149960E94CA5666E17BE0CE014F96D5
:100560000E942957BE01675E7F4FCE014F960E94C1
:1005700045566BE27BE00E942E56BE016D5E7F4FBA
:100580000E9445566EE27BE00E942E56BE01635FDC
:100590007F4F0E9445566BE27BE00E942E56BE01C3
:1005A000695F7F4F0E94455664E37BE00E942E56B0
:1005B000BC01CE0101960E942157CE0101960E94F6
:1005C000586ACE0101960E94C556CE014F960E94F0
:1005D000C556CE0149960E94C556CE0143960E944B
:1005E000C556CE010D960E94C556CE0107960E94B3
:1005F000C5566BEA72E1CE0149960E941957F090F8
:100600001B110F2D0F2C000C110B01151105A1F55D
:1006100020911C1130911D1140911E1150911F11FC
:1006200060E070E080EA90E40E947EB3AB01BC0120
:1006300022E0CE0101960E94CA566FEF78E0CE010B
:1006400007960E942957BE016F5F7F4FCE01079624
:100650000E94455668E679E00E942E56BC01CE0104
:1006600049960E94DC55CE0107960E94C556CE01E0
:1006700001960E94C55609C00130110531F46DE99B
:1006800072E1CE0149960E948C55C80102970297EB
:1006900038F58F2D9AE08902B0011124CE01019620
:1006A0000E945A5B69E37BE0CE0107960E942957BE
:1006B000BE016F5F7F4FCE0107960E94455661E6EF
:1006C00079E00E942E56BC01CE0149960E94DC556D
:1006D000CE0107960E94C556CE0101960E94C556CE
:1006E0000430110519F46BE872E105C005301105FD
:1006F00034F063E872E1CE0149960E948C55BE0148
:10070000675E7F4FCE0101960E942157CE01019670
:100710000E94586ACE0101960E94C55665E47BE0AE
:10072000CE0149960E949B56809118116091191133
:1007300070911A1183300CF04FC3CE0101960E94C4
:100740005A5B60E47BE0CE0107960E942957BE0108
:100750006F5F7F4FCE0107960E94455667E47CE0AD
:100760000E942E56BC01CE0149960E94DC55CE0156
:1007700007960E94C556CE0101960E94C556BE013D
:10078000675E7F4FCE0101960E942157CE010196F0
:100790000E94586ACE0101960E94C55640912011D0
:1007A00050912111609122117091231122E0CE010C
:1007B00007960E94CA5665E57BE0CE010D960E9421
:1007C0002957BE01695F7F4FCE010D960E944556A5
:1007D0006BE67BE00E942E56BC01CE0101960E9482
:1007E0002157CE0101960E94586ACE0101960E94BF
:1007F000C556CE010D960E94C556CE0107960E94A1
:10080000C556409136115091371160913811709151
:10081000391122E0CE0107960E94CA5662E77BE0BA
:10082000CE010D960E942957BE01695F7F4FCE0110
:100830000D960E94455660ED75E00E942E56BC0153
:10084000CE0101960E942157CE0101960E94586A5E
:10085000CE0101960E94C556CE010D960E94C55646
:10086000CE0107960E94C55689E0C82E82E0D82E98
:1008700001E010E099E1F92E8091070290910802C1
:10088000801791070CF44DC0F601A190B1906F0153
:10089000B501CE0107960E945A5BB801CE010D96B4
:1008A0000E945A5B65E87BE0CE0143960E9429577F
:1008B000BE01635F7F4FCE0143960E9445566DE8AF
:1008C0007BE00E942E56BE01695F7F4F0E94455615
:1008D00060E97BE00E942E56FA9CB001FB9C700DF3
:1008E000112465547D4F0E942E56BC01CE01019605
:1008F0000E942157CE0101960E94586ACE010196AE
:100900000E94C556CE0143960E94C556CE010D9653
:100910000E94C556CE0107960E94C5560F5F1F4F15
:10092000ABCF8091621190916311892B71F466E9CC
:100930007BE0CE0101960E942957CE0101960E94CC
:10094000586ACE0101960E94C5568091621190911D
:100950006311019771F465EA7BE0CE0101960E9474
:100960002957CE0101960E94586ACE0101960E9435
:10097000C5568091621190916311029771F46FEAEC
:100980007BE0CE0101960E942957CE0101960E947C
:10099000586ACE0101960E94C55660912902709155
:1009A0002A02CE0107960E945A5B61EC7BE0CE01E1
:1009B0000D960E942957BE01695F7F4FCE010D96AB
:1009C0000E944556BC01CE0101960E942157CE01DE
:1009D00001960E94586ACE0101960E94C556CE012A
:1009E0000D960E94C556CE0107960E94C5564091AD
:1009F000500250915102609152027091530222E0D4
:100A0000CE0107960E94CA566EED7BE0CE010D9690
:100A10000E942957BE01695F7F4FCE010D960E944B
:100A200045566EED75E00E942E56BC01CE01019632
:100A30000E942157CE0101960E94586ACE0101966C
:100A40000E94C556CE010D960E94C556CE0107964E
:100A50000E94C5564091550250915602609157022E
:100A60007091580222E0CE0107960E94CA566EEE9F
:100A70007BE0CE010D960E942957BE01695F7F4F32
:100A8000CE010D960E9445566EED75E00E942E56E1
:100A9000BC01CE0101960E942157CE0101960E9411
:100AA000586ACE0101960E94C556CE010D960E944D
:100AB000C556CE0107960E94C55610925402CE012B
:100AC00049960E94C55680919D1290919E12833046
:100AD000910508F06FC18130910541F460E070E04C
:100AE00089E992E10E947B55E82E57C0029709F0F0
:100AF00054C067E278E0CE0101960E942957BE01FA
:100B00006F5F7F4F89E992E16CD2182FCE01019679
:100B10000E94C556112309F440C061E070E089E9E4
:100B200092E10E947B55682FCE0101960E94F956F2
:100B3000BE016F5F7F4F8DE892E10E94E255CE01CA
:100B400001960E94C55660E070E089E992E10E943A
:100B50007B55E82E80911F148823F9F06EEF7BE01F
:100B6000CE0101960E94295769E972E1CE010196F2
:100B70000E94455666E67CE00E942E56BC0181E745
:100B80009FE00E948757CE0101960E94C5566DE8EE
:100B900072E181E79FE00E94AE6F8E2DEE0C990B03
:100BA0000E944AB8892BB1F00E94BE740E94A141F4
:100BB00066E67CE0CE0101960E9429574AE050E0AB
:100BC00060E070E0CE0101960E943693CE0101965E
:100BD0000E94C55669E972E1CE0107960E9421572D
:100BE00060E070E0CE0107960E947B55823409F4E4
:100BF00074C0D4F4803309F490C07CF4833209F4D7
:100C000083C08A3209F0A9C067E17CE089E992E1FA
:100C10000E949B568FEF9FEF8EC0813309F48EC0E8
:100C2000813409F44FC099C0813609F44BC034F4C3
:100C3000833409F45DC0843449F08FC0833609F4ED
:100C400057C00CF44AC0843609F087C080919112D5
:100C500090919212892B09F49FC061E070E0CE015F
:100C600007960E947B55182F80911F14882361F0EE
:100C700064E07CE081E79FE00E9460586DE872E1EB
:100C800081E79FE00E94AE6F10330CF4145E6AE2BD
:100C900070E0611B710917FD7395CE0101960E94EA
:100CA0005A5BBE016F5F7F4F8DE892E10E94E25573
:100CB000CE0101960E94C5568DE892E10E94105522
:100CC000CB0139C06BE07CE089E992E10E949B5640
:100CD0008091970C9091980C2EC06EE07CE089E991
:100CE00092E10E949B561092D30C8CEF9FEF23C091
:100CF00061E17CE089E992E10E949B5681E080936A
:100D0000D30C8DEF9FEF17C064E17CE089E992E19D
:100D10000E949B568EEF9FEF0EC064EE79E08DE847
:100D200092E10E949B5664EE79E089E992E10E948B
:100D30009B5680E090E00E94D70A2EC068E17CE0DC
:100D40008DE892E10E949B5668E17CE089E992E19E
:100D50000E949B5681E090E0EECFBE01695F7F4F1D
:100D60008DE892E10E94B05660E070E08DE892E17B
:100D70000E947B55082E000C990BC0970A9738F4F7
:100D80008DE892E10E941055CB010E94D70A64E6DB
:100D900070E080E090E035D2CE0107960E94C55603
:100DA0008CD36093C90C7093CA0C8093CB0C909336
:100DB000CC0C02C00E94A72480D36093C90C70930E
:100DC000CA0C8093CB0C9093CC0C64E67AE089E952
:100DD00092E10E949B5612C0CE0101960E945A5B7E
:100DE0006AE17CE0CE0107960E942957BE016F5F41
:100DF0007F4FCE0107960E944556B4CCA4960FB6FD
:100E0000F894DEBF0FBECDBFDF91CF911F910F9140
:100E1000FF90EF90DF90CF90BF90AF90089590E05B
:100E2000FC013197E231F10508F04EC08827E85502
:100E3000FF4F8F4F0C9406B6809180008F7703C0D0
:100E4000809180008F7D8093800008958091800044
:100E5000877FF9CF84B58F7702C084B58F7D84BD3D
:100E600008958091B0008F7703C08091B0008F7D8E
:100E70008093B0000895809190008F7707C0809193
:100E800090008F7D03C080919000877F80939000B9
:100E900008958091A0008F7707C08091A0008F7D7A
:100EA00003C08091A000877F8093A0000895809167
:100EB00020018F7707C0809120018F7D03C0809132
:100EC0002001877F809320010895CF93DF93FC0159
:100ED00024813581232B71F0FB01DC01CD91DC9164
:100EE00060817181CE010E9499B8009719F08C1B26
:100EF0009D0B02C08FEF9FEFDF91CF9108950F936D
:100F00001F93CF93DF93FC01C481D581209719F4FF
:100F1000FB01108211C0415051094C175D0708F4C4
:100F2000EA018B01FC0160817181AE01C8010E9460
:100F30008AB8C00FD11F1882DF91CF911F910F91F6
:100F40000895AF92BF92CF92DF92EF92FF920F93EC
:100F50001F93CF93DF93FC0124813581FB014481F2
:100F600055818901041B150B4115510551F12115BE
:100F7000310539F12417350720F10217130718F04E
:100F80008901015011097B01FC01A080B180C501DC
:100F9000DFEFCFEF6501C00ED11EC816D906A0F055
:100FA000F701608171810E9499B8009769F09C01F6
:100FB0002A193B090217130710F0D22FC32F0196ED
:100FC000ECCF8FEF9FEF02C08D2F9C2FDF91CF9141
:100FD0001F910F91FF90EF90DF90CF90BF90AF9057
:100FE0000895FB0144815581FC012481358124173A
:100FF000350778F080819181009759F0FB0160817D
:1010000071816115710529F00E947CB821E0892B5E
:1010100009F020E0822F0895FC01A089B1898C910C
:10102000A689B78982FD0FC09C91818D8F5F8F73D8
:10103000228D821749F0218DDF01A20FB11D5D962F
:101040009C93818F08958C910895CF93DF93282FDF
:1010500030E0F901EA56FC4E8491F901E05BFC4E68
:10106000D491F901E65FFC4EC491CC2389F0811143
:10107000D6DEEC2FF0E0EE0FFF1FE051FD4EA59104
:10108000B491EC91ED2381E090E021F480E002C086
:1010900080E090E0DF91CF9108951F93CF93DF938D
:1010A000282F30E0F901EA56FC4E8491F901E05B0B
:1010B000FC4ED491F901E65FFC4EC491CC23B9F00B
:1010C000162F8111ACDEEC2FF0E0EE0FFF1FEA527D
:1010D000FD4EA591B4919FB7F894111104C08C9165
:1010E000D095D82302C0EC91DE2BDC939FBFDF911B
:1010F000CF911F910895CF93DF9390E0FC01E05BC7
:10110000FC4E2491FC01E65FFC4E8491882361F142
:1011100090E0880F991FFC01E454FD4EC591D491D5
:10112000FC01EA52FD4EA591B491611109C09FB72F
:10113000F8948881209582238883EC912E230BC01C
:10114000623061F49FB7F8948881322F3095832301
:101150008883EC912E2B2C939FBF06C08FB7F894F9
:10116000E8812E2B28838FBFDF91CF91089586339E
:1011700008F0865390917B00282F2870977F922B40
:1011800090937B0020912C0590E4299F90011124DD
:101190008770822B80937C0080917A00806480939A
:1011A0007A0080917A0086FDFCCF809178002091B2
:1011B000790090E0922B08953FB7F8948091D11375
:1011C0009091D213A091D313B091D41326B5A89BBC
:1011D00005C02F3F19F00196A11DB11D3FBFBA2FC9
:1011E000A92F982F8827820F911DA11DB11DBC0129
:1011F000CD0142E0660F771F881F991F4A95D1F7EE
:1012000008958F929F92AF92BF92CF92DF92EF920A
:10121000FF926B017C01D0DF4B015C01C114D10452
:10122000E104F104E9F0C8DFDC01CB018819990978
:10123000AA09BB09883E9340A105B10578F321E0D6
:10124000C21AD108E108F10888EE880E83E0981EE2
:10125000A11CB11CC114D104E104F10421F7DECFBB
:10126000FF90EF90DF90CF90BF90AF909F908F90C6
:101270000895FF920F931F93CF93DF93CDB7DEB7FF
:101280002B970FB6F894DEBF0FBECDBF84ED9EE066
:101290009AD740E855E260E070E084ED9EE00E945D
:1012A000B77364E670E080E090E0ABDF8CED95E032
:1012B000A0E0B0E08093D80E9093D90EA093DA0E00
:1012C000B093DB0E64E670E080E090E09ADF8FEF91
:1012D000898381E08A8386E88B831C821D821E823B
:1012E0001F82188689E7898784ED9EE00E941D533E
:1012F00062E370E080E090E084DF84ED9EE00E9495
:101300004E5208974CF049E050E0BE016F5F7F4FAE
:1013100084ED9EE00E94245262E370E080E090E061
:1013200070DF84ED9EE00E947F52892B01F184EDF5
:101330009EE00E944E52089784F465E070E080E0E1
:1013400090E05FDF00E010E0F12C84ED9EE00E9471
:101350007F5202301105A4F50CC049E050E0BE01F7
:101360006F5F7F4F84ED9EE00E942452E6CFF12C08
:1013700027C084ED9EE00E947F52892B99F465E09E
:1013800070E080E090E03DDF02301105F1F69A85D3
:1013900089819813DACF9B858B819813D6CFFF2450
:1013A000F394D3CF84ED9EE00E945D52EAE0F0E03A
:1013B000EC0FFD1FE00FF11F80830F5F1F4FDFCF8A
:1013C00062E370E080E090E01CDF84ED9EE0FBD6FD
:1013D0008F2D2B960FB6F894DEBF0FBECDBFDF91D9
:1013E000CF911F910F91FF900895CF93DF930E94AB
:1013F000285B1092811380918513823018F098E059
:101400009093811390918613992339F0813029F4B8
:101410008091811384608093811362E370E080E0A7
:1014200090E0EFDE609187138CE793E10E94807E6D
:1014300068EE73E080E090E0E4DE60E38CE793E147
:101440000E94937ECBE4D6E4CE010197F1F760E3EE
:101450008CE793E10E94937E2197F1F760E38CE79C
:1014600093E10E94937E83E592E00197F1F760E2B9
:101470008CE793E10E94937E8091811380620E94A9
:101480002C7084E0809382138CE00E942C7081E0A9
:101490000E942C70CBE3DFE1CE010197F1F782E0EF
:1014A0008093831386E00E942C7082E00E942C704F
:1014B0002197F1F7DF91CF9108952FB7F8946091BC
:1014C000CD137091CE138091CF139091D0132FBF75
:1014D00008952F923F924F925F926F927F928F92D8
:1014E0009F92AF92BF92CF92DF92EF92FF920F93B3
:1014F0001F93CF93DF93CDB7DEB766970FB6F894FF
:10150000DEBF0FBECDBF7C016D8B7E8B5C8B4B8BAA
:10151000190164E67AE00E9429578EE1882E912C09
:101520008E010F5F1F4F2101032C000C6608770806
:10153000CD88DE88A12CB12CA214B3040CF07BC0A2
:10154000B501CE010D960E945A5BBE01635F7F4FCD
:10155000CE0107960E94215769E177E0CE010796F8
:101560000E942E566B897C890E944556B6010E94C6
:101570004556BC01C8010E94215740ED57E060E08C
:1015800070E0C80186D5C8010E94C556CE010796F5
:101590000E94C556CE010D960E94C55644E150E00A
:1015A00061E070E0C8010E94DF5F0E151F0521F0A9
:1015B000B801C7010E94E255C8010E94C556F70153
:1015C00084819581892BA9F160E070E0C7010E94B8
:1015D0007B55082E000C990BC0970A9740F4C70161
:1015E0000E94105564157505860597054CF06AE054
:1015F0007AE0F701808191810E946CB8892B59F4BF
:1016000081E0FFEFAF1ABF0A96E0C90ED11C882314
:1016100009F492CF15C06CED73E1C8010E9419570F
:1016200040ED57E060E070E0C80133D5C8010E948A
:10163000C55680E0E6CFE1E08E1A910809F078CF38
:10164000C70166960FB6F894DEBF0FBECDBFDF911F
:10165000CF911F910F91FF90EF90DF90CF90BF90AF
:10166000AF909F908F907F906F905F904F903F9042
:101670002F900895CF93DF93EC01483085E0580711
:101680006105710509F441C108F08DC0493481E05C
:1016900058076105710509F43BC1E0F5443481E068
:1016A00058076105710509F424C1E8F4413481E06B
:1016B00058076105710509F413C138F440345140ED
:1016C0006105710509F409C135C1423481E058074B
:1016D0006105710509F407C1433451406105710585
:1016E00009F404C127C1463481E05807610571053A
:1016F00009F405C108F400C1473481E058076105C9
:10170000710509F4FFC0483451406105710509F4C1
:10171000FCC010C1423085E058076105710509F42D
:10172000E2C0E8F4443781E058076105710509F427
:10173000F5C038F4423751406105710509F4F1C034
:10174000F9C0411585E058076105710509F4C5C068
:10175000413055406105710509F4C2C0EBC0453008
:1017600085E058076105710509F4C6C070F443307F
:1017700085E058076105710509F4B8C0443055404B
:101780006105710509F4B5C0D5C0463085E058073C
:101790006105710509F4B3C0473055406105710515
:1017A00009F4B0C0C7C04D3B82E458078FEF68070B
:1017B000710509F4BCC008F045C04F3E80E15807F0
:1017C0008FEF6807710509F49DC0E8F4423385E0A6
:1017D00058076105710509F4A4C038F44930554033
:1017E0006105710509F494C0A5C0443385E058072C
:1017F0006105710509F492C04D3F52406F4F71056C
:1018000009F48FC097C04D3D82E258078FEF6807FB
:10181000710509F483C038F4473E58416F4F710594
:1018200009F46AC087C04F3C80E358078FEF680710
:10183000710509F45EC0473C58436F4F710509F4C8
:1018400064C078C0473988E658078FEF680771058C
:1018500009F446C000F54D3A82E558078FEF680756
:10186000710509F461C030F4453B5A446F4F71056E
:10187000A1F160C0453A8AE558078FEF6807710506
:1018800009F446C04D3952466F4F710509F052C0F8
:101890006AE07AE051C0473588EA58078FEF680759
:1018A0007105C9F168F445388AE758078FEF680772
:1018B000710529F1473658496F4F7105A1F03AC0BB
:1018C0004F3480EB58078FEF6807710579F04D337F
:1018D000524C6F4F710529F12DC064EE79E02CC098
:1018E00068E17CE029C065E17CE026C062E17CE043
:1018F00023C06FE07CE020C06CE07CE01DC063E2B0
:101900007CE01AC060E67AE017C065E27CE014C0B3
:1019100067E27CE011C067E278E00EC063E476E045
:101920000BC061E679E008C06FE979E005C069E2C3
:101930007CE002C064E67AE0CE010E942957CE0125
:10194000DF91CF9108954F925F926F927F928F9225
:101950009F92AF92BF92EF92FF920F931F93CF93FC
:10196000DF93CDB7DEB762970FB6F894DEBF0FBE38
:10197000CDBF7C015B0185EE93E10E94F71D892BB1
:1019800031F464E67AE0C7010E94295728C14091EA
:10199000E9135091EA136091EB137091EC13CE01AF
:1019A000079668DE80911F14882359F16BE27CE072
:1019B000CE0101960E942957BE01695F7F4FCE017B
:1019C00001960E94455669E177E00E942E56BC01BF
:1019D00081E79FE00E948757CE0101960E94C5567D
:1019E0004091E9135091EA136091EB137091EC135D
:1019F00020E181E79FE00E94CE5781E79FE00E94AF
:101A0000AA6F60E070E0CE0107960E947B55182F08
:101A10008A3211F01092CC1350DD6093C90C709390
:101A2000CA0C8093CB0C9093CC0C64E67AE0CE0188
:101A30000D960E942957812F110F990BC0970A9775
:101A400008F05CC0CE0107960E9410556330710506
:101A5000810591050CF094C001E010E082E0982E21
:101A60000A151B050CF08CC06CE271E080E090E080
:101A7000C8DB90921A1010921D10412C512C32018B
:101A800085ED93E10E94F71D892B41F48EE1481604
:101A900051046104710409F08CC01CC08EE1481629
:101AA000510461047104B1F04091D9135091DA13DB
:101AB0006091DB137091DC13CE010196DBDDBE017A
:101AC0006F5F7F4FCE010D960E94E255CE010196C9
:101AD0000E94C55689899A89892B39F0BE01635FB6
:101AE0007F4FCE0107960E94DC550F5F1F4F64E6C3
:101AF0007AE0CE010D960E949B56B2CF6CE271E067
:101B000080E090E07EDB82E080931A1010921D103E
:101B1000812C912C540185ED93E10E94F71D892BB6
:101B200041F48EE188169104A104B10409F04CC07F
:101B30001CC08EE188169104A104B104B1F040915B
:101B4000D9135091DA136091DB137091DC13CE013D
:101B5000019690DDBE016F5F7F4FCE010D960E9412
:101B6000E255CE0101960E94C55689899A89892B32
:101B700039F0BE01635F7F4FCE0107960E94DC55AE
:101B800064E670E080E090E03CDB82E080931A1035
:101B900010921D10BE01695F7F4FC7010E9411574F
:101BA000CE010D960E94C556CE0107960E94C556DD
:101BB00016C06EE170E080E090E023DB8FEF481A02
:101BC000580A680A780A5CCF6EE170E080E090E025
:101BD00018DB8FEF881A980AA80AB80A9CCFC701A9
:101BE00062960FB6F894DEBF0FBECDBFDF91CF91E6
:101BF0001F910F91FF90EF90BF90AF909F908F90AB
:101C00007F906F905F904F900895AF92BF92CF9268
